:100000000C941D080C9445080C9445080C94450864
:100010000C9445080C9445080C9445080C9445082C
:100020000C94EE0B0C9445080C9445080C94450870
:100030000C9445080C9445080C9445080C9445080C
:100040000C9445080C9445080C94ED630C944508F9
:100050000C94DD680C9424690C9445080C944508B4
:100060000C9445080C9445080C943E620C94450889
:10007000485454502F312E3020323030204F4B0D09
:100080000A436F6E74656E742D547970653A2074EE
:100090006578742F68746D6C0D0A507261676D61BC
:1000A0003A206E6F2D63616368650D0A4163636575
:1000B00073732D436F6E74726F6C2D416C6C6F7720
:1000C0002D4F726967696E3A202A0D0A0D0A0048A1
:1000D0005454502F312E3020323030204F4B0D0AE7
:1000E000436F6E74656E742D547970653A2061703B
:1000F000706C69636174696F6E2F6A736F6E0D0A3D
:10010000436F6E6E6E656374696F6E3A20636C6FD9
:1001100073650D0A4163636573732D436F6E74726B
:100120006F6C2D416C6C6F772D4F726967696E3AF9
:10013000202A0D0A0D0A003C6D657461206E616D08
:10014000653D76696577706F727420636F6E746554
:100150006E743D2277696474683D363430223E0DFA
:100160000A00485454502F312E302034303120555D
:100170006E617574686F72697A65640D0A436F6E9B
:1001800074656E742D547970653A20746578742F97
:1001900068746D6C0D0A0D0A3C68313E34303120B4
:1001A000556E617574686F72697A65643C2F683149
:1001B0003E0077696E646F772E6C6F636174696F50
:1001C0006E3D222F223B3C2F7363726970743E0A8E
:1001D000006376007670006D7000647000637000DC
:1001E000677000766F00636F00736E007073007647
:1001F00073006373007672006372006A6F006A6E48
:10020000006A70006A63006A73006A6C00646C00C4
:1002100073750063750024460024460024463C7331
:1002200063726970743E2446005D002C24530024E0
:10023000530024465B0024440024460024463C6DC1
:1002400065746120687474702D65717569763D22DE
:10025000726566726573682220636F6E74656E7472
:100260003D22313B2075726C3D2F223E005D2C22D9
:100270006E73746174696F6E73223A24447D002C2E
:10028000002444007B22736E223A5B002446002443
:10029000463C7363726970743E616C6572742822A7
:1002A0004F7074696F6E732076616C75657320731F
:1002B000617665642E22293B24460024463C736304
:1002C000726970743E616C65727428224E65772085
:1002D00070617373776F726473206D757374206DC2
:1002E000617463682122293B77696E646F772E6C95
:1002F0006F636174696F6E3D222F766F223B3C2FD6
:100300007363726970743E0A0024463C73637269B9
:1003100070743E616C65727428224E65772070613E
:100320007373776F7264207365742E22293B2446A1
:100330000024463C7363726970743E616C6572742C
:10034000282256616C756573206F7574206F662066
:10035000626F756E642122293B77696E646F772E18
:100360006C6F636174696F6E3D222F766F223B3C28
:100370002F7363726970743E0A0024463C73637283
:100380006970743E616C657274282253637269707F
:10039000742075726C2073617665642E22293B246B
:1003A000460024463C7363726970743E24460052D2
:1003B00065626F6F74696E672E2E2E0024463C6D49
:1003C00065746120687474702D65717569763D225D
:1003D000726566726573682220636F6E74656E74F1
:1003E0003D2224443B2075726C3D2F223E003C731D
:1003F0006372697074207372633D2224452F76699D
:1004000065776F702E6A73223E3C2F73637269703A
:10041000743E0A003C2F7363726970743E0A0030A8
:100420005D3B766172206E6F7074733D24442C6C5A
:100430006F633D222445222C646576743D244C2C48
:10044000747A3D24442C646578703D24442C6D6599
:1004500078703D24443B00222446222C24442C2442
:10046000442C24442C003C7363726970743E7661A2
:1004700072206F7074733D5B0024462446007D003B
:100480002C00222446223A2444007B002446003CCF
:10049000736372697074207372633D2224452F6800
:1004A0006F6D652E6A73223E3C2F736372697074A0
:1004B0003E0A000A766172206C72756E3D5B2444C0
:1004C0002C24442C24442C244C5D3C2F73637269EF
:1004D00070743E0A005B302C305D5D3B0A766172C1
:1004E00020656E3D24442C72643D24442C72733D7F
:1004F00024442C6D6D3D24442C726473743D244C53
:100500002C6D61733D24442C7572733D24442C770B
:100510006C3D24442C697061733D24442C6C6F63E2
:100520003D222445223B005B24442C244C5D2C00BE
:10053000305D3B7661722070733D5B0024442C007B
:10054000766172206E6272643D24442C747A3D247C
:10055000442C73626974733D5B007661722076652A
:10056000723D24442C646576743D244C3B0A00247F
:100570004624463C7363726970743E005B302C30D5
:100580005D5D2C226C72756E223A5B24442C2444EF
:100590002C24442C244C5D7D005B24442C244C5D95
:1005A0002C00305D2C227073223A5B0024442C0016
:1005B0007B2264657674223A244C2C226E6272642B
:1005C000223A24442C22656E223A24442C2272645E
:1005D000223A24442C227273223A24442C226D6D38
:1005E000223A24442C2272647374223A244C2C2222
:1005F0006C6F63223A222445222C22736269747341
:10060000223A5B0024460077696E646F772E6C6F28
:10061000636174696F6E3D222F7670223B3C2F73AD
:1006200063726970743E0A00616C657274282250AE
:10063000726F6772616D202444206D6F6469666912
:10064000656422293B00616C65727428224E6577CF
:100650002070726F6772616D2061646465642E2220
:10066000293B0024463C7363726970743E003C73FE
:100670006372697074207372633D2224452F706C1D
:100680006F7470726F672E6A73223E3C2F736372B1
:100690006970743E0A00305D3B0024442C00766192
:1006A00072206D61736F703D5B00766172207365BF
:1006B000713D24442C6D61733D24442C776C3D24A2
:1006C000442C7364743D24442C6D746F6E3D24443B
:1006D0002C6D746F66663D24442C64657664617984
:1006E0003D24442C6465766D696E3D24442C64641D
:1006F0003D24442C6D6D3D24442C79793D24443BAC
:100700000024463C7363726970743E0024463C7357
:1007100063726970743E77696E646F772E6C6F6375
:100720006174696F6E3D222F7670223B3C2F73639C
:10073000726970743E0A003C2F7363726970743E74
:100740000A3C736372697074207372633D2224459E
:100750002F6D6F6470726F672E6A73223E3C2F7329
:1007600063726970743E0A005D3B002C244400767D
:1007700061722070726F673D5B24442C24442C24EA
:10078000442C24442C24442C24442C2444007661FE
:1007900072206E626F617264733D24442C706964D0
:1007A0003D24442C697061733D24443B002446245D
:1007B000463C7363726970743E003C736372697087
:1007C00074207372633D2224452F766965777072B9
:1007D0006F672E6A73223E3C2F7363726970743E9A
:1007E0000A00244624463C7363726970743E0024F8
:1007F000463C7363726970743E2446003C736372B6
:10080000697074207372633D2224452F7669657781
:10081000726F2E6A73223E3C2F7363726970743E4E
:100820000A00305D3B3C2F7363726970743E0A00AE
:1008300024442C00766172206E626F617264733D95
:1008400024442C6D61733D24442C697061733D24F4
:10085000442C6475723D5B00244624463C736372ED
:100860006970743E005D7D005D005D2C002C2444A9
:10087000005B24442C24442C24442C24442C244465
:100880002C24442C2444007B226E70726F677322E8
:100890003A24442C226E626F61726473223A2444BB
:1008A0002C226D6E70223A24442C227064223A5B12
:1008B000002446003C6872202F3E3C666F726D201B
:1008C0006E616D653D6F6620616374696F6E3D6337
:1008D00075206D6574686F643D6765743E3C703E5D
:1008E0003C623E4A6176617363726970742055524E
:1008F0004C3A3C2F623E203C696E707574207479CE
:1009000070653D746578742073697A653D33322073
:100910006D61786C656E6774683D31323720766141
:100920006C75653D22244522206E616D653D6A73BC
:10093000703E3C2F703E3C703E5365742055524CC7
:10094000207768657265204A6176617363726970A9
:100950007473206172652073746F7265642E204415
:10096000656661756C742069732024533C62722043
:100970002F3E4966206C6F63616C206F6E2075534B
:100980004420636172642C20757365202E202869D1
:100990002E652E20646F74293C2F703E3C703E3CC7
:1009A000623E50617373776F72643A3C2F623E3CD3
:1009B000696E70757420747970653D7061737377BA
:1009C0006F72642073697A653D3130206E616D65A8
:1009D0003D70773E3C696E70757420747970653D2A
:1009E0007375626D69743E3C2F703E3C6872202FB7
:1009F0003E3C2F666F726D3E002446003C2F7363B1
:100A0000726970743E0A005D3B002C2444007064DF
:100A10005B24445D3D5B24442C24442C24442C243E
:100A2000442C24442C24442C244400766172206EEF
:100A300070726F67733D24442C6E626F61726473D1
:100A40003D24442C697061733D24442C6D6E703DCF
:100A500024442C70643D5B5D3B0024463C73637210
:100A60006970743E616C65727428224368616E67B8
:100A700065732073617665642E22293B2446002726
:100A8000275D3B00272453272C0076617220736E6C
:100A9000616D65733D5B00305D3B3C2F7363726934
:100AA00070743E0A3C736372697074207372633DA4
:100AB0002224452F76696577736E2E6A73223E3C39
:100AC0002F7363726970743E0A0024442C00305DF9
:100AD0003B7661722069723D5B0024442C00766194
:100AE00072206D61736F703D5B00766172206E6283
:100AF0006F617264733D24442C6D61786C656E3D4A
:100B000024442C6D61733D24442C697061733D2431
:100B1000443B0024463C7363726970743E005D2C54
:100B2000226D61786C656E223A24447D002C00248D
:100B300044005D2C2269676E6F72655F7261696E39
:100B4000223A5B002C002444005D2C226D61736FFF
:100B500070223A5B002C0022245322007B22736E09
:100B6000616D6573223A5B002446005265636F6EC7
:100B70006E656374696E672E2E2E004E545020539E
:100B8000796E63696E672E2E2E00436F6E6E6563FD
:100B900074696E672E2E2E00446574656374696EE9
:100BA00067207553442E2E2E000001080006040015
:100BB0000145000082000040002000504F535420A7
:100BC000244620485454502F312E300D0A486F735C
:100BD000743A2024460D0A24462453416363657009
:100BE000743A202A2F2A0D0A436F6E74656E742D95
:100BF0004C656E6774683A2024440D0A436F6E7426
:100C0000656E742D547970653A206170706C6963FB
:100C10006174696F6E2F782D7777772D666F726D9F
:100C20002D75726C656E636F6465640D0A0D0A2420
:100C30005300474554202446245320485454502FF1
:100C4000312E300D0A486F73743A2024460D0A2461
:100C5000460D0A0D0A004163636570743A2074659D
:100C600078742F68746D6C00E30004FA00010000D2
:100C7000000166777600747A006E747000646863B1
:100C800070006970310069703200697033006970FA
:100C90003400677731006777320067773300677712
:100CA00034006870300068703100617200657874DB
:100CB0000073657100736474006D6173006D746F0F
:100CC0006E006D746F66007572730072736F0077DB
:100CD0006C00737474006970617300646576696494
:100CE00000636F6E006C69740064696D006E7470EF
:100CF00031006E747032006E747033006E74703434
:100D0000007265736574004669726D776172652063
:100D10007665722E0054696D65207A6F6E653A00B3
:100D20004E54502073796E633F00557365204448DC
:100D300043503F005374617469632E6970313A0007
:100D40005374617469632E6970323A00537461742C
:100D500069632E6970333A005374617469632E6954
:100D600070343A00476174657761792E6970313A61
:100D700000476174657761792E6970323A00476186
:100D800074657761792E6970333A004761746577CD
:100D900061792E6970343A004854545020706F7253
:100DA000743A00004175746F207265636F6E6E65F2
:100DB00063743F0023206F66206578702E20626F79
:100DC0006172643A0053657175656E7469616C2077
:100DD0006D6F64653F0053746174696F6E20646564
:100DE0006C61793A004D617374657220737461743B
:100DF000696F6E3A004D617374657220206F6E20CA
:100E000061646A2E3A004D6173746572206F666684
:100E10002061646A2E3A00557365207261696E2004
:100E200073656E736F723A004E6F726D616C6C79A0
:100E3000206F70656E3F00252057617465722074C5
:100E4000696D653A0053656C6674657374207469E6
:100E50006D653A0049676E6F7265207061737377D4
:100E60006F72643F004465766963652049443A00C7
:100E70004C434420436F6E74726173743A004C4368
:100E800044204261636B6C696768743A004C434468
:100E90002044696D6D696E673A004E545020736549
:100EA000727665722E6970313A004E545020736527
:100EB000727665722E6970323A004E545020736516
:100EC000727665722E6970333A004E545020736505
:100ED000727665722E6970343A00526573657420BB
:100EE000616C6C3F004D6F6E005475650057656412
:100EF0000054687500467269005361740053756E42
:100F000000206D696E00207365630025004E6F0040
:100F1000596573002B002B0020474D5400303000E2
:100F20003A002D002B000020202020002D44697362
:100F300061626C6564212D003A0045004D433A0022
:100F40003A002E002D0020002020003A0020004210
:100F5000333A686F6C6420746F2073617665004269
:100F6000333A73656C2042312F42323A636867002E
:100F70003D3D536574204F7074696F6E733D3D0045
:100F8000506C6561736520576169742E2E2E005276
:100F90006573657474696E6720454550524F4D0006
:100FA0007C3C3E5E2B3D3F2F5B5D3B2C2A225C0050
:100FB00000002100240027002A0000002200250054
:100FC00028002B0000002000230026002900020238
:100FD00002020202020204040404040404040303DF
:100FE00003030303030301010101010101010102E4
:100FF00004081020408001020408102040800102F3
:1010000004081020408080402010080402010000E5
:1010100000010200000000000000040307060000B9
:101020000000000000000000000000000000F50CBF
:10103000FC4351459560DA60046A11241FBECFEF6E
:10104000D0E1DEBFCDBF13E0A0E0B1E0E2E6F6ED17
:1010500002C005900D92AA3DB107D9F71EE0AAED96
:10106000B3E001C01D92A431B107E1F710E1CAE37A
:10107000D0E104C02297FE010E94F46ACE32D1076B
:10108000C9F70E94546A0C942F6B0C940000CF9304
:10109000DF93BC018230910510F462E070E0A09112
:1010A000120EB091130EED0140E050E0E0E0F0E0F0
:1010B00021C0888199818617970769F48A819B816D
:1010C000309719F09383828304C09093130E80931A
:1010D000120EFE0134C06817790738F44115510526
:1010E00019F08417950708F4AC01FE018A819B81F1
:1010F0009C01E9012097E9F641155105A9F1CA01C2
:10110000861B970B049708F4BA01E0E0F0E02AC0D0
:101110008D919C91119784179507F9F464177507C1
:1011200081F412968D919C911397309719F09383C7
:10113000828304C09093130E8093120EFD013296A9
:101140004CC0CA01861B970BFD01E80FF91F619384
:10115000719302978D939C9340C0FD01828193818E
:101160009C01D9011097A1F68091100E9091110E5B
:10117000892B41F48091C3019091C4019093110E89
:101180008093100E4091C5015091C6014115510543
:1011900041F44DB75EB78091C1019091C201481BE7
:1011A000590B2091100E3091110ECA01821B930B26
:1011B0008617970780F0AB014E5F5F4F8417950746
:1011C00050F0420F531F5093110E4093100EF9012F
:1011D0006193719302C0E0E0F0E0CF01DF91CF9125
:1011E0000895CF93DF93009709F450C0EC01229744
:1011F0001B821A82A091120EB091130E109709F162
:1012000040E050E0AC17BD0708F1BB83AA83FE01A4
:1012100021913191E20FF31FAE17BF0779F48D9141
:101220009C911197280F391F2E5F3F4F39832883D8
:1012300012968D919C9113979B838A83411551053A
:1012400071F4D093130EC093120E20C012968D919C
:101250009C911397AD01009711F0DC01D3CFFA01F7
:10126000D383C28321913191E20FF31FCE17DF07A1
:1012700069F488819981280F391F2E5F3F4FFA0149
:10128000318320838A819B8193838283DF91CF91F5
:101290000895A0E0B0E0EFE4F9E00C94FA6A6C0184
:1012A000009729F4CB010E9447086C01C1C08EEF62
:1012B000882E8FEF982E8C0C9D1C8601060F171F11
:1012C0000815190508F4B2C0F401A081B181A61770
:1012D000B707B8F0A530B10508F4AAC0CD0104974E
:1012E0008617970708F4A4C01297A61BB70BF8013E
:1012F000A193B193D4016D937C93CF010E94F10827
:1013000097C07B01EA1AFB0AEEEFFFEFEE0EFF1E1D
:1013100036016A0E7B1EC091120ED091130EAA24C4
:10132000BB24442455244AC0C615D705E1F548819D
:1013300059814E155F05B8F1CA0104978E159F05B6
:10134000B0F41296A40FB51FF401B183A0832A81D3
:101350003B814114510431F0D20113963C932E93FA
:10136000129766C03093130E2093120E61C08A81CB
:101370009B81F80193838283425050404E195F094C
:10138000518340834114510431F0D20113961C93D0
:101390000E93129704C01093130E0093120EF401D3
:1013A0007183608345C088819981A816B90608F4C5
:1013B0005C012E018A819B819C01E901209709F043
:1013C000B3CF8091100E9091110E86159705E9F418
:1013D000A616B706D0F42091C5013091C60121159B
:1013E000310541F42DB73EB78091C1019091C20102
:1013F000281B390B02171307C8F41093110E009322
:10140000100ED4016D937C9313C0CB010E9447084A
:10141000EC01009759F0F40140815181B6010E941E
:10142000790AC6010E94F1086E0102C0CC24DD24B5
:10143000C601CDB7DEB7E0E10C94166BFC0188273E
:101440009927E89421912032E9F3293010F02E30C9
:10145000C8F32B3241F02D3239F4689404C00E9455
:101460007D0B820F911D219120532A30C0F31EF471
:10147000909581959F4F08951F93FC019927882788
:10148000BC01E89411911032E9F3193010F01E30CC
:10149000C8F31B3251F01D3249F4689406C00E9413
:1014A000680B610F711D811D911D119110531A3030
:1014B000B0F33EF490958095709561957F4F8F4F76
:1014C0009F4F1F910895FB01DC0102C005900D9212
:1014D00041505040D8F70895FB01DC0104C08D91C4
:1014E0000190801921F441505040C8F7881B990B96
:1014F0000895FB01DC0102C001900D924150504063
:10150000D8F70895DC0101C06D9341505040E0F7D9
:101510000895FB01DC010D900020E9F7119701907F
:101520000D920020E1F70895FC018191861721F0CA
:101530008823D9F7992708953197CF010895FB01A2
:10154000DC0101900D920020E1F70895FB01DC0120
:101550004150504030F08D910190801919F40020D5
:10156000B9F7881B990B0895FB01DC0141505040ED
:1015700048F001900D920020C9F701C01D92415022
:101580005040E0F70895A0E0B0E0E9ECFAE00C94F8
:10159000026B7C01EB018A01690109C0CE01219631
:1015A000F6010995F70181937F0101501040011563
:1015B0001105A1F7CDB7DEB7E8E00C941E6BBF9222
:1015C000CF92DF92EF92FF920F931F937B018C01DA
:1015D000FB010995B82EC8010196F7010995C82E9F
:1015E000C8010296F7010995D82EC8010396F701A4
:1015F0000995982F6B2D7C2D8D2D1F910F91FF90AC
:10160000EF90DF90CF90BF900895A0E0B0E0EBE0C6
:10161000FBE00C94026BEC017B018A01690109C0BB
:10162000CE012196F70161917F01F60109950150E4
:10163000104001151105A1F7CDB7DEB7E8E00C9415
:101640001E6BBF92CF92DF92EF92FF920F931F9388
:10165000D52EC62EB72E79018C01642FF90109957C
:10166000C80101966D2DF7010995C80102966C2DF0
:10167000F7010995C80103966B2DF70109951F9194
:101680000F91FF90EF90DF90CF90BF900895FB01F6
:101690009F01E8944230C4F04532B4F44A3029F452
:1016A00097FB1EF4909581959F4F642F77270E949A
:1016B0008E6A805D8A330CF0895D8193CB0100973F
:1016C000A1F716F45DE251931082C9010C94C00B8E
:1016D000592F482F372F262F660F771F881F991FE6
:1016E000660F771F881F991F620F731F841F951F36
:1016F000660F771F881F991F08957AE0979F902D96
:10170000879F802D910D11240895FA01CF93FF93A7
:10171000EF932230CCF02532BCF4C22F2C2F33278C
:1017200044275527FF93EF930E94B56AEF91FF91ED
:10173000605D6A330CF0695D6193B901CA01605064
:1017400070408040904051F710828F919F91CF91CF
:101750000C94C00BFB019F01423074F0453264F4DD
:10176000642F77270E948E6A805D8A330CF0895D32
:101770008193CB010097A1F71082C9010C94C00B93
:10178000DC01FC01672F71917723E1F7329704C0E8
:101790007C916D9370836291AE17BF07C8F3089573
:1017A0009C01F999FECF32BD21BDF89A80B508950C
:1017B0009C01F999FECF1FBA32BD21BD60BD0FB6A5
:1017C000F894FA9AF99A0FBE0895FC01A681B781A0
:1017D0006D93B783A68381E090E008951F920F92E6
:1017E0000FB60F9211242F933F934F935F936F93F4
:1017F0007F938F939F93AF93BF93EF93FF938091CA
:10180000D7078F5F8093D7078091D707803128F063
:10181000E091D507F091D6070995FF91EF91BF911F
:10182000AF919F918F917F916F915F914F913F9178
:101830002F910F900FBE0F901F901895CF92DF92AF
:10184000EF92FF920F931F93CF93DF937B018C0155
:101850000894E11CF11C011D111DC0906D0A442368
:1018600061F430916A0A3695369536953170A1EA61
:10187000B8E0C1EED7E0DD2471C090916A0A969578
:10188000969596959170C1EAD8E061EE77E0EC2DDF
:10189000F0E0EE0FFF1FEE0FFF1FEC0FFD1F25C046
:1018A000288139814A815B81211531054105510526
:1018B000C9F0DB01ED92FD920D931C931397D801B3
:1018C000C701820F931FA41FB51F88839983AA8322
:1018D000BB832091C4027C018D01E20EF11C011D2D
:1018E000111D91E024966C5F7F4FCE17DF07C1F684
:1018F0009170990F990F990F80916A0A877F892BB0
:1019000037C04D915D916D917C91139741155105B3
:101910006105710501F1ED2DE695E695E695F0E09E
:10192000E259F54F808190E02D2D277002C09595EA
:1019300087952A95E2F780FD0EC0E882F9820A8336
:101940001B834E0D5F1D601F711F4D935D936D9343
:101950007C93139731E0D39414962496DC1488F288
:101960003170330F330F330F80916A0A877F832BD7
:1019700080936A0ADF91CF911F910F91FF90EF90B2
:10198000DF90CF900895A1E6B9E080E090E0FC01FF
:10199000EF51F84F1082118212821382FC01EF5531
:1019A000F74F10821182128213821D920496803C9E
:1019B000910569F7F999FECF8CE694E092BD81BD5F
:1019C000F89A80B58093D8071092D9071092DA0759
:1019D0001092DC071092DB071092DD071092DE07F1
:1019E0001092DF071092E00708951092940710926A
:1019F000930785E593E0909392078093910789E19F
:101A000080939E071092A1071092B4071092BB0713
:101A10001092BD0708950F931F93DF93CF93CDB717
:101A2000DEB76E970FB6F894DEBF0FBECDBF8C0148
:101A30008DE997E0B8010E943E4E8823F1F1CE0176
:101A40000196B80141E00E9478608E010B5F1F4F44
:101A500019C0C80162E174E040E052E00E941052F7
:101A60009C01442737FD4095542F203082E03807F1
:101A700080E0480780E05807B0F0C90160E143E02A
:101A80000E94BF342F89388D498D5A8D8F85988952
:101A9000A989BA89281739074A075B07D1F620E0D8
:101AA00030E040E050E0C90161E143E00E94BF3412
:101AB000CE0105960E94EA5181E06E960FB6F89429
:101AC000DEBF0FBECDBFCF91DF911F910F91089563
:101AD000AF92BF92DF92EF92FF920F931F93CF933B
:101AE000DF9300D000D000D0EDB7FEB7319601E90A
:101AF00017E0ADB7BEB712961C930E9311978CE802
:101B000092E0938382838FEC90E0958384830E949C
:101B1000E2390F900F90EDB7FEB71283018384E88E
:101B200092E0948383830E94E239FF240F900F9008
:101B30000F900F90D02EE12E21E8A22E22E0B22E9F
:101B4000CFE7D2E04FC00F2D10E000D000D000D082
:101B5000ADB7BEB71196EDB7FEB7D182E28213964C
:101B6000BC92AE921297F80193E0F595E7959A959D
:101B7000E1F7E259F54F808190E0980127703070CD
:101B800002C0959587952A95E2F781709070159619
:101B90009C938E9314970E94E23980916D0A90E095
:101BA00001972DB73EB72A5F3F4F0FB6F8943EBF5F
:101BB0000FBE2DBF08171907A1F000D000D0ADB798
:101BC000BEB71196DC9211971296EC92129714966A
:101BD000DC93CE9313970E94E2390F900F900F90F1
:101BE0000F90F39420916D0AF21608F4ACCF00D058
:101BF00000D000D0EDB7FEB7319681E997E0ADB7E0
:101C0000BEB712969C938E9311978DE692E09383C4
:101C10008283248315820E94E239EDB7FEB736969F
:101C20000FB6F894FEBF0FBEEDBF81E0DF91CF91FC
:101C30001F910F91FF90EF90DF90BF90AF900895AC
:101C4000AF92BF92CF92DF92EF92FF920F931F93CA
:101C5000CF93DF9300D000D000D0EDB7FEB7319620
:101C600001E917E0ADB7BEB712961C930E9311971A
:101C70008CE894E0938382838FEC90E09583848357
:101C80000E94E2390F900F90EDB7FEB712830183E7
:101C90008AE894E0948383830E94E239CDE4D2E021
:101CA000FF240F900F900F900F90E02E012F42E82D
:101CB000A42E44E0B42E30E8C32E34E0D32E2C8181
:101CC0003D818881F4E1FF1619F490E0CC9701C0C2
:101CD00090E04DB75EB7485050400FB6F8945EBFE5
:101CE0000FBE4DBFEDB7FEB73196ADB7BEB711967B
:101CF000EC92119712960C93B382A28235832483BF
:101D0000978386830E94E239EDB7FEB738960FB607
:101D1000F894FEBF0FBEEDBFF2E2FF16A1F000D0B7
:101D200000D0ADB7BEB71196EC92119712960C93F6
:101D300012971496DC92CE9213970E94E2390F907C
:101D40000F900F900F90F3942796B3E2FB1609F0D3
:101D5000B6CF00D000D081E997E0EDB7FEB792830F
:101D600081838EE794E0948383830E94E2390F900D
:101D70000F900F900F9081E0DF91CF911F910F9105
:101D8000FF90EF90DF90CF90BF90AF9008950F93AA
:101D90001F9300D000D000D0EDB7FEB7319601E917
:101DA00017E0ADB7BEB712961C930E93119789EF4B
:101DB00099E09383828380E790E0958384830E94F7
:101DC000E23900D0EDB7FEB73196ADB7BEB7129687
:101DD0001C930E93119784EB98E09383828380E8A1
:101DE00090E09583848380E091E0978386830E94CE
:101DF000E2398DB79EB708960FB6F8949EBF0FBE16
:101E00008DBF81E01F910F910895CF92DF92EF92E5
:101E1000FF920F931F93DF93CF9300D000D0CDB7E5
:101E2000DEB70E9435647B018C016E010894C11CF1
:101E3000D11C0E94D9310E94ED36C6016091CD01BE
:101E40000E94E5338823E1F0E980FA800B811C8150
:101E500080EC98EDA4E5BCE7E80EF91E0A1F1B1FF5
:101E60006091540270E080E090E024E833E040E0CC
:101E700050E00E94636AE60EF71E081F191F0EC08D
:101E80000E9435646E197F09800B910B685E734068
:101E90008040904070F2EE24FF248701B701C80112
:101EA0000F900F900F900F90CF91DF911F910F9196
:101EB000FF90EF90DF90CF900895EF92FF921F93E5
:101EC000DF93CF9300D000D0CDB7DEB780911F0352
:101ED0008983809126038A8380912D038B8380914F
:101EE00034038C8310E07E010894E11CF11C6091A6
:101EF000CD016F5F6093CD01C7010E944F366AEF3D
:101F000070E080E090E00E9443640E94050F9B0116
:101F1000AC01611571058105910519F41F5F14313C
:101F200031F7B901CA010F900F900F900F90CF9128
:101F3000DF911F91FF90EF9008952F923F925F9253
:101F40006F927F928F929F92AF92BF92CF92DF92C9
:101F5000EF92FF920F931F93DF93CF93CDB7DEB72E
:101F60006E970FB6F894DEBF0FBECDBF6C018091A7
:101F70006A0A86FF1DC1C60160E677E040E32BE2F6
:101F800031E00E94684D882309F412C180E697E091
:101F90000E943C0A7B018C01C60160E677E040E3C9
:101FA00021E331E00E94684D882309F401C1C80192
:101FB000B70120E831E541E050E00E94D76A6901AD
:101FC0007A01890180E697E00E943C0A20E831E529
:101FD00041E050E00E94D76A59012C153D0508F4F4
:101FE000E7C0025F1F4F0217130708F4E1C000D0DB
:101FF00000D000D0EDB7FEB7319601E917E0ADB7DC
:10200000BEB712961C930E93119782E392E09383CE
:1020100082838FEC90E0958384830E94E239EE24E2
:10202000FF2477247394EDB7FEB736960FB6F89475
:10203000FEBF0FBEEDBF60E6262E67E0362E55E0F0
:10204000852E912C8C0E9D1E502E612E02E114E0E7
:1020500097C0C60160E677E04AE050E00E94470B77
:1020600080E697E065E371E00E94890A8DE997E0D8
:1020700060E677E00E943E4E882309F47EC01D8210
:102080001F821C821B828DEA93E09A838983C4019C
:1020900060E677E041E00E94905801C07724C401D7
:1020A00060E677E04FE250E020E030E00E94AD5380
:1020B0001816190624F0C4010E94EA515EC0FC0102
:1020C000E15AF84F80818A3009F41082772081F03C
:1020D00000D000D000D0EDB7FEB73196ADB7BEB797
:1020E00011965C92119712966C928FE292E00FC05B
:1020F00000D000D000D0EDB7FEB73196ADB7BEB777
:1021000011965C92119712966C928BE292E09383F7
:102110008283358224820E94E239ADB7BEB716961B
:102120000FB6F894BEBF0FBEADBF0894E11CF11C02
:10213000C70169E170E00E94A26A892B09F0AECF65
:102140008091970790919807209195073091960775
:10215000821B930B60E140E00E94BF341092940711
:102160001092930710939607009395071093980782
:1021700000939707EE24FF2491CF0894C11CD11C33
:10218000AC14BD0408F065CF00D000D081E997E021
:10219000EDB7FEB79283818389E292E094838383D3
:1021A0000E94E23981E00F900F900F900F9001C0D4
:1021B00080E06E960FB6F894DEBF0FBECDBFCF9114
:1021C000DF911F910F91FF90EF90DF90CF90BF9024
:1021D000AF909F908F907F906F905F903F902F90E7
:1021E0000895CF93DF939C0110926007FC01A081BA
:1021F000B181C0E0D0E00FC09C919D3231F09B32A4
:1022000021F0892F80538A3068F4FE01E05AF84F9C
:10221000908321961196F901808191810A96A817E1
:10222000B90750F3C05AD84F18821196F901B183FB
:10223000A08380E697E00E941E0ADF91CF91089567
:102240004F925F926F927F928F929F92AF92BF92C6
:10225000CF92DF92EF92FF920F931F93DF93CF9372
:102260000F92CDB7DEB70E94E9415B016C0100D04F
:1022700000D000D0EDB7FEB7319601E917E0ADB759
:10228000BEB712961C930E93119784E096E0938349
:1022900082838FEC90E0958384830E94E239EDB7CE
:1022A000FEB772970FB6F894FEBF0FBEEDBF319622
:1022B000ADB7BEB712961C930E93119780EB95E0C5
:1022C00093838283A482B582C682D78280916C0A6E
:1022D0008087118680916A0A817082871386809137
:1022E0006A0A869581708487158680916A0A869528
:1022F000869581708687178680916A0A829581709B
:10230000808B118A8091800A9091810AA091820A23
:10231000B091830A828B938BA48BB58B80E690E07F
:10232000978B868B0E94E23990E0EDB7FEB77896E6
:102330000FB6F894FEBF0FBEEDBF78010CEA15E0B2
:1023400023C000D000D000D0EDB7FEB73196ADB7B6
:10235000BEB71196EC9211971296FC9213830283EA
:10236000A92FB0E0A259B54F8C918483158299832F
:102370000E94E23999819F5FEDB7FEB736960FB69E
:10238000F894FEBF0FBEEDBF80916C0AA1E96A2EE2
:10239000A7E07A2E9817A8F200D000D0ADB7BEB74C
:1023A00012967C926E92119782EA95E014969C9315
:1023B0008E9313970E94E23999240F900F900F90FB
:1023C0000F90C301762C892EF9E94F2EF5E05F2E90
:1023D00066C0A92DB0E0FD01EF59F64F608166237C
:1023E000A9F1CD01880F991F880F991FFC01EF51AA
:1023F000F84FE080F18002811381FC01EF55F74F27
:10240000AE14BF04C006D10648F02081318142815C
:1024100053812A193B094C095D0908C0208131818B
:10242000428153812E193F09400B510BAA0FBB1F4C
:10243000AA0FBB1FAF55B74F8D919D910D90BC91C9
:10244000A02D8E5F9F4FAF4FBF4F21F420E030E0B3
:1024500040E050E08DB79EB70A970FB6F8949EBF44
:102460000FBE8DBFEDB7FEB73196ADB7BEB71196B3
:102470007C92119712968C925382428264831582C9
:1024800026833783408751870E94E2399394EDB7C2
:10249000FEB73A960FB6F894FEBF0FBEEDBF80911F
:1024A0006D0A981608F495CF2DB73EB72E503040E0
:1024B0000FB6F8943EBF0FBE2DBFEDB7FEB73196F5
:1024C00081E997E0ADB7BEB712969C938E931197B2
:1024D0008CE795E0938382838091D907848315826A
:1024E0008091DA07868317828091DB079091DC0761
:1024F000918780878091DD079091DE07A091DF07AB
:10250000B091E00782879387A487B5870E94E2395C
:10251000EDB7FEB73E960FB6F894FEBF0FBEEDBF07
:1025200081E00F90CF91DF911F910F91FF90EF907D
:10253000DF90CF90BF90AF909F908F907F906F90E3
:102540005F904F900895BF92CF92DF92EF92FF92EB
:102550000F931F936C01FC01B080E1800E94E94160
:1025600020E831E541E050E00E94B56A8B2D8F777D
:10257000280F311D411D511DFF2400E010E0CA014C
:10258000B901A80197010E94B56AF0E8BF22B62AF6
:10259000F601B0821F910F91FF90EF90DF90CF90E6
:1025A000BF9008956F927F928F929F92AF92BF9249
:1025B000CF92DF92EF92FF920F931F934C01FC0199
:1025C000708061800E94E941A62CBB24CC24DD24CC
:1025D000BFE7EB2EE720FF24E60CF11C0027F7FCF9
:1025E0000095102F20E831E541E050E00E94B56AE7
:1025F000CA01B901A60195010E94B56AE61AF70A57
:10260000080B190BC801B701A60195010E94B56A14
:10261000F0E87F22762AF40170821F910F91FF90DB
:10262000EF90DF90CF90BF90AF909F908F907F9072
:102630006F900895EF92FF921F93CF93DF93182F1F
:102640007B010E94E9419B01AC01C12FD0E02F5FCB
:102650003F4F4F4F5F4FCE01880F991F880F991F33
:10266000FC01EF51F84F2083318342835383FC01F7
:10267000EF55F74FE114F10449F48EEF9FEFAFEF00
:10268000BFEF80839183A283B3830DC0C701AA27C4
:1026900097FDA095BA2F280F391F4A1F5B1F208373
:1026A000318342835383CF59D64F83E68883809109
:1026B0006A0A886080936A0ADF91CF911F91FF9028
:1026C000EF900895AF92BF92CF92DF92EF92FF9278
:1026D0000F931F93CF93DF938C010E5F1F4F20E06A
:1026E00030E006C0F901E15AF84F90830F5F1F4FA9
:1026F000E22FD8019C91892F80538A3028F42F5FD4
:102700003F4F2530310571F7F0E0E05AF84F108265
:1027100080E697E00E941E0AEC0197FDD4C08091EC
:102720006D0A90E08C179D070CF4CDC0F8018081F4
:102730008D3309F057C0209709F4C5C080916A0A0B
:1027400084FFC1C02197C80101962181203379F40B
:102750000E94E941EC2FF0E0EE0FFF1FEE0FFF1F8C
:10276000EF55F74F608371838283938319C02133C0
:1027700009F0A9C060E677E040E32AE331E00E9477
:10278000684D882319F460E070E007C080E697E0A8
:102790000E941E0ABC0197FD96C08C2F0E941A133E
:1027A00000D000D000D0EDB7FEB7319681E997E0B8
:1027B000ADB7BEB712969C938E9311978CE392E0BF
:1027C0009383828380E790E0958384830E94E2393B
:1027D00081E0EDB7FEB736960FB6F894FEBF0FBE98
:1027E000EDBF72C000D000D000D0EDB7FEB731967B
:1027F00081E997E0ADB7BEB712969C938E9311977F
:1028000089E392E09383828380E790E095838483D9
:102810000E94E239EDB7FEB736960FB6F894FEBFC8
:102820000FBEEDBF209721F480916D0A90E003C0A8
:102830008C2F9C2F9150C0E0D0E0E92EFF24082F70
:1028400010E061E9A62E67E0B62E56E3C52E52E0F1
:10285000D52E31C000D000D000D0ADB7BEB7119694
:10286000EDB7FEB7B282A1821396DC92CE92129798
:10287000F90143E0F595E7954A95E1F7E259F54FFF
:10288000808190E02770307002C0959587952A95D9
:10289000E2F78170907015969C938E9314970E9426
:1028A000E23921962DB73EB72A5F3F4F0FB6F89415
:1028B0003EBF0FBE2DBF9E012E0D3F1D20173107BD
:1028C0004CF281E001C080E0DF91CF911F910F9128
:1028D000FF90EF90DF90CF90BF90AF900895AF92B0
:1028E000BF92CF92DF92EF92FF920F931F93CF93FD
:1028F000DF932DB73EB7285030400FB6F8943EBF57
:102900000FBE2DBFEDB7FEB7319601E917E0ADB7A9
:10291000BEB712961C930E93119789E794E09383A8
:10292000828380E790E09583848387E391E09783B7
:1029300086830E94E2390F900F900F900F90EDB7B1
:10294000FEB71283018386E694E0948383830E941A
:10295000E239BDE4EB2EB2E0FB2EAA24C0E0D0E0C9
:102960000F900F900F900F90B02EC12E07E514E03E
:102970005C2F6D2FD70116968C91169781FF33C06F
:1029800014962D913C91159711964C9111978C911D
:10299000C43119F490E0CC9701C090E0EDB7FEB7D8
:1029A0003C970FB6F894FEBF0FBEEDBF3196ADB7A2
:1029B000BEB71196BC9211971296CC9213830283E4
:1029C0003583248346831782918780875287638764
:1029D0000E94E239A394EDB7FEB73C960FB6F89487
:1029E000FEBF0FBEEDBF219627E030E0E20EF31EE2
:1029F000C332D10509F0BCCF0E94E9416B017C01D3
:102A0000B09054020E94DF48ADB7BEB752970FB6E0
:102A1000F894BEBF0FBEADBFEDB7FEB7319601E96A
:102A200017E012961C930E9311972FE134E0338335
:102A30002283A482158220E630E037832683C08675
:102A4000D186E286F386B48615868687178685E06A
:102A500090E0918B808B0E94E239EDB7FEB73E96F5
:102A60000FB6F894FEBF0FBEEDBF1283018384E161
:102A700094E0948383830E94E23900D0EDB7FEB7DF
:102A80003196ADB7BEB712961C930E9311978EEE8A
:102A900093E09383828380E890E0958384830E940F
:102AA000E239EDB7FEB736960FB6F894FEBF0FBE0B
:102AB000EDBF81E0DF91CF911F910F91FF90EF90DB
:102AC000DF90CF90BF90AF900895BF92CF92DF92EA
:102AD000EF92FF920F931F93CF93DF9300D000D01C
:102AE00001E917E0ADB7BEB712961C930E9311978C
:102AF0008AE89AE014969C938E9313970E94E23989
:102B0000FF240F900F900F900F90B02EE12E10E643
:102B1000C12E17E0D12E04E81AE021C08F2D60E607
:102B200077E00E941C4400D000D000D0EDB7FEB783
:102B30003196ADB7BEB71196BC9211971296EC9232
:102B400013830283D582C4820E94E239F394EDB7E5
:102B5000FEB736960FB6F894FEBF0FBEEDBF80915C
:102B60006D0AC1E9D7E0F816C8F200D000D0ADB7C1
:102B7000BEB71296DC93CE9311978FE79AE0149626
:102B80009C938E9313970E94E2390F900F900F90B1
:102B90000F908E819F812C813D81821B930B60E180
:102BA00040E00E94BF34DF91CF911F910F91FF90C1
:102BB000EF90DF90CF90BF9008954F925F926F9209
:102BC0007F928F929F92AF92BF92CF92DF92EF92BD
:102BD000FF920F931F93DF93CF930F92CDB7DEB782
:102BE0000E94E9415B016C012DB73EB7285030408F
:102BF0000FB6F8943EBF0FBE2DBFEDB7FEB73196AE
:102C000001E917E0ADB7BEB712961C930E9311976A
:102C10008FE695E09383828380E790E095838483B9
:102C200087E391E0978386830E94E239EDB7FEB790
:102C300038960FB6F894FEBF0FBEEDBF0E94651523
:102C4000109294071092930782E194E09093960774
:102C50008093950790939807809397072DB73EB779
:102C60002A5030400FB6F8943EBF0FBE2DBFEDB7CF
:102C7000FEB73196ADB7BEB712961C930E9311975F
:102C80008AE595E0938382838FEC90E0958384833B
:102C9000A682B782C086D1860E94E2390F900F903B
:102CA000EDB7FEB73196ADB7BEB712961C930E9333
:102CB000119780E495E09383828380916C0A8483EA
:102CC000158280915402868317820E94E23990E037
:102CD000EDB7FEB738960FB6F894FEBF0FBEEDBF46
:102CE00078010CE315E023C000D000D000D0EDB790
:102CF000FEB73196ADB7BEB71196EC92119712960A
:102D0000FC9213830283A92FB0E0A259B54F8C9196
:102D10008483158299830E94E23999819F5FEDB780
:102D2000FEB736960FB6F894FEBF0FBEEDBF80918A
:102D30006C0A41E9642E47E0742E9817A8F200D07F
:102D400000D0ADB7BEB712967C926E92119780E319
:102D500095E014969C938E9313970E94E2399924E0
:102D60000F900F900F900F90C301762C892E37E2B1
:102D7000432E35E0532E66C0A92DB0E0FD01EF597A
:102D8000F64F60816623A9F1CD01880F991F880F46
:102D9000991FFC01EF51F84FE080F180028113810F
:102DA000FC01EF55F74FAE14BF04C006D10648F042
:102DB00020813181428153812A193B094C095D09E7
:102DC00008C020813181428153812E193F09400B77
:102DD000510BAA0FBB1FAA0FBB1FAF55B74F8D9149
:102DE0009D910D90BC91A02D8E5F9F4FAF4FBF4F17
:102DF00021F420E030E040E050E08DB79EB70A9724
:102E00000FB6F8949EBF0FBE8DBFEDB7FEB73196DB
:102E1000ADB7BEB711967C92119712968C925382E1
:102E200042826483158226833783408751870E94BC
:102E3000E2399394EDB7FEB73A960FB6F894FEBF19
:102E40000FBEEDBF80916D0A981608F495CF2DB78F
:102E50003EB72A5130400FB6F8943EBF0FBE2DBF8B
:102E6000EDB7FEB7319601E917E0ADB7BEB71296E0
:102E70001C930E93119785ED94E093838283809148
:102E80006A0A81708483158280916A0A86958170AE
:102E90008683178280916A0A8695869581708087DD
:102EA000118680916A0A829581708287138680914B
:102EB000800A9091810AA091820AB091830A848746
:102EC0009587A687B7878091CB02808B118A8091E6
:102ED000E002828B138A8091EE02848B158A8091A6
:102EE000FC02868B178A80E690E0918F808F0E948B
:102EF000E239EDB7FEB73C960FB6F894FEBF0FBEB1
:102F0000EDBF3196ADB7BEB712961C930E931197D5
:102F100083EB94E0938382838091D9078483158225
:102F20008091DA07868317828091DB079091DC0716
:102F3000918780878091DD079091DE07A091DF0760
:102F4000B091E00782879387A487B5870E94E23912
:102F5000EDB7FEB738960FB6F894FEBF0FBEEDBFC3
:102F60003196ADB7BEB712961C930E9311978FE8AA
:102F700094E09383828380E890E0958384830E9429
:102F8000E239EDB7FEB736960FB6F894FEBF0FBE26
:102F9000EDBF81E00F90CF91DF911F910F91FF90D6
:102FA000EF90DF90CF90BF90AF909F908F907F90E9
:102FB0006F905F904F900895FF920F931F93CF9360
:102FC000DF938C010E944B35109294071092930767
:102FD00082E194E0909396078093950790939807E9
:102FE00080939707A8014B5F5F4FD80115968C918E
:102FF000803221F4CA010E94DD158FC0CEECD1E0F1
:10300000A0E0B0E0682F772767FD7095FA2EE88181
:10301000F981849190E08617970709F08DC0319669
:10302000249130E0FA018181992787FD9095281736
:10303000390709F081C0AA0FBB1FAA0FBB1FA053FD
:10304000BE4FED91FC91CA010995882301F500D08E
:1030500000D000D0EDB7FEB7319681E997E0ADB76B
:10306000BEB712969C938E93119789E192E0938359
:10307000828382E691E0958384830E94E239EDB7F2
:10308000FEB736960FB6F894FEBF0FBEEDBFF6E161
:10309000FF1609F042C080916A0A86FF3EC0402FA9
:1030A000E0E6F7E0C801DC0101C081939A2F941B90
:1030B00015968C911597803229F0119627E0E0380B
:1030C000F20799F7E92FF0E0E05AF84F108280E616
:1030D00097E00E940B0D8823B9F500D000D000D0F6
:1030E000EDB7FEB7319681E997E0ADB7BEB712965E
:1030F0009C938E93119786E192E09383828382E67C
:1031000091E0958384830E94E239EDB7FEB736964D
:103110000FB6F894FEBF0FBEEDBF80919707909158
:1031200098072091950730919607821B930B61E1D8
:1031300040E00E94BF3408C0F39411962496A63153
:10314000B10509F063CFA3CFDF91CF911F910F910C
:10315000FF900895BF92CF92DF92EF92FF920F936C
:103160001F93CF93DF932DB73EB7285030400FB653
:10317000F8943EBF0FBE2DBFEDB7FEB7319601E903
:1031800017E0ADB7BEB712961C930E93119788E562
:1031900098E09383828380E790E09583848387E33C
:1031A00091E0978386830E94E239EDB7FEB73896A7
:1031B0000FB6F894FEBF0FBEEDBF0E9465151092CA
:1031C00094071092930782E194E09093960780937E
:1031D000950790939807809397072DB73EB72A508D
:1031E00030400FB6F8943EBF0FBE2DBFEDB7FEB70F
:1031F0003196ADB7BEB712961C930E93119784E328
:1032000098E09383828380916C0A848315828091F5
:10321000CB02868317828091FC02808711860E94F0
:10322000E239DD24E12C74E0F72EEDB7FEB73A96D3
:103230000FB6F894FEBF0FBEEDBFB02EC12E00E357
:1032400018E033C0F999FECFF2BCE1BCF89A90B512
:10325000F999FECF0894E11CF11CF2BCE1BCF89A8C
:1032600080B5D92FC0E000D000D000D0EDB7FEB7B8
:103270003196ADB7BEB71196BC9211971296CC920B
:10328000138302839E01280F311D358324830E94FE
:10329000E239D3940894E11CF11C8DB79EB70696D1
:1032A0000FB6F8949EBF0FBE8DBF80916D0AD816E1
:1032B00008F4C8CF00D000D001E917E0ADB7BEB721
:1032C00012961C930E93119782E298E014969C93A9
:1032D0008E9313970E94E23900D0EDB7FEB7319676
:1032E000ADB7BEB712961C930E9311978CEF97E073
:1032F0009383828380E890E0958384830E94E239FF
:10330000EDB7FEB736960FB6F894FEBF0FBEEDBF11
:1033100081E0DF91CF911F910F91FF90EF90DF90AF
:10332000CF90BF900895AF92BF92DF92EF92FF923D
:103330000F931F93DF93CF930F92CDB7DEB700D0DB
:1033400000D000D0EDB7FEB7319601E917E0ADB778
:10335000BEB712961C930E93119783E19BE0938363
:10336000828380E790E0958384830E94E239EDB701
:10337000FEB736960FB6F894FEBF0FBEEDBF0E94A3
:103380006515109294071092930782E194E0909350
:1033900096078093950790939807809397072DB78A
:1033A0003EB72C5030400FB6F8943EBF0FBE2DBF35
:1033B000EDB7FEB73196ADB7BEB712961C930E931C
:1033C00011978AEE9AE09383828380916C0A8483BA
:1033D000158280E190E0978386838091CB0280877D
:1033E00011868091FC02828713860E94E239EDB734
:1033F000FEB738960FB6F894FEBF0FBEEDBF12832E
:1034000001838EED9AE0948383830E94E23990E0F9
:103410000F900F900F900F9078010AED1AE023C0E3
:1034200000D000D000D0EDB7FEB73196ADB7BEB733
:103430001196EC9211971296FC9213830283A92F96
:10344000B0E0AC58B54F8C918483158299830E946B
:10345000E23999819F5FEDB7FEB736960FB6F894C3
:10346000FEBF0FBEEDBF80916C0AA1E9AA2EA7E0B6
:10347000BA2E9817A8F200D000D0ADB7BEB71296FA
:10348000BC92AE9211978EEC9AE014969C938E9318
:1034900013970E94E23900E00F900F900F900F9069
:1034A000C501DA2C192FFAECEF2EFAE0FF2E21C01D
:1034B00000D000D000D0EDB7FEB73196ADB7BEB7A3
:1034C0001196DC92119712961C93F382E282A02F40
:1034D000B0E0A658B54F8C91848315820E94E239E2
:1034E0000F5FEDB7FEB736960FB6F894FEBF0FBE6E
:1034F000EDBF80916C0AE1E9AE2EE7E0BE2E081721
:10350000B8F200D000D000D0EDB7FEB73196ADB71D
:10351000BEB71296BC92AE92119787E99AE0938358
:10352000828380E890E0958384830E94E239EDB73E
:10353000FEB736960FB6F894FEBF0FBEEDBF81E022
:103540000F90CF91DF911F910F91FF90EF90DF903F
:10355000BF90AF9008958F929F92AF92BF92CF92FB
:10356000DF92EF92FF920F931F93CF93DF9300D0E0
:1035700000D000D0EDB7FEB7319601E917E0ADB746
:10358000BEB712961C930E93119788E69BE0938327
:1035900082838FEC90E0958384830E94E2390F90C0
:1035A0000F90EDB7FEB7128301838CE59BE0948307
:1035B00083830E94E239FF240F900F900F900F90A9
:1035C000E02E012F30E6C32E37E0D32E27E5822EE2
:1035D0002BE0922E95E5A92E9BE0B92E3EC08F2DB3
:1035E00060E677E00E941C4400D000D000D0EDB728
:1035F000FEB73196ADB7BEB71196EC921197129601
:103600000C9393828282D582C4820E94E2392F2D4C
:1036100030E080916D0A90E00197EDB7FEB73696E5
:103620000FB6F894FEBF0FBEEDBF28173907A1F003
:1036300000D000D0ADB7BEB71196EC92119712969C
:103640000C9312971496BC92AE9213970E94E23993
:103650000F900F900F900F90F39480916D0AC1E935
:10366000D7E0F81608F4BBCF00D000D0EDB7FEB716
:10367000D283C18389E49BE0948383830E94E239EF
:10368000FF240F900F900F900F90CE01DC2EE92EAB
:1036900086E4882E8BE0982E04E4A02E0BE0B02E5A
:1036A00040C00F2D10E000D000D000D0ADB7BEB7A5
:1036B0001196EDB7FEB7D182E28213969C928E925C
:1036C0001297F801EC58F54F808114968C9314975B
:1036D00015961C920E94E23980916C0A90E0019745
:1036E0002DB73EB72A5F3F4F0FB6F8943EBF0FBECF
:1036F0002DBF08171907A1F000D000D0ADB7BEB795
:103700001196DC9211971296EC9212971496BC9235
:10371000AE9213970E94E2390F900F900F900F9086
:10372000F39480916C0AC1E9D7E0F81608F4B9CF98
:1037300000D000D0EDB7FEB7D283C18382E39BE017
:10374000948383830E94E239FF240F900F900F909F
:103750000F90CE01DC2EE92E1FE2812E1BE0912E70
:10376000BDE2AB2EBBE0BB2E40C00F2D10E000D061
:1037700000D000D0ADB7BEB71196EDB7FEB7D1827D
:10378000E28213969C928E921297F801E658F54FBA
:10379000808114968C93149715961C920E94E2399E
:1037A00080916C0A90E001972DB73EB72A5F3F4F9A
:1037B0000FB6F8943EBF0FBE2DBF08171907A1F032
:1037C00000D000D0ADB7BEB71196DC92119712961B
:1037D000EC9212971496BC92AE9213970E94E23923
:1037E0000F900F900F900F90F39480916C0AC1E9A5
:1037F000D7E0F81608F4B9CF00D000D000D0EDB76C
:10380000FEB73196ADB7BEB71296DC93CE93119743
:103810008EE19BE09383828380E190E095838483B3
:103820000E94E239EDB7FEB736960FB6F894FEBFA8
:103830000FBEEDBF81E0DF91CF911F910F91FF90FF
:10384000EF90DF90CF90BF90AF909F908F900895B2
:103850009C018091FC02882311F081E00895C90148
:1038600060E677E040E32CE331E00E94684D882376
:1038700031F080E697E00E943245811181E00895A1
:103880000F931F93DF93CF93CDB7DEB7C058D040CF
:103890000FB6F894DEBF0FBECDBF8C010D5F1F4F7A
:1038A000C8010E94281C882309F440C0C8018E0169
:1038B0000F5F1F4FB80140E82FE331E00E94684DD1
:1038C000882341F0C8010E94B44D80E890E0B8011F
:1038D0000E940D452DB73EB7285030400FB6F894E2
:1038E0003EBF0FBE2DBFEDB7FEB7319681E997E021
:1038F000ADB7BEB712969C938E9311978AE793E06B
:103900009383828380E790E09583848382EB91E0C8
:10391000978386830E94E23981E02DB73EB7285F06
:103920003F4F0FB6F8943EBF0FBE2DBFC058DF4FBC
:103930000FB6F894DEBF0FBECDBFCF91DF911F91C0
:103940000F9108958F929F92AF92BF92CF92DF9284
:10395000FF920F931F93DF93CF9300D000D0CDB78A
:10396000DEB773E0C72ED12CC80ED91EC6010E9447
:10397000281C882309F4B3C083E789831A821B8239
:103980001C8210E062E0862E912C8C0E9D1E5E0142
:103990000894A11CB11C1AC0812F90E0B4014AE028
:1039A00050E00E94470BC60160E677E040E39501D6
:1039B0000E94684D882349F080E697E00E94B44D4C
:1039C000812F60E677E00E9441441F5F80916D0A7D
:1039D000181710F38DE68983FF2452E0852E912C71
:1039E0008C0E9D1E5E010894A11CB11C1AC00F2DE7
:1039F00010E0C801B4014AE050E00E94470BC60144
:103A000060E677E040E395010E94684D882341F02D
:103A100080E697E00E941E0A0C58154FD8018C933F
:103A2000F39480916C0AF81610F30E94824489E6A0
:103A30008983FF2442E0842E912C8C0E9D1E5E0112
:103A40000894A11CB11C1AC00F2D10E0C801B401CC
:103A50004AE050E00E94470BC60160E677E040E391
:103A600095010E94684D882341F080E697E00E940E
:103A70001E0A0658154FF8018083F39480916C0A52
:103A8000F81610F30E946B442DB73EB72850304013
:103A90000FB6F8943EBF0FBE2DBFEDB7FEB73196FF
:103AA00081E997E0ADB7BEB712969C938E931197BC
:103AB0008AE59AE09383828380E790E0958384830C
:103AC00082EB91E0978386830E94E23981E0EDB733
:103AD000FEB738960FB6F894FEBF0FBEEDBF0F903D
:103AE0000F900F900F90CF91DF911F910F91FF904A
:103AF000DF90CF90BF90AF909F908F9008958F925E
:103B00009F92AF92BF92CF92DF92EF92FF920F936C
:103B10001F93CF93DF93EC017A018B01CB01BA01A4
:103B20000E94D6404C01C801B7010E94D0405C0100
:103B30008889882309F481C0D880D7FE21C0C98034
:103B400021E02C15E8F4C801B70120E831E541E097
:103B500050E00E94B56ACA01B9012C2D30E040E066
:103B600050E00E94B56A2FE7D2222D2D30E040E0D0
:103B700050E0621773078407950709F05EC031C0F3
:103B8000C801B7010E94C440288130E090E005964A
:103B900067E070E00E94A26A02C0359527958A9579
:103BA000E2F720FF4AC0C801B7010E94CA40D82EE0
:103BB000888187FF16C08981882319F4D0FE11C03F
:103BC0003CC0813071F48FE1D816B9F12DE1D216E5
:103BD00009F042C0C801B7010E94BE400297E1F55A
:103BE0002CC08CE390E0889E9001899E300D989EB9
:103BF000300D11242A0D3B1D4A815B8124173507A6
:103C0000E0F08C819D8182179307B8F0EE81FF81EF
:103C1000309799F0241B350B40E0C901BF010E9489
:103C20008E6A6E9FC0016F9F900D7E9F900D112434
:103C30008217930719F441E001C040E0842FDF911F
:103C4000CF911F910F91FF90EF90DF90CF90BF9099
:103C5000AF909F908F900895D0FCC3CFEECF982F58
:103C60009B018091D807981768F461E1969FB00195
:103C7000112462597B4FC90141E150E020ED3BE046
:103C80000E94C30A0895CF92DF92EF92FF920F93A2
:103C90001F93DF93CF93CDB7DEB762970FB6F8943B
:103CA000DEBF0FBECDBF8C010D5F1F4FC8010E944C
:103CB000B44DC80160E677E040E323E431E00E94C0
:103CC000684D882309F42BC180E697E00E941E0A04
:103CD0007C012FEF8F3F92070CF421C18091D80710
:103CE00090E0E816F9060CF01AC18DB79EB7089758
:103CF0000FB6F8949EBF0FBE8DBFEDB7FEB73196DD
:103D000001E917E0ADB7BEB712961C930E93119759
:103D10008DEA97E09383828380E790E095838483A4
:103D200087E391E0978386830E94E239EDB7FEB77F
:103D300038960FB6F894FEBF0FBEEDBF0E94651512
:103D4000109294071092930782E194E09093960763
:103D50008093950790939807809397072DB73EB768
:103D60002A5030400FB6F8943EBF0FBE2DBFEDB7BE
:103D7000FEB73196ADB7BEB712961C930E9311974E
:103D80008EE897E09383828380916C0A8483158206
:103D9000F782E6828091FC02808711860E94E239D8
:103DA000EDB7FEB73A960FB6F894FEBF0FBEEDBF63
:103DB000FFEFEF16FFEFFF0609F48FC08E2D7E0197
:103DC0000894E11CF11CB7010E942F1E8A818230E9
:103DD00018F0C7010E94D2122DB73EB722513040D1
:103DE0000FB6F8943EBF0FBE2DBFEDB7FEB73196AC
:103DF00001E917E0ADB7BEB712961C930E93119769
:103E00008FE697E0938382838989848315828981F1
:103E1000868317828A81808711868B819C81938714
:103E200082878D819E81958784878F8198859787EA
:103E3000868789859A85918B808B0E94E23990E0F4
:103E4000EDB7FEB772960FB6F894FEBF0FBEEDBF8A
:103E50006801EBE6EE2EE7E0FE2E8E01055F1F4FB8
:103E600022C000D000D000D0EDB7FEB73196ADB77C
:103E7000BEB71196CC9211971296DC92F382E28231
:103E8000D801A90FB11D8C91848315829A8B0E9451
:103E9000E2399A899F5FEDB7FEB736960FB6F89470
:103EA000FEBF0FBEEDBF80916C0A9817D0F200D014
:103EB00000D081E997E0ADB7BEB712969C938E9380
:103EC000119788E697E014969C938E9313970E941F
:103ED000E2390F900F900F900F9000D000D000D0DB
:103EE000EDB7FEB7319681E997E0ADB7BEB7129650
:103EF0009C938E93119787E397E09383828380E866
:103F000090E0958384830E94E23981E0EDB7FEB7AB
:103F100036960FB6F894FEBF0FBEEDBF01C080E02D
:103F200062960FB6F894DEBF0FBECDBFCF91DF9182
:103F30001F910F91FF90EF90DF90CF9008952F92F7
:103F40003F924F925F926F927F928F929F92AF9229
:103F5000BF92DF92EF92FF920F931F93DF93CF9365
:103F6000CDB7DEB761970FB6F894DEBF0FBECDBFF9
:103F700000D000D000D0EDB7FEB7319601E917E0D0
:103F8000ADB7BEB712961C930E93119781EB98E0D4
:103F9000938382838FEC90E0958384830E94E2393F
:103FA00000D000D0EDB7FEB73196ADB7BEB71296D0
:103FB0001C930E93119787E898E0938382838091F6
:103FC000D8078483158280916C0A8683178285E3E3
:103FD00090E0918780870E94E239FF24EDB7FEB719
:103FE0003A960FB6F894FEBF0FBEEDBF4E0108948F
:103FF000811C911CD02EE12E1BE0212E312C2C0E89
:104000003D1EB8E64B2EB8E05B2EAAE66A2EA8E06D
:104010007A2EF2E1AF2EF4E0BF2EACC08F2DB401AA
:104020000E942F1E8A81823018F0C4010E94D21291
:104030008DB79EB742970FB6F8949EBF0FBE8DBF47
:10404000EDB7FEB73196ADB7BEB71196DC921197BA
:104050001296EC9281E798E0938382838989848326
:1040600015828981868317828A81808711868B8158
:104070009C81938782878D819E81958784878F819C
:1040800098859787868789859A85918B808B0E94F2
:10409000E23910E0ADB7BEB752961DC000D000D0D7
:1040A00000D0EDB7FEB73196ADB7BEB71196DC9232
:1040B00011971296EC928DE698E093838283D1015A
:1040C000A10FB11D8C91848315820E94E2391F5F7C
:1040D000ADB7BEB716960FB6F894BEBF0FBEADBF54
:1040E00080916C0A1817D0F20F2D10E08091D8073C
:1040F00090E001970817190749F000D000D0EDB7FC
:10410000FEB7D182E282748263820EC000D000D0FA
:10411000ADB7BEB71196DC9211971296EC9212973A
:1041200014965C924E9213970E94E2390F900F9072
:104130000F900F900370107003301105D1F480912F
:104140009707909198072091950730919607821BC9
:10415000930B60E140E00E94BF34109294071092EC
:104160009307B0929607A0929507B0929807A092F5
:104170009707F3948091D807F81608F44FCF00D032
:1041800000D081E997E0EDB7FEB79283818385E6A1
:1041900098E0948383830E94E2390F900F900F90F0
:1041A0000F9081E061960FB6F894DEBF0FBECDBFD1
:1041B000CF91DF911F910F91FF90EF90DF90BF9013
:1041C000AF909F908F907F906F905F904F903F90B7
:1041D0002F9008952F923F924F925F926F927F920D
:1041E0008F929F92AF92BF92CF92DF92EF92FF9207
:1041F0000F931F93DF93CF93CDB7DEB761970FB6C1
:10420000F894DEBF0FBECDBF8DB79EB70C970FB62B
:10421000F8949EBF0FBE8DBFEDB7FEB7319601E992
:1042200017E0ADB7BEB712961C930E9311978BE2B1
:104230009AE0938382838091D8078483158280914A
:104240006C0A868317828091FC028087118685E341
:1042500090E0938782870E94E239DD24EDB7FEB7B4
:104260003C960FB6F894FEBF0FBEEDBF4E0108940A
:10427000811C911CC02E012F2BE0222E312C2C0EE4
:104280003D1E4C2C512E97E0692E9AE0792E82E14A
:10429000A82E84E0B82E9AC08D2DB4010E942F1E46
:1042A0008A81823018F0C4010E94D212ED2CFF24C2
:1042B0008DB79EB744970FB6F8949EBF0FBE8DBFC3
:1042C000EDB7FEB73196ADB7BEB71196CC92119748
:1042D00012960C938EE09AE093838283F582E482B7
:1042E0008989868317828981808711868A8182875E
:1042F00013868B819C81958784878D819E8197878A
:1043000086878F819885918B808B89859A85938B01
:10431000828B0E94E23910E0ADB7BEB754961DC043
:1043200000D000D000D0EDB7FEB73196ADB7BEB724
:104330001196CC92119712960C938AE09AE093838F
:104340008283D101A10FB11D8C91848315820E94BB
:10435000E2391F5FADB7BEB716960FB6F894BEBF71
:104360000FBEADBF80916C0A1817D0F200D000D0FC
:10437000EDB7FEB741825282748263820E94E239B5
:10438000F3E0EF22FF240F900F900F900F9083E047
:10439000E816F104D1F48091970790919807209145
:1043A000950730919607821B930B60E140E00E94D5
:1043B000BF341092940710929307B0929607A09280
:1043C0009507B0929807A0929707D3948091D80749
:1043D000D81608F461CF00D000D081E997E0ADB7DE
:1043E000BEB712969C938E9311978CEF99E014961A
:1043F0009C938E9313970E94E2390F900F900F9029
:104400000F9061960FB6F894DEBF0FBECDBFCF916F
:10441000DF911F910F91FF90EF90DF90CF90BF90B1
:10442000AF909F908F907F906F905F904F903F9054
:104430002F9008952F923F924F925F926F927F92AA
:104440008F929F92AF92BF92CF92DF92EF92FF92A4
:104450000F931F93DF93CF9300D0CDB7DEB78C01BE
:104460000D5F1F4FC8010E94B44D0E94E9415B01DE
:104470006C010E94B5402C01C601B5010E94BE40EE
:104480003C01C601B5010E94CA404C01C601B501FC
:104490000E94D6409A838983C601B5010E94D0400C
:1044A0001C01C80160E677E040E327E431E00E94A8
:1044B000684D882361F080E697E00E941E0A4C0157
:1044C000009729F4C601B5010E94CA404C01C801F9
:1044D00060E677E040E329E431E00E94684D8823FC
:1044E00029F080E697E00E941E0A3C01C80160E6C0
:1044F00077E040E32BE431E00E94684D882329F007
:1045000080E697E00E941E0A2C0100D000D000D067
:10451000EDB7FEB7319651E9E52E57E0F52EADB770
:10452000BEB71296FC92EE92119781E097E09383CA
:10453000828380E790E0958384830E94E239EDB71F
:10454000FEB736960FB6F894FEBF0FBEEDBF0E94C1
:104550006515109294071092930782E194E090936E
:1045600096078093950790939807809397072DB7A8
:104570003EB72A5130400FB6F8943EBF0FBE2DBF54
:104580000DB71EB70F5F1F4FADB7BEB71296FC92A7
:10459000EE9211978AEA96E0F801938382838091E4
:1045A000BD02848315828091CB028683178280911D
:1045B000EE02808711868091C402828713868091E3
:1045C000D202848715868091D90286871786C60114
:1045D000B50120E831E541E050E00E94B56AD8011C
:1045E00051963C932E9350978CE390E0E981FA81A9
:1045F0009C01E29FC001E39F900DF29F900D11245A
:10460000820D931D53969C938E93529755969C9230
:104610008E92549757967C926E92569759965C92CA
:104620004E9258970E94E2394DB75EB74A5E5F4F8F
:104630000FB6F8945EBF0FBE4DBFADB7BEB71296B2
:10464000FC92EE9211978EE996E014969C938E93CD
:1046500013970E94E23900E00F900F900F900F9097
:10466000BE2CEF2C4AE9C42E46E0D42E21C000D047
:1046700000D000D0EDB7FEB73196ADB7BEB71196FA
:10468000BC9211971296EC92D382C282A02FB0E016
:10469000AC58B54F8C91848315820E94E2390F5F2C
:1046A000EDB7FEB736960FB6F894FEBF0FBEEDBF5E
:1046B00080916C0A31E9832E37E0932E0817B8F207
:1046C00000D000D0ADB7BEB712969C928E921197D3
:1046D00086E996E014969C938E9313970E94E23994
:1046E0000F900F900F900F900E94EA2000D000D002
:1046F00000D0EDB7FEB73196ADB7BEB712969C921B
:104700008E9211978EE696E09383828380E890E004
:10471000958384830E94E239EDB7FEB736960FB6D3
:10472000F894FEBF0FBEEDBF81E00F900F90CF91C8
:10473000DF911F910F91FF90EF90DF90CF90BF908E
:10474000AF909F908F907F906F905F904F903F9031
:104750002F9008950F931F938DB79EB708970FB6AC
:10476000F8949EBF0FBE8DBFEDB7FEB7319601E93D
:1047700017E0ADB7BEB712961C930E93119782EE59
:1047800097E09383828380E790E09583848387E337
:1047900091E0978386830E94E2398DB79EB7089691
:1047A0000FB6F8949EBF0FBE8DBF0E946515109284
:1047B00094071092930782E194E090939607809378
:1047C000950790939807809397070E94EA2000D05E
:1047D00000D000D0EDB7FEB73196ADB7BEB7129698
:1047E0001C930E9311978AEB97E09383828380E862
:1047F00090E0958384830E94E2398DB79EB7069638
:104800000FB6F8949EBF0FBE8DBF81E01F910F9130
:104810000895DF92EF92FF920F931F93DF93CF9350
:10482000CDB7DEB761970FB6F894DEBF0FBECDBF30
:104830002091D807821708F043C0222309F440C012
:1048400090E001968C0174E0000F111F7A95E1F75A
:10485000080F191F02591B4F61E1D62E7E010894E3
:10486000E11CF11C13C0C701B80141E150E020ED8B
:104870003BE00E94C30AC8014197B70141E150E003
:1048800028ED3BE00E94050B0F5E1F4F2091D807DB
:104890002D9DC001112482599B4F0817190718F349
:1048A00021502093D807F999FECF1FBA8CE694E0E7
:1048B00092BD81BD20BD0FB6F894FA9AF99A0FBE49
:1048C00061960FB6F894DEBF0FBECDBFCF91DF91DA
:1048D0001F910F91FF90EF90DF900895CF93DF939A
:1048E000EC012396CE010E94B44DCE010E94281CFB
:1048F000882309F450C0CE0160E677E040E323E46A
:1049000031E00E94684D882309F445C080E697E0B5
:104910000E941E0A9C018FEF2F3F380781F41092EE
:10492000D807F999FECF1FBA8CE694E092BD81BDFD
:1049300010BC0FB6F894FA9AF99A0FBE09C080918C
:10494000D80790E02817390734F5822F0E940924F0
:1049500000D000D000D0EDB7FEB7319681E997E0E6
:10496000ADB7BEB712969C938E9311978CE097E0EB
:104970009383828380E790E0958384830E94E23969
:1049800081E02DB73EB72A5F3F4F0FB6F8943EBF88
:104990000FBE2DBF01C080E0DF91CF910895982F09
:1049A0008091D807981760F481E1989FC001112485
:1049B00082599B4F41E150E028ED3BE00E94050BFE
:1049C0000895BC019091D8079533F0F481E1989F48
:1049D000C001112482599B4F41E150E028ED3BE09A
:1049E0000E94050B2091D8072F5F2093D807F999D3
:1049F000FECF1FBA8CE694E092BD81BD20BD0FB6FC
:104A0000F894FA9AF99A0FBE0895BF92CF92DF9266
:104A1000EF92FF920F931F93DF93CF93CDB7DEB743
:104A200063970FB6F894DEBF0FBECDBF7C018C013B
:104A30000D5F1F4FC8010E94B44DC8010E94281C81
:104A4000882309F403C1C80160E677E040E323E46A
:104A500031E00E94684D882309F4F8C080E697E0B1
:104A60000E941E0A6C012FEF8F3F92070CF4EEC0DC
:104A70008091D80790E0C816D9060CF0E7C01A83D9
:104A8000098387E690E0E80EF91E0DC0C8016DE4C9
:104A900071E043E050E00E94A60A009779F00F5FB2
:104AA0001F4F1A83098309811A81D8018C918823A9
:104AB00009F4CCC00E151F0548F3C8C00D5F1F4F89
:104AC0001A8309838E010F5F1F4FC8010E94F110E6
:104AD0008B8BC8010E94F1108B83C8010E94F110DA
:104AE0008C83C8010E94F1109E838D83C8010E94AF
:104AF000F11098878F83C8010E94F1109A878987E7
:104B0000C8010E94F1109C878B87FF24B02EE12EF4
:104B10008E01035F1F4F09C08B2D9E2D0E94F11047
:104B2000F801EF0DF11D8083F39480916C0AF81663
:104B300098F306C0FC01EF0DF11D1082F39402C042
:104B4000CE010D96B5E0BF15A8F78C81823020F01C
:104B5000CE0103960E94A31200D000D000D0EDB782
:104B6000FEB7319601E917E0ADB7BEB712961C93B8
:104B70000E93119783E696E09383828380E790E01B
:104B8000958384830E94E239EDB7FEB736960FB65F
:104B9000F894FEBF0FBEEDBFBE016D5F7F4FFFEF0C
:104BA000CF16FFEFDF06C1F4CB010E94E12400D055
:104BB00000D0ADB7BEB712961C930E93119786E442
:104BC00096E014969C938E9313970E94E2390F906F
:104BD0000F900F900F9022C08C2D0E94CF2400D0F8
:104BE00000D000D0EDB7FEB73196ADB7BEB7129684
:104BF0001C930E93119788E296E093838283089426
:104C0000C11CD11CD582C4820E94E239EDB7FEB727
:104C100036960FB6F894FEBF0FBEEDBF00D000D0A1
:104C200081E997E0ADB7BEB712969C938E9311972A
:104C300087E096E014969C938E9313970E94E23936
:104C400081E00F900F900F900F9001C080E063966D
:104C50000FB6F894DEBF0FBECDBFCF91DF911F918D
:104C60000F91FF90EF90DF90CF90BF900895EF925B
:104C7000FF920F931F93DF93CF93CDB7DEB7A59726
:104C80000FB6F894DEBF0FBECDBF80916A0A86FFD3
:104C900088C06091DD077091DE078091DF079091F9
:104CA000E00720E831E541E050E00E94B56ACA0122
:104CB000B90140E657E02AE030E00E94850B80E62B
:104CC00097E065E371E00E94890A1C861E861B86B8
:104CD0001A868DEA93E099878887ECE0EE2EF12C16
:104CE000EC0EFD1EC70160E677E042E40E9490589A
:104CF0004E8D5F8D68A179A1C7010E94824F8E0100
:104D00000F5F1F4FC80161E571E00E94BC68C801D8
:104D10006091DA070E944D68C80163E571E00E9466
:104D20007968C8016091D9070E944D68C80163E5A0
:104D300071E00E9479686091DB077091DC07C8011F
:104D40000E941F68C80163E571E00E947968409184
:104D5000DD075091DE076091DF077091E007C80121
:104D60000E94ED67C80165E571E00E947968C8019D
:104D700067E571E00E947968C80160E677E040E38A
:104D800050E020E030E00E945D67CE01089660E6CA
:104D900077E00E945360C7010E94EA51C8010E9457
:104DA000D668A5960FB6F894DEBF0FBECDBFCF91E3
:104DB000DF911F910F91FF90EF900895CF93DF93B4
:104DC000EC0180916A0A86FF11C0CE0165E371E0B3
:104DD0000E94890A8DE997E0BE010E943E4E882319
:104DE00029F08DE997E0BE010E943A4EDF91CF9104
:104DF0000895CF93DF93EC012396CE010E94B44D2A
:104E0000CE010E94281C8823D9F1CE0160E677E00C
:104E100040E32AE531E00E94684D882389F180E66D
:104E200097E00E94DE262DB73EB7285030400FB6DF
:104E3000F8943EBF0FBE2DBFEDB7FEB7319681E9A6
:104E400097E0ADB7BEB712969C938E9311978CE105
:104E500092E09383828380E790E09583848382EB62
:104E600091E0978386830E94E23981E02DB73EB7B7
:104E7000285F3F4F0FB6F8943EBF0FBE2DBF01C055
:104E800080E0DF91CF9108950E94BD440E94674960
:104E9000A1E6B9E080E090E0FC01EF51F84F10820C
:104EA000118212821382FC01EF55F74F108211829A
:104EB000128213821D920496803C910569F7089531
:104EC0004F925F926F927F928F929F92AF92BF921A
:104ED000CF92DF92EF92FF920F931F93DF93CF93C6
:104EE000CDB7DEB7E5970FB6F894DEBF0FBECDBFE6
:104EF000A3E0AA2EB12CA80EB91EC5010E94281C41
:104F0000882309F43CC15090540240905B020DE4A8
:104F100012E0EE24CC24DD244E010894811C911C67
:104F2000F2E06F2E712C6C0E7D1E2C2D9D2DD80164
:104F300016968C91169781FF3BC011968C91119714
:104F4000813009F41C92D401E9E5F3E085E0019099
:104F50000D928150E1F7822FB3014AE050E00E94A8
:104F6000470BC50160E677E040E394010E94684D7D
:104F70008823F1F0F801F180F1E0FF1619F4D8016F
:104F8000FC9216C080E697E00E941E0A9C01B4E1E4
:104F9000CB1611F4245C3F4F37FD08C08F2D90E0F5
:104FA000821793071CF0F801208302C0EE24E394DB
:104FB0000894C11CD11C095F1F4FF3E2CF16D10426
:104FC00009F0B3CFC50160E677E040E32EE531E0BC
:104FD0000E94684D882351F080E697E00E94B44D0E
:104FE00080E690E060E677E00E940D45C50160E64E
:104FF00077E040E322E631E00E94684D8823F1F03B
:1050000080E697E00E94B44D80E697E00E943C0A5B
:10501000162F072FF82ED92E0E944427612F702FAC
:105020008F2D9D2D0E94BC4180916A0A85FF06C08C
:10503000612F702F8F2D9D2D0E94BC43EE2089F093
:1050400000D000D000D0EDB7FEB7319681E997E0EF
:10505000ADB7BEB712969C938E93119781E393E000
:10506000B5C00E94E944C50160E677E040E326E66A
:1050700031E00E94684D882309F444C08E010A5F24
:105080001F4FC501B80140E32AE631E00E94684D98
:10509000882309F48BC080E697E0B80140E150E036
:1050A0000E94A60A009709F081C080E490E060E6C3
:1050B00077E00E940D452DB73EB7285030400FB61F
:1050C000F8943EBF0FBE2DBFEDB7FEB7319681E914
:1050D00097E0ADB7BEB712969C938E93119789E077
:1050E00093E09383828380E790E09583848382EBCF
:1050F00091E0978386830E94E23981E0EDB7FEB7A5
:10510000389670C02DB73EB7285030400FB6F8948F
:105110003EBF0FBE2DBFEDB7FEB7319681E997E0D8
:10512000ADB7BEB712969C938E9311978FE892E01D
:105130009383828380E790E09583848382EB91E080
:10514000978386830E94E239EDB7FEB738960FB693
:10515000F894FEBF0FBEEDBF80915402851531F467
:10516000442061F480915B02882341F010929907FA
:1051700010929A0710929B0710929C0781E0E59687
:105180000FB6F894DEBF0FBECDBFCF91DF911F9158
:105190000F91FF90EF90DF90CF90BF90AF909F90D6
:1051A0008F907F906F905F904F90089500D000D0C7
:1051B00000D0EDB7FEB7319681E997E0ADB7BEB745
:1051C00012969C938E9311978BEB92E0938382833C
:1051D00080E790E0958384830E94E23981E0EDB717
:1051E000FEB736960FB6F894FEBF0FBEEDBFC7CF21
:1051F000EF92FF920F931F93CF93DF93EC012396CF
:10520000CE010E94281C882309F407C1CE0160E664
:1052100077E040E32EE631E00E94684D882311F0EC
:105220000E944427CE0160E677E040E322E731E0C8
:105230000E94684D882309F44CC080E697E00E94E4
:105240001E0A181619060CF044C02DB73EB7285098
:1052500030400FB6F8943EBF0FBE2DBFEDB7FEB77E
:10526000319601E917E0ADB7BEB712961C930E93C5
:1052700011978CEB93E09383828380E790E0958392
:10528000848384E190E0978386830E94E2390F90C3
:105290000F900F900F90EDB7FEB7128301838FEA46
:1052A00093E0948383830E94E2390F900F900F90D4
:1052B0000F908091970790919807209195073091D2
:1052C0009607821B930B61E140E00E94BF340E946D
:1052D0001644CE0160E677E040E326E731E00E9425
:1052E000684D882399F080916007813339F480916B
:1052F0006A0A80FD0BC00E94CE4908C0803331F499
:1053000080916A0A80FF02C00E94C449CE0160E613
:1053100077E040E329E731E00E94684D8823E9F017
:1053200080916007813351F480916A0A84FD15C031
:105330000E94442780916A0A80610BC0803369F41F
:1053400080916A0A84FF09C00E94442780916A0AFA
:105350008F7E80936A0A0E940849CE0160E677E05A
:1053600040E32CE731E00E94684D882351F180E64C
:1053700097E00E941E0AEC0118161906F4F40E9428
:10538000E9417B018C01BE01882777FD8095982F2C
:1053900020E13EE040E050E00E94636AE60EF71E26
:1053A000081F191FE092800AF092810A0093820A76
:1053B0001093830A0E94BA4904C0009771F50E94B5
:1053C000A8492DB73EB7285030400FB6F8943EBFDD
:1053D0000FBE2DBFEDB7FEB7319681E997E0ADB7AF
:1053E000BEB712969C938E93119782EA93E09383B3
:1053F000828380E790E09583848382EB91E09783BA
:1054000086830E94E23981E0EDB7FEB738960FB689
:10541000F894FEBF0FBEEDBF01C080E0DF91CF91D9
:105420001F910F91FF90EF900895BF92CF92DF925E
:10543000EF92FF920F931F93DF93CF9300D0CDB7DE
:10544000DEB77C018C010D5F1F4FC8010E94B44D77
:10545000C8010E94281C882309F4A0C01A8309836C
:1054600027E630E0E20EF31E0DC0C8016FE771E0E1
:1054700043E050E00E94A60A009779F00F5F1F4FAB
:105480001A83098309811A81D8018C91882309F430
:1054900085C00E151F0548F381C00D5F1F4F1A838D
:1054A00009830E944427FF2400E014E0EE246E01EB
:1054B0000894C11CD11C8EEFB82E37C0C6010E94C3
:1054C000F110F999FECF1FBA12BD01BD90BD0FB604
:1054D000F894FA9AF99A0FBEF999FECF1FBA0F5FA6
:1054E0001F4F12BD01BD0150104080BD0FB6F89492
:1054F000FA9AF99A0FBE0097A9F02F2D30E0F90122
:10550000EE0FFF1FEE0FFF1FEF55F74FA0E0B0E0CB
:1055100080839183A283B3832F59364FF901B082E0
:10552000EE24E394F3940E5F1F4F80916D0AF816FA
:1055300008F4C4CFEE2031F00E94E9414091BD0251
:105540000E941E0C2DB73EB7285030400FB6F8947D
:105550003EBF0FBE2DBFEDB7FEB7319681E997E094
:10556000ADB7BEB712969C938E9311978FEE97E0CE
:105570009383828380E790E09583848382EB91E03C
:10558000978386830E94E23981E0EDB7FEB73896B3
:105590000FB6F894FEBF0FBEEDBF01C080E00F90C4
:1055A0000F90CF91DF911F910F91FF90EF90DF90BF
:1055B000CF90BF9008952F923F924F925F926F923B
:1055C0007F928F929F92AF92BF92CF92DF92EF9293
:1055D000FF920F931F93DF93CF9300D000D0CDB7EE
:1055E000DEB71091CB0290916A0A292F21702A838D
:1055F000892E82944FE0842231E0832291FD0CC0F9
:105600008091E002882311F4EE2408C0E92EE6948C
:10561000E69441E0E42211F0EE24E3940E94E94193
:105620005B016C019924212E3324A7C0892D90E0C1
:10563000FC01E658F54F3081FC01E259F54F20811D
:10564000A92DAA0FAA0FAA0FA98300E010E0422EED
:105650005524632E7724882009F088C0F980F00E45
:10566000EF2DF0E0FC83EB83EF59F64FE081EE3F46
:1056700009F47CC0FA81FF2361F0EE2009F476C0C2
:10568000C301002E02C0959587950A94E2F780FD2C
:105690006DC0C201002E02C0959587950A94E2F76D
:1056A00080FF49C08F2D60E00E9499448B819C81CE
:1056B00001962816390621F1F092D907EB81FC8179
:1056C000EF59F64F80818093DA07EB81FC81EE0F72
:1056D000FF1FEE0FFF1FEF51F84F80819181950161
:1056E000281B390B3093DC072093DB07A092DD07E2
:1056F000B092DE07C092DF07D092E0070E94372603
:10570000EB81FC81EE0FFF1FEE0FFF1FDF01AF519A
:10571000B84F1D921D921D921C921397EF55F74F93
:1057200010821182128213828B819C818F59964F35
:10573000DC011C921BC0EE23C9F0EB81FC81EE0F53
:10574000FF1FEE0FFF1FDF01AF51B84F1D921D92DB
:105750001D921C921397EF55F74F108211821282FF
:105760001382EB81FC81EF59F64F10820F5F1F4FC0
:105770000830110509F06FCF939480916C0A981648
:1057800008F454CF0F900F900F900F90CF91DF91AE
:105790001F910F91FF90EF90DF90CF90BF90AF904F
:1057A0009F908F907F906F905F904F903F902F9041
:1057B0000895EF92FF920F931F939B01AC0180918C
:1057C0005B02882309F443C080916B0A82958F7035
:1057D00009F03DC080916A0A83FD39C08091990724
:1057E00090919A07A0919B07B0919C070097A10503
:1057F000B10569F079018A01E81AF90A0A0B1B0B55
:10580000D801C70181589145A140B04000F12093D3
:10581000990730939A0740939B0750939C078BE717
:105820009BE061E00E942E460E945D0F7B018C018F
:10583000611571058105910551F00E94BC4180916F
:105840006A0A85FF04C0C801B7010E94BC431F91CA
:105850000F91FF90EF900895AF92BF92CF92DF9299
:10586000EF92FF920F931F935B016C01E0909109FF
:10587000F09092090091930910919409E114F104B8
:105880000105110549F46093910970939209809381
:105890009309909394099AC080916A0A83FD96C0F7
:1058A00080916B0A82958F7021E030E002C0220F58
:1058B000331F8A95E2F7442737FD4095542FD601D0
:1058C000C5018E199F09A00BB10B7C018D01DA0176
:1058D000C90164E0880F991FAA1FBB1F6A95D1F701
:1058E000821B930BA40BB50B8E159F05A007B10768
:1058F00008F06CC085E59AE06FE041E00E94A03EB0
:1059000085E59AE064E00E94523EA0929109B0922F
:105910009209C0929309D09294098AEE99E00E946C
:10592000A0360E9435647B018C010E94D9310E940F
:10593000ED368AEE99E00E946139882361F40E9475
:1059400035646E197F09800B910B683C71058105E8
:10595000910558F328C080916B0A8F7002C08F7038
:10596000806680936B0A80916B0A82958F7090E0BD
:10597000039764F18091AF02882341F18BE69BE0AD
:1059800060E00E942E466091DA037091DB0387ECA1
:1059900091E00E940F4D8823C9F080916B0A8F70AF
:1059A00080936B0A13C080916B0A282F22952F7069
:1059B0002F5F2F70922F9295907F8F70892B8093FD
:1059C0006B0A30E02730310554F6CDCF1F910F918F
:1059D000FF90EF90DF90CF90BF90AF90089584B785
:1059E000877F84BF8091600088618093600081E23E
:1059F00080936000809160008064809360000E94CA
:105A0000DD4B0E942A4A0E94C30C9091A80280E0BC
:105A10002091A102820F911D9093DB038093DA0302
:105A20006CE370E080E090E00E94B34180916A0AEC
:105A300085FD03C080E090E002C08CED93E40E94FD
:105A40005C4264EF71E080E090E00E94436480E09B
:105A50000E94934B88E99BE061E00E942E468DE90D
:105A600097E060E044E00E945D4E882329F0809139
:105A70006A0A806480936A0A8AE89BE061E00E9477
:105A80002E466091DA037091DB0387EC91E00E946F
:105A90000F4D882321F080916B0A8F7004C0809194
:105AA0006B0A8F70806180936B0A64EF71E080E015
:105AB00090E00E9443640E9467490E94E94160931C
:105AC000840A7093850A8093860A9093870A0895C2
:105AD0001F93CF93DF9382E00E949F45182FC82F1A
:105AE000D0E086FF54C00E94E9416093840A70931D
:105AF000850A8093860A9093870A809111036FEF3D
:105B000070E0681B71098CE00E940066CE018F7006
:105B100090708230910589F08430910501F10197F0
:105B2000B1F517FF03C00E94CE4931C060912A022F
:105B300070912B0282EE99E009C017FF03C00E940A
:105B4000C44925C08AEE99E060E070E00E94974861
:105B500060ED77E080E090E00E94436418C017FF9A
:105B600006C081E00E949F450E94164410C020910B
:105B70006B0A822F8F7090E060916C0A019670E042
:105B80000E94A26A8F70207F282B20936B0ADF91DE
:105B9000CF911F9108952F923F924F925F926F92F3
:105BA0007F928F929F92AF92BF92CF92DF92EF92AD
:105BB000FF920F931F93DF93CF93CDB7DEB7AA97D2
:105BC0000FB6F894DEBF0FBECDBF2091BD022C8B67
:105BD0003091CB023B8B0E94D9310E94ED369093DD
:105BE000960980939509009721F084529C4F0E945A
:105BF000DC17A8951092D7070E94682D0E94E941F2
:105C00005B016C0180919B0990919C09A0919D0979
:105C1000B0919E098A159B05AC05BD0509F4DBC250
:105C2000A0929B09B0929C09C0929D09D0929E09B6
:105C300080E00E94934B80916A0A2091800A309103
:105C4000810A4091820A5091830A81FF08C0A216FE
:105C5000B306C406D50650F00E94A84907C0A21694
:105C6000B306C406D50610F40E94BA498091840A8E
:105C70009091850AA091860AB091870A0097A105A4
:105C8000B105C9F04E96A11DB11D8A159B05AC0545
:105C9000BD0588F4809118036FEF70E0681B7109EF
:105CA0008CE00E9400661092840A1092850A10927D
:105CB000860A1092870A0E94E84580916A0A84FD4C
:105CC000C4C083FF04C04C89442309F0BEC0C60190
:105CD000B5012CE330E040E050E00E94B56A790164
:105CE0008A018091970990919809A0919909B091A2
:105CF0009A09E816F9060A071B0709F4A6C0E092FC
:105D00009709F09298090093990910939A096624CB
:105D100010E09B89892F90E09AA789A78AC0862DD9
:105D2000BE016F5F7F4F0E942F1ECE010196B6010C
:105D3000A5010E947F1D882309F47AC029853A8530
:105D40002115310509F474C0A0916C0AAE8B77243B
:105D50001A8A190144245524B62DBF5FB8A753C031
:105D60008A89880DE82EFF24C7010196E9A5FAA5C6
:105D7000E817F907E1F1ACA1BDA18C9190E0082CE6
:105D800002C0959587950A94E2F780FD30C0EEA198
:105D9000FFA1808190E0082C02C0959587950A9418
:105DA000E2F780FF24C08701000F111F000F111FB1
:105DB0000F55174F6091EE0270E080E090E0A20175
:105DC00091010E94636A24E630E040E050E00E94C6
:105DD000B56AD8012D933D934D935C931397E1E6FB
:105DE000F9E0EE0EFF1EE8A5D701EC9311E0089450
:105DF000811C911CF8E08F16910409F0B1CF7394C7
:105E00002A89285F2A8B3E89731690F4872D90E0AB
:105E100088249924AC014259554F5DA34CA3ABE0B3
:105E2000B0E0AC0FBD1FA80FB91FBFA3AEA398CFA2
:105E300063948091D807681608F471CF112329F074
:105E4000C601B5014C890E941E0C80916A0A83FF2D
:105E500054C14424FB89EF2FF0E0FC8FEB8F2B899A
:105E600021502D8F30E0C901880F991F880F991F8D
:105E7000AC014F51584F5F8F4E8FDC01AF55B74F7C
:105E8000B9A3A8A3F901EF59F64FFBA3EAA316C1E2
:105E9000842D90E0FC01E259F54F2081F42DFF0F95
:105EA000FF0FFF0FFD8B66247724422F50E0588FA1
:105EB0004F8BDC01AC58B54FBA8FA98F5D88560C5B
:105EC000852C992491E6E92E99E0F92EE80CF91C2D
:105ED000F7018081882309F44FC08401000F111F4E
:105EE000000F111FF801EF55F74F80819181A281BA
:105EF000B381A816B906CA06DB06F0F1852D60E06D
:105F00000E949944C40101962B8D3C8D28173907B6
:105F1000E1F05092D907D7018C918093DA070F51A5
:105F2000184FF801808191819501281B390B30931E
:105F3000DC072093DB07A092DD07B092DE07C0925A
:105F4000DF07D092E0070E943726F401EE0FFF1F13
:105F5000EE0FFF1FDF01AF51B84F1D921D921D9232
:105F60001C921397EF55F74F108211821282138201
:105F7000F401EF59F64F10828F89988D062C02C0DC
:105F8000959587950A94E2F780FD8FC09401220FC2
:105F9000331F220F331F89010F51184FF8018081E1
:105FA0009181A281B381A816B906CA06DB0608F45E
:105FB0007CC0F1EA2F2EF8E03F2E220E331EF101B5
:105FC00080819181A281B381A816B906CA06DB0639
:105FD00008F06BC0852D61E00E949944FB89FF2386
:105FE00009F463C0C40101962B8D3C8D2817390735
:105FF00009F45BC0A98DBA8D8C9190E0062C02C08B
:10600000959587950A94E2F780FF4FC0BC89BB2322
:1060100009F44BC080916A0A84FD47C08091D20286
:10602000F8012081318142815381280F311D411DAA
:10603000511DAE8DBF8D2D933D934D935C93139762
:106040008091D902E82EFF2400E010E084EC9FEF5D
:10605000AFEFBFEFE80EF91E0A1F1B1FF101808191
:106060009181A281B381E80EF91E0A1F1B1FA8A10E
:10607000B9A1ED92FD920D931C931397E1E6F9E01F
:106080008E0E9F1ED4018C91EAA1FBA18083A216E3
:10609000B306C406D50648F0AE14BF04C006D10648
:1060A00020F48D8D61E00E9499440894611C711C5C
:1060B000F8E06F16710409F001CF439480916C0AE7
:1060C000481608F4E5CE0E94DB2A0E946749309109
:1060D0006D0AE1EAF8E020E00DC081919191A19173
:1060E000B1910197A109B1098E5F9F4FAF4FBF4F8B
:1060F00020F02F5F231788F363C05B89552369F075
:1061000080916A0A84FF09C010916D0A40E021E085
:1061100030E08B89682F70E02EC09C899923A1F311
:1061200031C0842F90E06217730711F1DC01E3E0C6
:10613000B695A795EA95E1F7542F5770FD01E259FE
:10614000F54F808190E0052E02C0959587950A94C1
:10615000E2F780FF0DC0AC58B54F8C9190E002C0C3
:10616000959587955A95E2F780FF02C061E006C0D9
:106170004F5F2F5F3F4F4117A0F260E08B89815046
:106180000E9499440E94DB2A0E946749C601B5011A
:1061900023E030E040E050E00E94B56A9B01AC0192
:1061A000225A3C4F81E0D9016C910E940348C601FC
:1061B000B5010E942C2CC601B5010E94D92B0BC041
:1061C0000E94BD4480916A0A877F80936A0AB091D9
:1061D000CB02BB8B92CFAA960FB6F894DEBF0FBE50
:1061E000CDBFCF91DF911F910F91FF90EF90DF9086
:1061F000CF90BF90AF909F908F907F906F905F9067
:106200004F903F902F9008958091A10961E00E94E6
:10621000376578940895FF920F931F93082F162FD8
:10622000F42EF8948091A10960E00E9437651F71F7
:10623000102B1EBD0DB407FEFDCFFEBC0DB407FE36
:10624000FDCF0E9404311F910F91FF9008951F937D
:10625000182F282F30E0207630708091A20990E02E
:106260002817390799F080EA6FE143E00E940B316B
:10627000412F40764093A20950E085E0559547951F
:106280008A95E1F780E86FE10E940B311F91089534
:106290000F931F93182F062F0E94273180E4612F40
:1062A000402F0E940B311F910F9108950F931F9360
:1062B000182F072F0E944831812F8F5F602F0E9477
:1062C00048311F910F91089588E360EB0E94483197
:1062D000089588E361EB0E94483108950F931F935E
:1062E000182F062FF8948091A10960E00E9437656D
:1062F000802F8F71812B8EBD0DB407FEFDCF1EBC8C
:106300000DB407FEFDCF07FF04C01EBC0DB407FE91
:10631000FDCF1EB50E940431812F1F910F9108956A
:106320001F93182F0E94273180E0612F0E946E3149
:106330001F91089584ED61E10E94483182ED61E092
:106340000E9448318AEE0E94903180FDFBCF82EDA1
:1063500060E00E94483189ED0E94903190E096956E
:10636000879596958795817008950F931F93CF9386
:10637000DF93EC018B01F8948091A10960E00E9409
:1063800037658AE38EBD0DB407FEFDCF09C01EBC84
:106390000DB407FEFDCF8EB5F80181938F012197D3
:1063A0002097A9F70E940431DF91CF911F910F919F
:1063B00008950F931F93DF93CF9300D000D000D0A8
:1063C000CDB7DEB789E30E949031882319F400E04D
:1063D00010E048C06091A3097091A40980E00E9478
:1063E000563186E090E0BE016F5F7F4F0E94B5316D
:1063F00089819A819093A4098093A3092B813C8180
:10640000E0919F09F091A0098D8187FD03C000E014
:1064100010E00EC0245030408F0101501040201772
:10642000310708F48901C8016CED73E00E94B531B1
:10643000F801E452FC4F10826091A3097091A40905
:106440008CE06130780724F08CE06FEF7BE003C0D4
:10645000615070408CE00E94563180E86EE140E46B
:106460000E940B31C80126960FB6F894DEBF0FBE0E
:10647000CDBFCF91DF911F910F9108950F931F937F
:10648000CF93DF938C01EB01F8948091A10960E038
:106490000E9437658AE78EBD0DB407FEFDCF08C0A8
:1064A00088818EBD0DB407FEFDCF219601501040AE
:1064B00001151105A9F70E940431DF91CF911F91B9
:1064C0000F910895CF93DF93EC010FC08CE10E94F0
:1064D000903181FF0AC080E86FE140E80E940B31F3
:1064E00080EA6FE140E80E940B3180E06FE10E949A
:1064F0006E3183FDEBCF82E060E07CE00E9456319C
:10650000BE016050744F86E00E9456318AE760E019
:1065100040E00E940B31CE016CED73E00E943E32F0
:1065200080E86FE148E00E940B31DF91CF91089540
:1065300084E061E00E94F86484E061E00E943765D5
:1065400085E061E00E94F86487E061E00E94F86401
:1065500086E060E00E94F86485E061E00E943765B3
:1065600085E060E00E94376587E060E00E94376563
:1065700080E58CBD8DB581608DBD08951F93CF934F
:10658000DF93EB01142F9093A00980939F090CB423
:1065900006FC02C00E9498321093A109812F61E08D
:1065A0000E94F8640E9404318FEF60E04FEF0E9478
:1065B0000B3162E070E080E090E00E94436480E094
:1065C0006DE10E946E318823D1F31092A4091092DC
:1065D000A30988E060E070E00E9456318CE060E042
:1065E00070E00E9456318AE06FEF7BE00E945631E6
:1065F00084E060E07CE00E94563186E06FEF71E15C
:106600000E9456310E94693188E26FE370E30E9474
:10661000563180E369EF77EF0E94563180EC6DE0F0
:106620000E94483181EC60E00E94483180E862ECD1
:1066300042E30E940B3186EC62E17CE00E9456311D
:1066400084EC62E10E9448318AEC6CED75E00E94B6
:10665000563184EE68810E94483185EE69810E943E
:10666000483182EE6A810E94483183EE6B810E943C
:10667000483180EE6C810E94483181EE6D810E942C
:10668000483184ED60E10E94483186ED60E071E0C0
:106690000E9456318AEE0E94903180FDFBCF8FE13F
:1066A0000E94273180E86BE140EC0E940B3180E8CA
:1066B0006FE144E00E940B3182E70E949031863006
:1066C00008F08F5FDF91CF911F910895DF92EF92D5
:1066D000FF920F931F93CF93DF93D82E862FBA018B
:1066E000213041F4675F7F4F9B0140E050E06950EB
:1066F00070400EC0223029F020E030E040E050E051
:1067000007C0625070409B0140E050E06E5F7F4FD9
:10671000E82EFF248CED93E0E80EF91E8B01E701D3
:106720000FC0F881E0E0898190E08E2B9F2BA0E0E4
:10673000B0E0280F391F4A1F5B1F229602501040FD
:106740000230110570F7CB018E7FD701A80FB91F5A
:106750006817790779F08C9190E0A0E0B0E0BA2F4B
:10676000A92F982F882702C040E050E0280F391F3A
:106770004A1F5B1FCA01AA27BB270097A105B105C5
:1067800099F7C90180959095ED2DF0E0E452FC4F0A
:1067900090838183DF91CF911F910F91FF90EF90B4
:1067A000DF9008951092F4031092F50380E4809333
:1067B000F0031092F1038093F20388E16EE044E16C
:1067C00050E020E00E9466330895282F662321F0D0
:1067D000809101048617E1F4809102048823C1F4BA
:1067E000809103048833A1F48091FF038B3781F4F7
:1067F000E22FF92F80912E04838380912F048283CE
:1068000080913004818380913104808381E00895F8
:1068100080E008950F931F93BC010CED13E0C801B5
:106820000E94F74DC80106966CED79E00E94F74D85
:106830001F910F910895EF92FF920F931F937B0189
:106840000E940A340AEF13E0C801B7010E94FF4D0D
:10685000C801049762EE79E00E94FF4D1F910F91ED
:10686000FF90EF900895EF92FF920F931F93CF93B5
:10687000DF937C01EB018A0180EB99E00E941B34DD
:106880008881807F803E49F088819981AA81BB817F
:106890008F5F9F4FAF4FBF4F31F48CED93E061E6B8
:1068A00073E00E94F74D88E08093E8031092E903BB
:1068B0008AEE93E061EB7BE049E050E00E94630ADE
:1068C0001092EC0381E18093F30310930004009392
:1068D0000104F092FE03E092FF0310920204109272
:1068E000040410920504DF91CF911F910F91FF9046
:1068F000EF900895EF92FF920F931F9302EE13E033
:10690000C8010E940A3474E1E72EF12CE00EF11E5A
:10691000C8014896B7010E94FF4DC70162EE79E0B9
:106920000E94FF4D0E94D2331F910F91FF90EF9074
:106930000895BC0181E08093A5098AEE99E00E9448
:10694000FF4D08950F931F938C0188969093EC034D
:106950008093ED030E94D23310920E0410920F0424
:10696000045E1F4F82E36AE1A80122E00E946633C1
:10697000C8014A960E9462321F910F910895FF92BA
:106980000F931F93CF93DF93EC01F62E042F10E0AB
:106990008091B8099091B909A091BA09B091BB0949
:1069A0002B2F33274427552720930204A093030459
:1069B0009093040480930504F0920B04CE010E948E
:1069C000A2341F5F011720F79E0140E050E0809144
:1069D000B8099091B909A091BA09B091BB09820F89
:1069E000931FA41FB51F8093B8099093B909A09372
:1069F000BA09B093BB09DF91CF911F910F91FF901E
:106A00000895CF93DF939C01862F806180930B04C0
:106A1000643029F02115310511F421E030E0909126
:106A200000048091FE03809300049093FE039091F4
:106A300001048091FF03809301049093FF03C5E05C
:106A4000D4E08881A901480F511D2C814C832883F3
:106A5000252F3327219754E0C130D50791F71D86A4
:106A60001E8680E589871092EC0388E28093ED030F
:106A70000E947A3484E08B871C8682E36AE14CE1D1
:106A800050E022E00E94663386E390E00E9462328A
:106A9000DF91CF9108958091B6099091B70960E098
:106AA0000E9401358091020490E0A0E0B0E0BA2F8E
:106AB000A92F982F882720910304820F911DA11DD3
:106AC000B11DBA2FA92F982F882720910404820F77
:106AD000911DA11DB11DBA2FA92F982F8827209194
:106AE0000504820F911DA11DB11D8093B8099093DB
:106AF000B909A093BA09B093BB090895E82FA091F2
:106B0000EC03B091ED03F0910A044091000450E0D1
:106B1000292F30E04217530709F08EC080910104FD
:106B20008E1709F089C080910B04E82F81FF4EC0B9
:106B30001092EC038CE28093ED030E947A3482E1A0
:106B400080930B04909100048091FE0380930004D5
:106B50009093FE03909101048091FF0380930104C0
:106B60009093FF03E5E0F4E021E030E08081A901AB
:106B7000480F511D44831082252F3327319754E04D
:106B8000E130F50799F715861686118212828091F9
:106B90002902838314828D5F8093290282E0818B96
:106BA00084E0828B95E0938B148A80E681879387BB
:106BB00088E7848782E36AE140E250E022E00E94B5
:106BC00066338AE390E00E94623236C084FF34C0AC
:106BD0004F2F50E084E0559547958A95E1F79A2F1D
:106BE00080E02B2F30E0282B392BCA01880F991F0A
:106BF000880F991F281B390B2451304037FF02C0E2
:106C000020E030E03093B7092093B609232B69F0D8
:106C10009A01220F331F220F331F2E5D3F4F685002
:106C200070406217730740F009C0E0FF05C080E0C4
:106C300090E060E00E94013520E030E0C901089555
:106C40000F931F93DF93CF930F92CDB7DEB78C01D5
:106C5000045E1F4F1093EC030C511040802F845E94
:106C60008093ED0389830E94D233085F1F4F1093F6
:106C700002048981845180930304085F1F4F88E2D6
:106C80006AE1A80121E00E946633C8014A960E9489
:106C900062320F90CF91DF911F910F910895FF9273
:106CA0000F931F939C01F62E80EB99E0B9010E948F
:106CB0001B3408EE13E088E08093E8031092E903A8
:106CC000C801029661EB7BE049E050E00E94630A54
:106CD0008CE48093ED0381E18093F3030E94D2332F
:106CE000109200048BE7809301048AE08093FE03F6
:106CF000F092FF031092020488E380930304109241
:106D0000040410920504025E1F4F80E3F801119203
:106D10008A95E9F7C80168E67CE04AE050E00E9405
:106D2000630A88E26AE140E450E021E00E946633B1
:106D30008AE590E00E9462321F910F91FF900895C2
:106D4000EF92FF920F931F93BC0180EB99E00E949A
:106D50001B3408EE13E038E0F32EF092E8031092B3
:106D6000E903C801029661EB7BE049E050E00E9434
:106D7000630A84E58093ED03EE24E394E092F30349
:106D80000E94D233F092FE031092FF03109200048F
:106D90001092010485E0809302048091E5098093BC
:106DA000030410920404E0920504C8014E9662E4C4
:106DB00070E048E350E00E94820A84E262E240E42C
:106DC00050E020E00E94663382E690E00E9462324A
:106DD0001F910F91FF90EF900895DF92EF92FF9235
:106DE0000F931F93CF93DF93EC018091FA098823CF
:106DF00019F0CE010E94AB3B209709F0BFC08091F3
:106E0000A5098570F1F18091260290912702892BC6
:106E1000C1F50E949A318823A1F181E693E00E9496
:106E20000A3488E08093E803A6E0FA2EF092E903A2
:106E30008AEE93E069EA7BE048E050E00E94630A52
:106E40000CEF13E0D8011D92FA94E9F7C8010A97F4
:106E50006CED79E00E94F74DC80106966AEE79E084
:106E60000E94FF4DC801049762EE79E00E94FF4D39
:106E70008091A50988608093A5098AE290E00E942C
:106E80006232809126029091270201969093270208
:106E9000809326028091A609813009F002C2809178
:106EA000A50981FFFEC102E00093A6098091280296
:106EB0008F5F809328028F711091A7091295110F8F
:106EC000107E182BE090A809D090A90980EB99E0DA
:106ED00066EF79E00E941B34F8E0FF2EF092E803A1
:106EE0001092E9038AEE93E061EB7BE049E050E029
:106EF0000E94630A8CE28093ED0386E08093F303A3
:106F00000E94D233E0920004D09201048BE080937F
:106F1000FE031093FF03E2E0F4E0DF011D92FA9418
:106F2000E9F780912902809304048D5F8093290200
:106F300080E680930A0400930B0483E080930C04A2
:106F400010920D0410920E0410920F04109210046F
:106F5000109211040093120484E0809313040093B0
:106F6000140486E28093150482E36AE140E250E073
:106F700022E00E9466338AE390E0AEC08091FA037B
:106F80008F3E79F48091FB038F3F59F48091FC038D
:106F90008F3F39F48091FD038A3F19F42AE230E0F3
:106FA00082C1C932D10508F47CC11091E8031830C0
:106FB00009F082C18091E903863009F07DC182E049
:106FC00094E062EE79E044E050E00E946C0A0097A1
:106FD00009F072C18091F103813029F582EE93E0CE
:106FE0000E940A341092F00382E08093F1038CEF48
:106FF00093E062EF73E00E94F74D82EF93E06CED57
:1070000079E00E94F74D82E094E068EF73E00E941F
:10701000FF4D88EF93E062EE79E00E94FF4D8AE237
:1070200090E00E9462328091A50983FF3AC11091DD
:10703000F103123009F035C188EF93E06AEE79E090
:1070400044E050E00E946C0A009709F02AC180EBEE
:1070500099E062EF73E00E94F74D1093A50921C1FA
:10706000183009F01EC18091E903882309F019C185
:107070008091EA03853409F014C18AEF93E062EE4F
:1070800079E044E050E00E946C0A009709F009C1E1
:107090008091F303813019F58091FE038830F9F473
:1070A000E091AA09F091AB09309719F086EF93E0CF
:1070B00009950E947A341092FE0380910004883F63
:1070C00028F0809101048F5F809301048091000477
:1070D000885F80930004CE010E946232E2C00E9469
:1070E000503D882351F08091F303813131F4CE017A
:1070F0000E94553D882309F0D4C0C633D10528F439
:107100008091F303863009F0CCC0809100048B306D
:1071100009F0BEC086EF93E066EF79E044E050E00E
:107120000E946C0A009709F0BCC080910B04382FB4
:1071300082FF13C0E091AC09F091AD09309759F08E
:107140008091010482958695877063E040E050E06D
:1071500020E030E0099585E090C09091EC0380E05C
:107160002091ED03022F10E0082B192B80910A04C7
:10717000482F50E0E4E055954795EA95E1F7CA01BC
:10718000880F991F880F991F081B190B0451104075
:1071900017FF02C000E010E08091A609823079F567
:1071A00031FF21C034FF1FC080E090E060E00E940A
:1071B000013588E180930B04E091AE09F091AF09AD
:1071C000309719F420E030E007C08091FF038295EA
:1071D0008695877009959C0183E08093A609C90173
:1071E0000E94A2345EC081E08093A60934FF03C0F0
:1071F00080E090E002C0C801019664E046C08330A0
:1072000081F50115110579F1E091AC09F091AD0915
:10721000309749F1440F551F440F551FCE01089771
:107220004E5D5F4F8417950708F4AC01C801840FC9
:10723000951FC817D90710F0980103C09E01241BA1
:10724000350B8091010482958695877060E00995E1
:107250008091FB09882319F0C80168E016C0C801B5
:1072600008C08530F1F030FF0BC08330D1F0C80189
:10727000019669E00E94013586E08093A60911C05D
:107280000115110571F0C80160E00E94013509C0C7
:1072900080912A0290912B02BE010E947E359C01B2
:1072A00002C020E030E0C901DF91CF911F910F9122
:1072B000FF90EF90DF900895CA32D10508F0D0CE4C
:1072C000F0CFBC018091F3038130A1F48091FE03E3
:1072D000882381F480910604823461F486EF93E080
:1072E00044E050E00E946C0A9C0180E0232B19F4DA
:1072F00081E0089580E008950F931F93CF93DF936B
:107300009C01EB018A011092FA09009729F082EEA4
:1073100099E0B9010E94FF4D209719F0CE010E941B
:1073200099340115110529F082EF99E0B8010E9406
:10733000FF4D81E0DF91CF911F910F910895AF92A2
:10734000BF92CF92DF92FF920F931F93CF93DF9361
:107350008C01EB01F42E1092FA0938E341E050E081
:1073600060E070E018C0832F90E0FC01B3E0F59579
:10737000E795BA95E1F7E454F64F877090705A019B
:107380006B0104C0AA0CBB1CCC1CDD1C8A95D2F777
:1073900020812A292083315031F78CED99E0BE01FC
:1073A0000E94F74DC8016CED79E04F2D0E94BE326E
:1073B000DF91CF911F910F91FF90DF90CF90BF9001
:1073C000AF900895CF92DF92EF92FF920F931F93A9
:1073D000DF93CF93CDB7DEB7EB84FC84CD84DE841E
:1073E000DE011F9601C0D801F6018491882309F4BB
:1073F000BCC00894C11CD11C843209F099C0F601AC
:107400000894C11CD11C8491863409F45FC0873470
:1074100034F4843469F0853409F08AC06EC08C3449
:10742000C9F1833509F445C0883409F081C00DC025
:107430008D010E5F1F4FF701668177818D919C91C1
:107440004AE050E00E94470B7EC02C91822F992782
:1074500087FD909514E0959587951A95E1F78F70C3
:107460002F702A300CF0295F8A300CF0895F8D0173
:107470000E5F1F4FF701A681B781805DFD018193EB
:10748000205D11962C933196D7011796FC93EE93BD
:107490001697A9CF8D010C5F1F4F6D917D918D9136
:1074A0009C91F701468157812AE030E00E94850BCC
:1074B0004AC08D010E5F1F4F6D917C91D7011696CA
:1074C0008D919C9117970E949F0A3DC08D010E5F80
:1074D0001F4F2D913C910AC0D7011696ED91FC915A
:1074E000179781931796FC93EE931697F9012F5FE8
:1074F0003F4F8491882381F776CF8D010E5F1F4F18
:107500002D913C910AC0D7011696ED91FC911797E9
:1075100081931796FC93EE931697F999FECF32BD9F
:1075200021BDF89A80B52F5F3F4F882361F75BCF6D
:10753000F70126813781F90181939F01F701378394
:1075400026838D0150CFD70116968D919C91179768
:10755000FC0101900020E9F73197E81BF90B8E0F31
:107560009F1FF701978386833ECFCF91DF911F91B5
:107570000F91FF90EF90DF90CF900895DF93CF931E
:1075800000D000D000D0CDB7DEB7DE011196E7E61F
:10759000F3E086E001900D928150E1F786E191E001
:1075A000ECEDF3E0DF019C011D9221503040E1F74A
:1075B0008091FC09833019F46EEE79E003C0BE01BE
:1075C0006F5F7F4F84E490E043E450E00E943334E7
:1075D0008091FC09833039F08CED93E0BE016F5F40
:1075E0007F4F0E94F74D81E080930604809307044B
:1075F00086E0809308048091090A90910A0AA0917C
:107600000B0AB0910C0A80930A0490930B04A09388
:107610000C04B0930D048091FC09833039F486E0AA
:1076200094E00C9662EE79E00E94FF4D82E294E0D5
:107630006CED79E00E94F74DA2EFB4E0E3E4F2E0F4
:1076400002C081918D9332E0E934F307D1F7909134
:10765000FC09992311F083E001C081E08093F804D4
:107660008DE38093F90487E08093FA0481E08093AE
:10767000FB04ACEFB4E0ECEDF9E002C081918D9336
:1076800089E0E23EF807D1F78CE08093020580E1C3
:1076900080930305ECE2F2E0A4E0B5E002C0819142
:1076A0008D9322E0EC33F207D1F724E135E03093FB
:1076B0000E0A20930D0A913069F582E38093140538
:1076C00084E080931505D9011296E2EEF9E002C03C
:1076D00081918D9339E0E63EF307D1F786E38093FD
:1076E0001A0584E080931B058CE195E090930E0AC7
:1076F00080930D0ADC01EEEEF9E002C081918D93DA
:1077000089E0E23FF807D1F780E295E090930E0A16
:1077100080930D0A20910D0A30910E0AD901EDE3F4
:10772000F2E002C081918D9382E0E334F807D1F753
:10773000C901069690930E0A80930D0A86509440D4
:107740000E94203626960FB6F894DEBF0FBECDBF3E
:10775000CF91DF910895DF92EF92FF920F931F93E5
:10776000CF93DF938C018091FC09823009F4F7C03C
:10777000833030F4882351F1813009F054C14AC07C
:10778000833021F0843009F04EC1E9C00E94356495
:107790002091010A3091020A4091030A5091040A93
:1077A000E090FD09F090FE090091FF091091000A98
:1077B0002E0D3F1D401F511F621773078407950749
:1077C00008F431C10E94BE3A84E017C00E943564BB
:1077D0006093090A70930A0A80930B0A90930C0A2B
:1077E0001092E2091092E3091092E4091092E5095F
:1077F0000E94BE3A0E94693181E08093FC090E9498
:1078000035646093050A7093060A8093070A909383
:10781000080A09C10634110508F4F0C08091FF037D
:10782000833409F0EBC020910A0430910B0440919D
:107830000C0450910D048091090A90910A0AA091BC
:107840000B0AB0910C0A281739074A075B0709F0A1
:10785000D5C0C6EFD4E0FE01A80144525C4FDF0161
:10786000119691819D012F5F3F4F8081853321F4D7
:1078700011968C91823039F0F901E90FF11DE4176E
:10788000F50768F3BBC082EE99E066E174E00E9400
:10789000FF4D5CEDE52E53E0F52EE00EF11EFE01EE
:1078A0003196D9808F010F5F1F4F88818630A9F0F4
:1078B000873030F4813059F0833009F045C00AC078
:1078C0008633E9F18A3361F08333F1F509C086EE3E
:1078D00099E037C08AEE99E034C082EF99E031C078
:1078E000618170E080E090E0982F872F762F6627E7
:1078F000F8012181620F711D811D911D982F872F25
:10790000762F66272281620F711D811D911D982F90
:10791000872F762F66272381620F711D811D911D90
:1079200028EE33E040E050E00E94636A6093010A71
:107930007093020A8093030A9093040A05C08EEEA6
:1079400099E0B8010E94FF4DE801CD0DD11DCE1583
:10795000DF0508F4A4CF0E94BE3A82E04ECF063481
:10796000110508F44BC08091FF03833409F046C031
:1079700020910A0430910B0440910C0450910D04A5
:107980008091090A90910A0AA0910B0AB0910C0A01
:10799000281739074A075B0789F5E6EFF4E0A801E5
:1079A00044525C4FDF01119691819D012F5F3F4F43
:1079B0008081853321F411968C91853039F0F9015D
:1079C000E90FF11DE417F50768F318C00E94643150
:1079D0000E9435646093FD097093FE098093FF094E
:1079E0009093000A8091EA09882321F08AEE99E0B9
:1079F0000E94993483E08093FC0915C00E9435648D
:107A00002091050A3091060A4091070A5091080A10
:107A1000205F384D4F4F5F4F2617370748075907EC
:107A200010F41092FC09DF91CF911F910F91FF90FC
:107A3000EF90DF900895CF93DF9381E08093FA0970
:107A40009091E109892F82958F70805D80933A0231
:107A50009F70905D90933B021092FC090E943564E8
:107A6000EB0104C00E94D9310E94AB3B8091FC091C
:107A7000833061F00E9435646C1B7D0B6053754749
:107A800028F40E949A31882389F3ECCF90E080910A
:107A9000FC09833009F491E0892FDF91CF9108959B
:107AA0008091370A811181E00895CF92DF92EF92A1
:107AB000FF920F931F93CF93DF93CFE0DAE030E094
:107AC000CC24DD2429C02A814B818091000490E0E0
:107AD000042F10E080179107D9F4909101049217B8
:107AE000B9F48C818823A1F02091030430E0285060
:107AF0003040F0900204EE242E0D3F1DE881F98104
:107B0000892F942F66EF73E046E054E0099531E049
:107B10000894C11CD11C25968091370A90E0C816A4
:107B2000D9068CF2832FDF91CF911F910F91FF9097
:107B3000EF90DF90CF9008950F931F938C01FC017D
:107B4000868160E00E94376581E090E00E94B36426
:107B5000F801868161E00E94376581E090E00E9433
:107B6000B364F801868160E00E94376584E690E0A6
:107B70000E94B3641F910F910895CF92DF92EF920C
:107B8000FF920F931F93CF93DF93D82EC92E282FE8
:107B9000392FC9018C01C0E0D0E0E62EFF24F801A6
:107BA000878161E00E94F864B7010C2E02C07595D0
:107BB00067950A94E2F76170F80187810E94376542
:107BC00021960F5F1F4FC830D10549F78D2D9C2D91
:107BD0000E949C3DDF91CF911F910F91FF90EF90FC
:107BE000DF90CF900895CF92DF92EF92FF920F93A4
:107BF0001F93CF93DF93D82EC92E282F392FC90179
:107C00008C01C0E0D0E0E62EFF24F801878161E01E
:107C10000E94F864B7010C2E02C0759567950A940E
:107C2000E2F76170F80187810E94376521960F5F46
:107C30001F4FC430D10549F78D2D9C2D0E949C3DCE
:107C4000DF91CF911F910F91FF90EF90DF90CF9038
:107C500008951F93CF93DF93EC01162F8C81642F2F
:107C60000E9437658D818F3F19F060E00E94376573
:107C70008F8584FF05C0CE01612F0E94BD3D0EC0DF
:107C8000612F70E084E0759567958A95E1F7CE01E4
:107C90000E94F33DCE01612F0E94F33DDF91CF9111
:107CA0001F91089541E00E94293E81E090E00895EF
:107CB00040E00E94293E0895EF92FF920F931F9398
:107CC000CF93DF938C017A016770660F660F660FA2
:107CD00060640E94583EC0E0D0E0D801ED91FC9174
:107CE000D701AC0FBD1F0190F081E02DC8016C9150
:107CF00009952196C830D10581F7DF91CF911F9169
:107D00000F91FF90EF900895FC016089862F8160AC
:107D1000808B6960CF010E94583E0895FC01608904
:107D20006E7F608B68600E94583E0895FC016089F8
:107D3000862F8460808B6C60CF010E94583E08952E
:107D4000DF93CF93CDB7DEB728970FB6F894DEBF99
:107D50000FBECDBF9C01FE013196A5E7B3E088E0E0
:107D60000D9001928150E1F7F9018389481710F0D5
:107D7000482F4150E42FF0E0EE0FFF1FEC0FFD1FE6
:107D80008181680F6068C9010E94583E28960FB62D
:107D9000F894DEBF0FBECDBFCF91DF91089561E0B3
:107DA0000E94583E80ED97E00E94B3640895CF93FF
:107DB000DF93EC01423018F08F8588608F874B8B02
:107DC0001C8A222329F0413019F48F8584608F8723
:107DD00080E593EC0E94B3648C8160E00E9437657B
:107DE0008E8160E00E9437658D818F3F19F060E0E1
:107DF0000E9437656F8564FD1DC0CE0163E00E945F
:107E0000F33D84E991E10E94B364CE0163E00E94F6
:107E1000F33D84E991E10E94B364CE0163E00E94E6
:107E2000F33D86E990E00E94B364CE0162E00E94D7
:107E3000F33D16C06062CE010E94583E84E991E194
:107E40000E94B3646F856062CE010E94583E86E94D
:107E500090E00E94B3646F856062CE010E94583E3C
:107E60006F856062CE010E94583E84E0888BCE010F
:107E70000E94963ECE010E94CF3E82E0898BCE01C9
:107E800066E00E94583EDF91CF9108956F927F92F5
:107E90008F92AF92CF92EF920F931F93DF93CF9376
:107EA000CDB7DEB73C01162F842FF3014483258321
:107EB0000683E782C086A18682869D8593879E85FC
:107EC00094879F8595879889968761E00E94F864DA
:107ED000F30185818F3F19F061E00E94F864F3019E
:107EE000868161E00E94F864112319F0F30117867E
:107EF00003C080E1F3018787C30160E141E020E036
:107F00000E94D73ECF91DF911F910F91EF90CF90BC
:107F1000AF908F907F906F9008958F929F92AF92C5
:107F2000BF92CF92DF92EF92FF920F931F93CF9366
:107F3000DF937B018C01EA012CE330E040E050E06C
:107F40000E94B56A6883C801B7012CE330E040E0C5
:107F500050E00E94B56A122F032FF42EE52E622FF7
:107F6000732F842F952F2CE330E040E050E00E94E7
:107F7000B56A6983612F702F8F2D9E2D2CE330E021
:107F800040E050E00E94B56A122F032FF42EE52E38
:107F9000622F732F842F952F28E130E040E050E0CE
:107FA0000E94B56A6A83612F702F8F2D9E2D28E164
:107FB00030E040E050E00E94B56A79018A01C801D2
:107FC000B7016C5F7F4F8F4F9F4F27E030E040E05D
:107FD00050E00E94B56A6F5F6B8320E0AA24BB2447
:107FE000650101C02F5F822E9924F401EE54F84FF1
:107FF000CF0183709070892B99F4CF0164E670E013
:108000000E94A26A892B39F4CF0160E971E00E94D5
:10801000A26A892B29F48EE691E0A0E0B0E004C0CA
:108020008DE691E0A0E0B0E0A80EB91ECA1EDB1EEE
:10803000C501A0E0B0E0E816F9060A071B0790F6B4
:108040002E83F401EE54F84F83E0882E912C8E227B
:108050009F228114910499F4CF0164E670E00E949C
:10806000A26A892B39F4CF0160E971E00E94A26A0B
:10807000892B29F48EE691E0A0E0B0E004C08DE603
:1080800091E0A0E0B0E0A81AB90ACA0ADB0A980198
:1080900087010A191B092C093D09CF0164E670E02C
:1080A0000E94A26A7C01CF0160E971E00E94A26A8D
:1080B000AC01EDE7F3E060E0613051F4811491042C
:1080C00049F4E114F10441F44115510529F002C0CD
:1080D000808103C08CE101C08DE190E0A0E0B0E0C0
:1080E000081719072A073B0740F0081B190B2A0B32
:1080F0003B0B6F5F31966C30F9F66F5F6D83802FAD
:108100008F5F8C83DF91CF911F910F91FF90EF9044
:10811000DF90CF90BF90AF909F908F900895EF9297
:10812000FF920F931F937B018C0180914F0A9091D6
:10813000500AA091510AB091520AE816F9060A07AE
:108140001B0771F0C801B70144E45AE00E948D3F5B
:10815000E0924F0AF092500A0093510A1093520A8B
:108160001F910F91FF90EF9008950E948F402091F2
:108170004A0A30E02E54384FC90108950E948F40BA
:108180008091490A90E008950E948F408091470AAB
:1081900090E008950E948F408091480A90E00895F1
:1081A0000E948F408091450A90E008950E948F4080
:1081B0008091460A90E008954F925F926F927F926D
:1081C0008F929F92AF92BF92CF92DF92EF92FF92E7
:1081D0000F931F93CF93DF934C01DC0116961C91F4
:1081E000612F70E080E090E020E833E341EE51E061
:1081F0000E94636A5B016C0122EB37E0E12FF0E043
:10820000EE54F84F1DC0C90183709070892BB1F4F2
:10821000C90164E670E00E94A26A892B39F4C901A1
:1082200060E971E00E94A26A892B41F480E891E53F
:10823000A1E0B0E0A80EB91ECA1EDB1E2F5F3F4FA3
:108240002E173F0701F7D40115968C91482E55241F
:10825000C90164E670E00E94A26A7C01C90160E97C
:1082600071E00E94A26A8C01C1E0D0E093E0692E27
:10827000712C6222732227C0C230D10591F461149F
:10828000710479F4E114F10419F40115110549F4AC
:1082900080E89BE3A6E2B0E0A80EB91ECA1EDB1E72
:1082A00011C0FE01E458FC4F608170E080E090E076
:1082B00020E831E541E050E00E94636AA60EB71E57
:1082C000C81ED91E2196C415D505B4F2D401129644
:1082D0006C9170E080E090E020E13EE040E050E012
:1082E0000E94636A7B018C01F401618170E080E08F
:1082F00090E02CE330E040E050E00E94636AE60E3C
:10830000F71E081F191FD4018C91E80EF11C011DE6
:10831000111D14966C9170E061507040882777FDB4
:108320008095982F20E831E541E050E00E94636A93
:10833000E60EF71E081F191FEA0CFB1C0C1D1D1D65
:10834000B701C801DF91CF911F910F91FF90EF907E
:10835000DF90CF90BF90AF909F908F907F906F9065
:108360005F904F9008956093490270934A02809302
:108370004B0290934C02089560933A0A70933B0A23
:1083800080933C0A90933D0A2091490230914A0221
:1083900040914B0250914C02260F371F481F591F26
:1083A00020933E0A30933F0A4093400A5093410A7B
:1083B00082E090E09093430A8093420A0E943564E1
:1083C00060934B0A70934C0A80934D0A90934E0A27
:1083D0000895EF92FF920F931F931CC02F5F3F4FA2
:1083E0004F4F5F4F20933A0A30933B0A40933C0A29
:1083F00050933D0A88EE93E0A0E0B0E0E80EF91E4D
:108400000A1F1B1FE0924B0AF0924C0A00934D0A80
:1084100010934E0A0E943564E0904B0AF0904C0A8B
:1084200000914D0A10914E0A6E197F09800B910B35
:1084300020913A0A30913B0A40913C0A50913D0A02
:10844000685E73408040904048F680913E0A90916B
:108450003F0AA091400AB091410A281739074A07FC
:108460005B07E8F0E091380AF091390A3097B9F0EB
:108470000995611571058105910519F00E94BC41AE
:108480000EC020E030E08091420A9091430A892B8F
:1084900011F021E030E03093430A2093420A6091CA
:1084A0003A0A70913B0A80913C0A90913D0A1F91D3
:1084B0000F91FF90EF9008959093390A8093380AB6
:1084C00080913A0A90913B0AA0913C0AB0913D0AF2
:1084D00080933E0A90933F0AA093400AB093410ACA
:1084E0000E94E9410895482F6AE00E94826A282F7D
:1084F00030E084E0220F331F8A95E1F7842F0E9439
:10850000826A892F820F0895CF93DF93EC018091C7
:10851000530A9091540A8836910559F586EE9CE0ED
:1085200068E670E00E94A06086EE9CE060E00E9439
:10853000226188810E947342682F70E06F777070AB
:1085400086EE9CE00E94226189810E947342682F1E
:1085500086EE9CE00E9422618A810E947342682F0D
:1085600086EE9CE00E9422618B810E947342682FFC
:108570002DC08F36910509F04AC086EE9CE06FE66B
:1085800070E00E94A06086EE9CE060E00E942261A4
:1085900088810E947342682F606886EE9CE00E948A
:1085A000226189810E947342682F86EE9CE00E94BE
:1085B00022618A810E947342682F86EE9CE00E94AD
:1085C00022618B810E947342682F686086EE9CE076
:1085D0000E9422618C810E947342682F86EE9CE08B
:1085E0000E9422618D810E947342682F86EE9CE07A
:1085F0000E9422618E818E510E947342682F86EE06
:108600009CE00E94226186EE9CE00E946561DF9101
:10861000CF91089588E690E09093540A8093530A8E
:1086200086EE9CE068E670E00E94A06086EE9CE02A
:1086300060E00E94226186EE9CE00E9465618823D2
:10864000D9F08FE690E09093540A8093530A86EE17
:108650009CE06FE670E00E94A06086EE9CE060E027
:108660000E94226186EE9CE00E946561882321F0D1
:108670001092540A1092530A08951F93CF93DF93D8
:10868000EC016091530A7091540A6115710509F467
:108690006FC086EE9CE00E94A06086EE9CE060E0E9
:1086A0000E94226186EE9CE00E9465616091530AFF
:1086B0007091540A86EE9CE047E050E00E9476619B
:1086C00086EE9CE00E94B360282F2F7722952F70B2
:1086D0001AE0219F900111248F70820F888386EE0B
:1086E0009CE00E94B360282F22952F70219F90015B
:1086F00011248F70820F898386EE9CE00E94B36004
:10870000282F2F7322952F70219F900111248F7095
:10871000820F8A8386EE9CE00E94B36087708B8311
:1087200086EE9CE00E94B360282F22952F70219F37
:10873000900111248F70820F8C8386EE9CE00E9442
:10874000B360282F22952F70219F900111248F70E4
:10875000820F8D8386EE9CE00E94B360282F2F70DD
:10876000225E82958F70819FC0011124280F2E8375
:10877000DF91CF911F9108950F931F93DF93CF93B4
:10878000CDB7DEB727970FB6F894DEBF0FBECDBFCB
:108790008E010F5F1F4FA8010E948D3FC8010E94EC
:1087A000844227960FB6F894DEBF0FBECDBFCF919F
:1087B000DF911F910F9108950F931F93DF93CF9334
:1087C000CDB7DEB727970FB6F894DEBF0FBECDBF8B
:1087D0008E010F5F1F4FC8010E943D43C8010E94D8
:1087E000DC4027960FB6F894DEBF0FBECDBFCF9109
:1087F000DF911F910F91089586EE9CE00E947A61AF
:1088000008959C01F999FECF32BD21BDF89A80B53B
:1088100008959C01F999FECF1FBA32BD21BD60BDFC
:108820000FB6F894FA9AF99A0FBE0895E091880A63
:10883000F091890A09950895DB01482F50E0405FC7
:108840005F4F84E0440F551F8A95E1F750961C92C4
:10885000509720E030E0F999FECFC901840F951FB1
:1088600092BD81BDF89A80B5FD01E20FF31F8083B0
:10887000882331F02F30310519F02F5F3F4FEBCFB8
:108880000895DB01482F50E0405F5F4F94E0440FB4
:10889000551F9A95E1F750961C92509720E030E0D2
:1088A000FD01E20FF31FE081F999FECF1FBAC90164
:1088B000840F951F92BD81BDE0BD0FB6F894FA9A62
:1088C000F99A0FBEEE2331F02F30310519F02F5FEA
:1088D0003F4FE6CF089586E694E0FC01EC5EF94F49
:1088E000E081F999FECF1FBA92BD81BDE0BD0FB600
:1088F000F894FA9AF99A0FBE019624E08C36920702
:1089000061F7089580E694E0FC01EC5EF94FE081A8
:10891000F999FECF1FBA92BD81BDE0BD0FB6F894A4
:10892000FA9AF99A0FBE019624E08636920761F70B
:108930000895282F277086958695869590E0662362
:1089400069F0FC01E259F54F81E090E002C0880F28
:10895000991F2A95E2F72081282B0DC0FC01E259CE
:10896000F54F81E090E002C0880F991F2A95E2F749
:108970008095208128232083089510926E0A1092FA
:108980006F0A1092700A1092710A1092720A109275
:10899000730A0895EDE4F2E020E030E0F999FECFAB
:1089A00032BD21BDF89A80B580832F5F3F4F379647
:1089B0002332310599F78091B6028F5F80936C0A5C
:1089C00090E023E0880F991F2A95E1F780936D0AC4
:1089D0000895EBE3F3E082E290E02081F999FECF85
:1089E0001FBA92BD81BD20BD0FB6F894FA9AF99ACC
:1089F0000FBE019737972FEF8F3F920771F7809146
:108A0000B6028F5F80936C0A90E033E0880F991F65
:108A10003A95E1F780936D0A0895AC01FB010FC010
:108A2000F999FECF1FBADA01A80FB11DB2BDA1BDE1
:108A300020BD0FB6F894FA9AF99A0FBE31968E2F90
:108A4000861B2081222361F7F999FECF1FBA480FB8
:108A5000511D52BD41BD10BC0FB6F894FA9AF99A57
:108A60000FBE0895582F282F392FF9018E2F851BFF
:108A7000F999FECF90E0805C9F4F92BD81BDF89A3E
:108A800080B59081882331F0992349F0891739F412
:108A90003196ECCF80E0992319F481E0089580E0CD
:108AA00008951092580A1092570A81E793E0909324
:108AB000560A8093550A0895EF92FF920F931F93E1
:108AC000CF93DF93E82E162F042FF22E662321F08A
:108AD000623081F4222371F08E2D0E948B65892BE8
:108AE00011F000E024C0FF2011F480E001C080E814
:108AF000082B1DC0C0E0D0E08E2D0E948B65892B15
:108B000081F4113031F0123061F483E0C032D807C3
:108B100044F461E070E080E090E00E9443642196BC
:108B2000EBCFFF2019F4C052D3400CF00068802F27
:108B3000DF91CF911F910F91FF90EF9008950F93C8
:108B40001F93082F10918A0A107861E070E080E08E
:108B500090E00E9443648FE10E948B65892B21F491
:108B60008FE1602F41E013C08EE10E948B65892B5D
:108B700021F48EE1602F42E00AC08DE10E948B65F6
:108B8000892B11F040E007C08DE1602F44E0212FD8
:108B90000E945C45482F80918A0A90E08F70907007
:108BA000242F30E0892B39F42F703070232B71F093
:108BB000842F806406C02F703070232B39F4842FEB
:108BC000806240938A0A1F910F910895842FF9CFF4
:108BD0008BE00E948B6540E02091E70230E0821735
:108BE000930709F041E0440F440F80916A0A8B7F9C
:108BF000842B80936A0A0895EF92FF920F931F933C
:108C00008C0145E5E42E4AE0F42E6AE070E00E9413
:108C1000A26AC7014AE050E00E944A67C8016AE0C0
:108C200070E00E94A26ABC01C7014AE050E00E94C5
:108C30004A671F910F91FF90EF900895CF93DF93B4
:108C4000EC0104C085E59AE00E948A66FE01219647
:108C500064916623B9F7DF91CF9108950F931F9325
:108C6000CF93DF938C01462F85E59AE060E00E9468
:108C7000A03EE80104C085E59AE00E948A669E0154
:108C8000201B822FFE01219664916623A1F799276C
:108C900087FD9095C0E1D0E0C81BD90B05C08DE4DD
:108CA0009FE00E941E462197D7FFF9CFDF91CF9119
:108CB0001F910F910895EF92FF920F931F93CF93FF
:108CC000DF937C018C01F3E0000F111FFA95E1F7AF
:108CD000081B190B035B1D4FF8018281938160E033
:108CE0000E942E4686E29FE061E00E942E4685E5C6
:108CF0009AE060E041E00E94A03EF801868180FF9A
:108D000005C085E59AE00E94843E04C085E59AE0AE
:108D10000E948E3EF3E1EF16F10409F45EC084E197
:108D2000E816F10454F4E1E0EE16F104B1F0FCE0D1
:108D3000EF16F10409F08CC065C08BE1E816F10470
:108D400009F46AC0ECE1EE16F10409F475C0F4E12F
:108D5000EF16F10409F07CC047C080915402C82F7F
:108D6000D0E0E097D7FD05C084E29FE00E941E4658
:108D700007C082E29FE00E941E46D095C195DF4F5A
:108D8000CE0164E070E00E94A26A85E59AE04AE0C4
:108D900050E00E944A6780E29FE00E941E46CE019A
:108DA00064E070E00E94A26ABC01E4E0660F771FF5
:108DB000EA95E1F7681B790B29F48DE19FE00E94A9
:108DC0001E4606C085E59AE04AE050E00E944A67E8
:108DD00088E19FE00E941E4661C086E19FE00E94FC
:108DE0001E466091D20220C08091D9028C3320F0BF
:108DF00084E19FE00E941E466091D90270E06C53AE
:108E0000704007C07091A80260E08091A102680FD5
:108E1000711D85E59AE00BC060910A038DE070E05A
:108E20000E94006660910A0385E59AE070E04AE0DE
:108E300050E00E944A6732C0809111036FEF70E0EA
:108E4000681B71098CE00E94006660911103ECCFF1
:108E5000F70153E0EE0FFF1F5A95E1F7EE19FF09F6
:108E6000E35BFD4F81816081813051F4662319F409
:108E70008DE09FE002C080E19FE00E941E4607C097
:108E800085E59AE070E04AE050E00E944A6787E199
:108E9000E816F10419F48BE09FE011C0C701439775
:108EA000029720F0E8E1EE16F10419F486E09FE065
:108EB00006C0F1E1EF16F10421F481E09FE00E9489
:108EC0001E46DF91CF911F910F91FF90EF90089573
:108ED000EF92FF920F931F93182F092F0E945B466A
:108EE000212F302FC9018C018AEAE82E82E00E94EE
:108EF0009F45482F282F30E0C9018F709070823035
:108F00009105D9F08430910561F1019709F068C0AD
:108F1000F801B3E0EE0FFF1FBA95E1F7E01BF10B8C
:108F2000E35BFD4F868180FF5EC090818181891760
:108F300009F459C09F5F908356C0F801A3E0EE0F7B
:108F4000FF1FAA95E1F7E01BF10BE35BFD4F868164
:108F500080FF46C08081882309F442C0815080830D
:108F60003FC046FF3DC047FF0BC080913B038823B5
:108F700011F0E0923B030E94E944FF24F39434C0D3
:108F80000330110541F480916202882309F1FF2426
:108F90000CE010E029C00C30110521F4FF240EE094
:108FA00010E022C00531110541F48091E0028823D0
:108FB00079F4FF2407E110E017C00231110541F4F4
:108FC0008091CB02882321F4FF2405E110E00CC03E
:108FD000C801019663E270E00E94A26A8C0103C09E
:108FE000442309F483CFFF24C8010E945B46FF207D
:108FF00009F47CCF85E59AE00E948E3E1F910F9187
:10900000FF90EF9008950F931F93CF93DF93482F16
:10901000062F85E59AE060E00E94A03E80916B0AF1
:109020008F7019F48CE39FE010C08AE39FE00E94E8
:109030001E4660916B0A6F7085E59AE070E04AE029
:1090400050E00E944A6788E39FE00E941E4680919C
:109050006A0A80FD06C08CE29FE061E00E942E4615
:1090600026C0E0916B0AEF70F0E0E259F54F1081F5
:10907000C1E0D0E080916B0A8F7051F48091CB02F7
:1090800090E0C817D90721F410FD06C06DE405C0B3
:1090900010FD02C06FE501C0602F85E59AE00E94D7
:1090A0008A662196C930D10511F01695E3CF87E283
:1090B0009FE00E941E4685E59AE06DE041E00E9437
:1090C000A03E80916A0A81FD06C082FF09C080919E
:1090D000E002882329F085E59AE063E00E94523E91
:1090E00085E59AE06EE041E00E94A03E80916A0A28
:1090F00086FF05C085E59AE062E00E94523E85E564
:109100009AE06FE041E00E94A03E60E080916B0A2F
:1091100082958F7090E003970CF061E085E59AE00E
:109120000E94523EDF91CF911F910F910895EF92CF
:10913000FF920F931F93CF93DF938C017B0185E503
:109140009AE00E94CF3E85E59AE060E040E00E9410
:10915000A03EC0E0D0E0F801EC0FFD1F608185E586
:109160009AE070E04AE050E00E944A6782E49FE0A3
:109170000E941E462196C330D10569F7F80163812C
:1091800085E59AE070E04AE050E00E944A6785E594
:109190009AE060E041E00E94A03E80E49FE00E94EF
:1091A0001E4685E59AE0B7014AE050E00E944A6712
:1091B000DF91CF911F910F91FF90EF90089584E080
:1091C0000E94DE659C0183E02E3B380710F080E0B2
:1091D000089583E02734380710F081E0089582E095
:1091E0002B3E380710F082E0089582E0223A3807DB
:1091F00010F083E0089582E02536380710F084E00F
:1092000008952353324010F085E008958FEF0895BC
:1092100020916A0A2170F999FECF1FBA80E390E08D
:1092200092BD81BD20BD0FB6F894FA9AF99A0FBE8F
:1092300020916A0A22952170F999FECF1FBA81E325
:1092400090E092BD81BD20BD0FB6F894FA9AF99ACC
:109250000FBE4091800A5091810A6091820A7091FC
:10926000830A82E390E029E034E40E94210B089510
:10927000F999FECF80E390E092BD81BDF89A90B558
:10928000917080916A0A8E7F892B80936A0AF9997E
:10929000FECF81E390E092BD81BDF89A90B59170C8
:1092A0009295907F80916A0A8F7E892B80936A0ABB
:1092B00082E390E061E074E40E94DF0A6093800A38
:1092C0007093810A8093820A9093830A0895EF92A3
:1092D000FF920F931F93CF93DF9383E060E00E9490
:1092E000376503E71AE080916A0A80FD02C060E0FA
:1092F00002C0F8016081C7E0D0E0E62EFF2486E1DD
:1093000060E00E943765B7010C2E02C07595679525
:109310000A94E2F7617085E10E94376586E161E0B9
:109320000E9437652197FFEFCF3FDF0741F70150DC
:1093300010408AE00D361807B1F683E061E00E9424
:109340003765DF91CF911F910F91FF90EF900895B6
:1093500080916A0A8D7F80936A0A1092800A109227
:10936000810A1092820A1092830A0E9408490E9480
:109370006749089580916A0A826080936A0A0E9410
:1093800008490E946749089580916A0A8E7F8093F8
:109390006A0A0E9467490E940849089580916A0AF2
:1093A000816080936A0A0E9467490E940849089573
:1093B000AF92BF92CF92DF92FF920F931F93CF9302
:1093C000DF935B016C01FF24C1E0D0E03CC085E588
:1093D0009AE00E94CF3E85E59AE060E040E00E947E
:1093E000A03E0F2D10E0B8016F5F7F4F85E59AE03A
:1093F0004AE050E00E944A6710926E0A10926F0A8B
:109400001092700A1092710A1092720A1092730AE6
:1094100093E0169507959A95E1F70259154F8F2D10
:1094200087709E0102C0220F331F8A95E2F7C9019F
:10943000F8012081282B20830E946749C601B501CD
:109440000E944364F39480916D0AF81608F4BFCF2C
:10945000FF24FBCF64EF71E080E090E00E94436462
:10946000F999FECF12BC11BCF89A90B5943620F44D
:109470008AE0989F902D11249F3C59F4F999FECFD2
:1094800082E290E092BD81BDF89A80B58A3A09F0F7
:1094900091C00E94E9440E94084980E490E063E89A
:1094A00071E00E940D4580E690E06CE871E00E945A
:1094B0000D4580E890E066E971E00E940D458FE877
:1094C0009FE060E00E942E4680E89FE061E00E94FD
:1094D0002E4680E091E0F999FECF1FBA92BD81BD82
:1094E00010BC0FB6F894FA9AF99A0FBE019628E0CC
:1094F0008030920781F720E031E0E1E0F0E043E5E1
:10950000F999FECF1FBA32BD21BD40BD0FB6F89408
:10951000FA9AF99A0FBEF999FECF1FBA2F5F3F4F03
:1095200032BD21BD21503040CF016AE070E00E9481
:10953000A26A605D60BD0FB6F894FA9AF99A0FBE00
:10954000F999FECF1FBA2E5F3F4F32BD21BDCF012B
:109550006AE070E00E94A26A805D80BD0FB6F89458
:10956000FA9AF99A0FBE225F3F4F84E02030380705
:1095700011F03196C5CF80E694E02FEFF999FECF38
:109580001FBA92BD81BD20BD0FB6F894FA9AF99A20
:109590000FBE019634E08636930781F764EF71E0E1
:1095A00080E090E00E944364E091880AF091890A8B
:1095B000099528C00E94CA4420E634E0F999FECFFC
:1095C00032BD21BDF89A80B5F901EC5EF94F808378
:1095D0002F5F3F4F84E02636380781F726E634E0D8
:1095E000F999FECF32BD21BDF89A80B5F901EC5E44
:1095F000F94F80832F5F3F4F84E02C36380781F787
:109600000E94384980E00E949F4590E08F709070E2
:109610008230910521F18430910521F1019709F003
:109620004CC064E670E080E090E00E9443648DE10D
:109630000E948B65892B29F460E273E080E090E062
:109640000BC06091F50270E080E090E028EE33E01E
:1096500040E050E00E94636A0E94D8492EC082E236
:1096600090E020C080E79FE060E00E942E4660ED21
:1096700077E080E090E00E9443648FE59FE060E047
:109680000E942E468FE49FE061E00E942E4680E01B
:109690000E949F4586FFFBCF85E59AE00E94CF3E62
:1096A00080E090E00E94684780913B03882329F086
:1096B000E091880AF091890A09958CE061E00E94A6
:1096C000F8648DE061E00E94F86460910A038DE027
:1096D00070E00E940066809111036FEF70E0681BDC
:1096E00071098CE00E9400660895DF93CF93CDB797
:1096F000DEB727970FB6F894DEBF0FBECDBFCE0101
:1097000001960E943D438C8190E0059667E070E0F1
:109710000E94A26A27960FB6F894DEBF0FBECDBF97
:10972000CF91DF910895DF92EF92FF920F931F93F5
:10973000D82E0E94E9417B018C0185E59AE060E02A
:109740004D2D0E94A03EC801B7010E94D6400E9444
:10975000FC458BE49FE00E941E46C801B7010E94B1
:10976000D0400E94FC4588E49FE00E941E460E9473
:10977000754BE82FF0E0EE0FFF1FEE5BFC4F808192
:1097800091810E941E4686E49FE00E941E46C80109
:10979000B7010E94BE400E94FC4584E49FE00E9405
:1097A0001E46C801B7010E94CA400E94FC451F9195
:1097B0000F91FF90EF90DF9008958F92AF92CF922C
:1097C000EF920F931F93DF93CF93CDB7DEB7A097A0
:1097D0000FB6F894DEBF0FBECDBF83E061E00E94FC
:1097E000F86481E061E00E94F86486E161E00E9433
:1097F000F86485E161E00E94F86483E061E00E9422
:10980000376581E061E00E94376510926E0A109220
:109810006F0A1092700A1092710A1092720A1092D6
:10982000730A0E94674981E060E00E94376580E02A
:1098300061E00E94F86480E061E00E94376511E019
:10984000109381008CE061E00E94F8648DE061E09B
:109850000E94F86460910A038DE070E00E94006647
:10986000809111036FEF70E0681B71098CE00E941A
:10987000006600D000D0EDB7FEB73196ADB7BEB7E9
:1098800011961C9211821282138285E59AE061E0A2
:1098900043E12FEF02E1E4E1EE2E75E1C72E56E140
:1098A000A52E37E1832E0E94463F0F900F900F9018
:1098B0000F9085E59AE060E142E020E00E94D73E0B
:1098C0008BE060E00E94F8648BE061E00E94376505
:1098D00086EE9CE00E947A6180916A0A81608178BC
:1098E00080936A0A10926B0A10936C0A88E0809346
:1098F0006D0A1092800A1092810A1092820A1092C8
:10990000830A1092840A1092850A1092860A109295
:10991000870ADE011196E1EAF3E001900D92815091
:10992000E1F7DE011996E9E9F3E088E001900D9294
:109930008150E1F7DE015196E1E9F3E088E0019022
:109940000D928150E1F7DE015996E9E8F3E088E0F5
:1099500001900D928150E1F785E59AE061E08E017A
:109960000F5F1F4FA8010E945C3E1A821B8281E09C
:109970008C8385E59AE060E0A8010E945C3E85E565
:109980009AE062E0AE01475F5F4F0E945C3E85E572
:109990009AE063E0AE014F5E5F4F0E945C3E85E55A
:1099A0009AE064E0AE01475E5F4F0E945C3E8CE14E
:1099B00061E00E94F8648CE160E00E9437658FE10D
:1099C00060E00E94F8648EE160E00E94F8648DE13E
:1099D00060E00E94F8648FE161E00E9437658EE1EB
:1099E00061E00E9437658DE161E00E9437650E9469
:1099F0000A43882329F480916A0A806280936A0A64
:109A0000A0960FB6F894DEBF0FBECDBFCF91DF9109
:109A10001F910F91EF90CF90AF908F9008950F937B
:109A20001F93DF93CF93CDB7DEB728970FB6F89487
:109A3000DEBF0FBECDBFFC018B0180910303858388
:109A400084E893E0BF0144E00E949F39882311F429
:109A500090E032C010932B0200932A0280916202A0
:109A6000882319F00E941B3D21C0809169028983DF
:109A7000809170028A83809177028B8380917E022D
:109A80008C83809185028D8380918C028E8380915E
:109A900093028F8380919A028887CE010196BE013E
:109AA0006B5F7F4F40E050E00E947C3990E088235C
:109AB00009F491E081E09827892F28960FB6F89451
:109AC000DEBF0FBECDBFCF91DF911F910F910895E3
:109AD000CF93DF93DC01EB01722F632F822F932F43
:109AE0009C01F90150E016C08081981771F43196FD
:109AF0008081882371F411968C918D3331F4872FF6
:109B0000962F9C01F90151E004C0872F962F9C01EC
:109B1000F90111969C91992339F0903229F09A30ED
:109B200019F0552309F304C0513011F030E018C08A
:109B30006A2F50E04150504002C0299311963A2FAD
:109B4000361B2C91222359F0203249F02A3039F06B
:109B5000263229F0832F90E08417950774F318823A
:109B6000832FDF91CF910895CF93DF93FC01EC0118
:109B700037C08B3211F480E231C0853279F5DF01D4
:109B800011969181392F30533A3070F0892F8156D8
:109B9000863010F4375208C0892F8154863010F077
:109BA00030E002C0392F3753FD01319611962C91C8
:109BB000922F90539A3070F0822F8156863010F495
:109BC000975208C0822F8154863010F090E002C076
:109BD000922F9753832F8295807F892B899331967B
:109BE0008081882331F61882DF91CF910895DC01BE
:109BF000FB0186E001900D928150E1F708959C01F0
:109C0000FB0180819181A281B381F90180839183DD
:109C1000A283B383089540E082E002C0880F4F5FC3
:109C2000861710F44630D1F7242F30E0C9019595FE
:109C3000879580658CBD40FF02C080E004C080E055
:109C4000463009F081E08DBD089584E061E00E9416
:109C5000376584E061E00E94F86486E060E00E947D
:109C6000F86485E061E00E94F86487E061E00E94AA
:109C7000F86408954E960E94685808954E960E9482
:109C8000A0580895CF93DF93EC01662331F06E96D0
:109C9000D0938C0AC0938B0A6E9788A1882321F0F9
:109CA000CE014E960E94EA51CE014E962596BE01F7
:109CB0000E943A4FDF91CF9108950F931F93CF9356
:109CC000DF93EC010E948F5F8823C9F08E010B5F48
:109CD0001F4FC801BE0141E00E947859882339F422
:109CE000C801BE0140E00E947859882341F0CE01AE
:109CF00061E00E94424E882319F081E001C080E0BB
:109D0000DF91CF911F910F9108950F931F93CF93E0
:109D1000DF93DC01EB018A0180E090E020E2FE01AC
:109D2000E80FF91F208301968B309105C1F757E0AA
:109D300040E024C0622F2E3219F080EA9FE007C075
:109D40005A3051F15AE048E018C0321729F1FC01AD
:109D5000019634913323C9F75417F0F02132E0F023
:109D60002F37D0F4822F81568A3110F4622F60523F
:109D7000FE01E40FF11D60834F5F11962C912223A9
:109D800011F02F32B9F6F801B183A08390E08881F9
:109D9000803219F091E001C090E0892FDF91CF91DE
:109DA0001F910F910895CF92DF92EF92FF920F9340
:109DB0001F93DF93CF9300D000D0CDB7DEB77C01E7
:109DC000FC0186899789A08DB18D89839A83AB83A5
:109DD000BC8300E010E06E010894C11CD11C4981D5
:109DE0005A816B817C81D70114968D919C91159736
:109DF00096010E941F5B882379F1D7011496ED919B
:109E0000FC9115978481080F111DB0E100301B07EC
:109E100018F529813A814B815C818289803131F446
:109E2000285F3F4F40405040D0F205C0285F3F4F71
:109E30004F4F5F40A0F2C801A0E0B0E029E0880FDA
:109E4000991FAA1FBB1F2A95D1F7F701828B938B0D
:109E5000A48BB58B81E001C080E00F900F900F9034
:109E60000F90CF91DF911F910F91FF90EF90DF90B6
:109E7000CF900895CF93DF93EC01FB018A81882373
:109E8000D1F57D836C8382898031C9F582E08A8334
:109E90001E8A1F8A188E198E83899489A0E0B0E0EB
:109EA00035E0880F991FAA1FBB1F3A95D1F78A8BFF
:109EB0009B8BAC8BBD8B0FC083E08A838589968991
:109EC000A789B08D8E8B9F8BA88FB98FCE010E94F2
:109ED000D34E882381F081E089831E821F821886F9
:109EE00019861A861B861C861D861E861F86188A62
:109EF000198A1B8201C080E0DF91CF9108958032E2
:109F0000D1F7DACF6F927F928F929F92AF92BF92EA
:109F1000CF92DF92EF92FF920F931F93CF93DF9335
:109F2000EC017A018B012A81222309F480C08A89FD
:109F30009B89AC89BD8984179507A607B70708F4E4
:109F400076C085C0E114F1040105110551F41E82AB
:109F50001F82188619861A861B861C861D8681E03C
:109F600067C02A853B854C855D85EC81FD818185B7
:109F700090E00996215030404040504039014A015C
:109F8000082E04C096948794779467940A94D2F725
:109F90002F5F3F4F4F4F5F4F0894E108F1080109D1
:109FA00011095701680104C0D694C794B794A794C7
:109FB0008A95D2F70894E11CF11C011D111DA6140D
:109FC000B704C804D90428F021153105410551050D
:109FD00049F48E899F89A88DB98D8E839F83A88728
:109FE000B98716C0A618B708C808D90811C04E818D
:109FF0005F81688579858C819D8194010E941F5BBA
:10A000000894A108B108C108D108882331F40FC011
:10A0100046E0842E912C8C0E9D1EA114B104C10427
:10A02000D10429F7EA86FB860C871D8798CF80E04C
:10A03000DF91CF911F910F91FF90EF90DF90CF9024
:10A04000BF90AF909F908F907F906F900895223037
:10A0500009F078CFE7CFCF93DF93EC01462F6E85E1
:10A060007F85888999890E943459AC01009719F439
:10A0700020E030E00AC08B81282F30E065E0220F1D
:10A08000331F6A95E1F7240F351FC901DF91CF9186
:10A0900008950F931F93CF93DF938C01FC0182816E
:10A0A0008823F1F1818187FF38C0C80161E00E94F7
:10A0B0002B50EC010097A1F18881853E89F1F801D0
:10A0C0008281823040F482899389A489B5898C8FFA
:10A0D0009D8FAE8FBF8FF801868997899B8F8A8F5E
:10A0E00086899789A08DB18DCD01AA27BB279D8B2D
:10A0F0008C8BE0918D0AF0918E0A309751F0BE0161
:10A100006A5E7F4FCE0148960995888D998D9B8B0D
:10A110008A8BF80181818F7781830E94EC5804C07B
:10A1200081E0F801808380E0DF91CF911F910F9152
:10A1300008956F927F928F929F92AF92BF92CF922B
:10A14000DF92EF92FF920F931F93DF93CF9300D094
:10A1500000D0CDB7DEB77C015A016B01DC0112964D
:10A160008C911297813009F091C011968C9181FFEA
:10A170008DC0A0C00097A105B10511F481E087C092
:10A18000F7016284738484849584C701B601A501B4
:10A190000E94824F882309F479C0D70114968D91CB
:10A1A0009C911597A114B104C104D10489F4569669
:10A1B0004D915D916D917C9159970E948E5B8823A2
:10A1C00009F464C0F701168A178A108E118E44C0F4
:10A1D000D70116964D915D916D917C9119979E01D5
:10A1E0002F5F3F4F0E941F5B882309F44FC0D701A8
:10A1F0001496ED91FC91159749815A816B817C8170
:10A200008289803149F4483FBFEF5B07B0E06B07BC
:10A21000B0E07B0748F020C0483F8FEF58078FEF32
:10A2200068078FE07807C0F4CF010E948E5B882317
:10A2300069F1D70116964D915D916D917C911997B9
:10A2400014968D919C9115970FEF1FEF2FEF3FE024
:10A250000E94AF5A8823D1F0F701A28AB38AC48A38
:10A26000D58A818180688183C7010E9449508823F3
:10A2700069F0B601A5016A147B048C049D0410F4F6
:10A28000B401A301C7010E94824F01C080E00F907A
:10A290000F900F900F90CF91DF911F910F91FF9032
:10A2A000EF90DF90CF90BF90AF909F908F907F9076
:10A2B0006F900895F70182899389A489B5898417DD
:10A2C0009507A607B70708F055CFE0CF1F93CF93A8
:10A2D000DF93EC01142F262F30E0F90185E0EE0F1B
:10A2E000FF1F8A95E1F7EC56F54F8385817121F0C8
:10A2F000842F827109F064C08091940C9091950C28
:10A30000A091960CB091970C8E879F87A88BB98BE4
:10A310006B83F901B5E0EE0FFF1FBA95E1F7EC563C
:10A32000F54F2489358940E050E0A90133272227E1
:10A330002E8B3F8B488F598F828D938DA0E0B0E09C
:10A34000282B392B4A2B5B2B2E8B3F8B488F598F19
:10A35000838590E088719070009751F4848D958D7D
:10A36000A68DB78D8A8B9B8BAC8BBD8B81E008C093
:10A37000409731F5CE010E94D34E882309F184E045
:10A380008A83812F8F7089831E821F821886198687
:10A390001A861B861C861D8614FF18C0CE0140E05D
:10A3A00050E060E070E00E949950882379F408C082
:10A3B0004A895B896C897D89CE010E94824F02C0E7
:10A3C0001A8280E0DF91CF911F91089515FDF0CFA3
:10A3D00081E0F8CF0F931F938C010E944950F80140
:10A3E00012821F910F910895CF93DF93EC0140E00B
:10A3F00050E060E070E00E949950882369F0CE013F
:10A4000061E00E942B50FC01009731F085EE8083C3
:10A410001A820E94EC5801C080E0DF91CF9108952C
:10A420002F923F924F925F927F928F929F92AF9224
:10A43000BF92CF92DF92EF92FF920F931F93DF9321
:10A44000CF93CDB7DEB728970FB6F894DEBF0FBE17
:10A45000CDBF98878F835E834D83DC0112968C91EC
:10A460001297882309F41EC111968C9180FF1AC19E
:10A4700034C1F501EE19FF09FE83ED837A83698308
:10A480008F81988506969C838B834D805E8003C167
:10A49000AF81B8851A962D913D914D915C911D9794
:10A4A0008FEF282E81E0382E222233221496ED9150
:10A4B000FC91159759016A0109E0D694C794B794A5
:10A4C000A7940A95D1F774807A947A2012968C9189
:10A4D000823049F4E588F6880789108DEA0CFB1C68
:10A4E0000C1D1D1D35C02114310411F5772001F517
:10A4F000211531054105510559F4EF81F88586890B
:10A500009789A08DB18D86839783A087B18710C06E
:10A51000AF81B88516964D915D916D917C9119979B
:10A52000CF012B813C810E941F5B882309F4BAC0B4
:10A53000EF81F88546815781608571858481958199
:10A540000E94CC587B018C01E70CF11C011D111DF0
:10A550002114310499F4F0E04F16F2E05F0670F038
:10A560002091940C3091950C4091960C5091970C41
:10A57000E216F3060407150709F0CFC0C801B701BA
:10A5800040E00E943459009709F48CC040E052E04A
:10A590004219530942014415550508F44A019C012A
:10A5A000220D331D89819A81B901A4010E94790A83
:10A5B00059C08091990C90919A0CB801A7012981FA
:10A5C0003A810E945B5F882309F46CC0812C12E001
:10A5D000912E48C0D52CD694AF81B88512968C9117
:10A5E0001297823049F01496ED91FC911597848171
:10A5F00087198D1508F4D82EE216F30604071507FF
:10A6000070F02D0D311D411D511DE216F30604079A
:10A61000150728F40E94EC58882309F443C0809160
:10A62000990C90919A0CB801A7010E94385F882379
:10A63000C9F109811A81FF2408C0B8010E94365E61
:10A6400000501E4F882371F1F3948091990C9091E2
:10A650009A0CFD1490F30E941E5F882319F19D2C23
:10A66000990C8824E981FA81E80DF91DFA83E983C0
:10A67000940140E050E0EF81F88582859385A485C0
:10A68000B585820F931FA41FB51F82879387A48768
:10A69000B587481859084114510409F0F9CE4D8185
:10A6A0005E8102C04FEF5FEFCA0128960FB6F894A3
:10A6B000DEBF0FBECDBFCF91DF911F910F91FF90F5
:10A6C000EF90DF90CF90BF90AF909F908F907F9052
:10A6D0005F904F903F902F900895AF81B88552962C
:10A6E000AD90BD90CD90DC9055971A96ED90FD9071
:10A6F0000D911C911D97ED81FE819F0140E050E07E
:10A70000D601C5018E199F09A00BB10B2817390777
:10A710004A075B0708F0ADCEB1CEF0E04F16F4E08B
:10A720005F0608F057CF45CFDF93CF930F92CDB799
:10A73000DEB7BE016F5F7F4F41E050E00E941052D4
:10A74000019719F02FEF3FEF03C08981282F30E0E8
:10A75000C9010F90CF91DF9108952F923F924F92B0
:10A760005F926F927F928F929F92AF92BF92CF92A1
:10A77000DF92EF92FF920F931F93DF93CF930F928D
:10A78000CDB7DEB72C015B013A01490100E010E0D2
:10A79000EE24EA94FE2C1E010894211C311C13C0E7
:10A7A0000A0D1B1DF80160838114910419F46A30AD
:10A7B00049F41EC0772767FD7095C4010E94940A72
:10A7C0000097B1F4860168010894C11CD11CC6141D
:10A7D000D70444F5C201B10141E050E00E9410529B
:10A7E0007C0181309105F1F469816D30C9F6EBCFC0
:10A7F0008601A00EB11EF5011082C8010F90CF9105
:10A80000DF911F910F91FF90EF90DF90CF90BF905D
:10A81000AF909F908F907F906F905F904F903F9000
:10A820002F900895F7FEE5CF0FEF1FEFE6CFCF9300
:10A83000DF93EC019C012A5F3F4F8C819D8141E0B9
:10A8400050E060E070E00E94F55B8823A1F08E8903
:10A850009F89A88DB98D0097A105B10559F48E8106
:10A860009F81A885B9858E8B9F8BA88FB98F898191
:10A870008068898381E0DF91CF9108953F924F9264
:10A880005F926F927F928F929F92AF92BF92CF9280
:10A89000DF92EF92FF920F931F93DF93CF93CDB789
:10A8A000DEB72A970FB6F894DEBF0FBECDBF4C01BE
:10A8B000162F072F5A874987DC0112968C91129721
:10A8C000813009F0B0C111968C9181FFACC1C9C132
:10A8D000F401428953896489758982859385A485A9
:10A8E000B58584179507A607B70731F0C4010E9404
:10A8F000824F882309F497C1812F902F9C013887BC
:10A900002F8329853A853E832D8351C1D401149626
:10A91000ED91FC911597DA01C90119E0B695A7955B
:10A92000979587951A95D1F7F480FA94F8228901C2
:10A930001170FF2009F052C00115110509F04EC039
:10A94000D40116964D915D916D917C9119974115A9
:10A9500051056105710571F1CF019E012F5F3F4FD8
:10A960000E941F5B882309F45EC129813A814B81D3
:10A970005C81D4011496ED91FC9115978289803108
:10A9800049F4283FBFEF3B07B0E04B07B0E05B075F
:10A9900048F019C0283FEFEF3E07EFEF4E07EFE01A
:10A9A0005E0788F4D40116962D933D934D935C93E6
:10A9B000199714C0F40186899789A08DB18D0097ED
:10A9C000A105B10531F4C4010E941754882331F464
:10A9D0002AC1F40186839783A087B187D401169694
:10A9E0004D915D916D917C91199714968D919C91EB
:10A9F00015970E94CC585B016C01AF0CB11CC11CB7
:10AA0000D11C01151105C9F4ED81FE81E050F24021
:10AA1000D8F5D4011A962D913D914D915C911D97D9
:10AA200052968D919D910D90BC91A02D28173907BC
:10AA30004A075B0710F045E001C041E0C601B501DF
:10AA40000E943459009709F4EEC040E052E0401BE8
:10AA5000510B4D805E804415550508F42A019C0178
:10AA6000200F311FC9016F817885A2010E94790AE8
:10AA7000040D151D0050124009F07DC00E9431598F
:10AA8000882309F078C0CFC0ED81FE81E050F4400A
:10AA900000F58091940C9091950CA091960CB0913A
:10AAA000970C8A159B05AC05BD0511F40E94BD5895
:10AAB0008091990C90919A0CB601A5012F8138854F
:10AAC0000E94E45E882309F4AEC0412CF2E05F2EC0
:10AAD00052C0D4011496ED91FC91159784818F1981
:10AAE0003E803694831508F4382E032D10E020E0C4
:10AAF00030E08091990C90919A0CB601A5010E94CA
:10AB00009C5E882309F48FC06F807884860175016C
:10AB100022C08091940C9091950CA091960CB091CC
:10AB2000970CE816F9060A071B0711F40E94BD5896
:10AB30008091990C90919A0CB3010E94105EE0E014
:10AB4000F2E06E0E7F1E0894E11CF11C011D111D28
:10AB5000882309F468C08E2D8A198315D0F280915C
:10AB6000990C90919A0C0E94EA5D882309F45BC0CD
:10AB7000532C550C4424920140E050E0F4018285AE
:10AB80009385A485B585820F931FA41FB51F828767
:10AB90009387A487B5872F813885240D351D388785
:10ABA0002F838D819E81841995099E838D83D40185
:10ABB0001A962D913D914D915C911D97ED81FE81ED
:10ABC000EF2B09F0A3CE52968D919D910D90BC91E3
:10ABD000A02D82179307A407B50740F4D40152961D
:10ABE0002D933D934D935C9355970BC080918D0AA7
:10ABF00090918E0A892B59F0E985FA85EF2B39F06F
:10AC0000D40111968C911197806811968C93F40160
:10AC1000818183FF05C0C4010E944950882319F037
:10AC200049855A8505C081E0D4018C934FEF5FEFD1
:10AC3000CA012A960FB6F894DEBF0FBECDBFCF91E2
:10AC4000DF911F910F91FF90EF90DF90CF90BF9019
:10AC5000AF909F908F907F906F905F904F903F90BC
:10AC6000089582FD35CE48CE9F92AF92BF92CF928B
:10AC7000DF92EF92FF920F931F93CF93DF938C019C
:10AC8000FC0182899389A489B589805E9F4FAF4179
:10AC9000B04008F05CC0C8010E941754882309F432
:10ACA00056C0D80116964D915D916D917C91199782
:10ACB00014968D919C9115970E94CC585B016C0164
:10ACC00045E00E943459EC01009709F442C080E04D
:10ACD00092E0FE019C01119221503040E1F79C2E40
:10ACE000ED2EFF24F39411C0B601A5014F0D511DA7
:10ACF000611D711D8091990C90919A0C292D3E2D0A
:10AD00000E94E45E882319F1F394D8011496ED9122
:10AD1000FC9115972481F21638F330E040E050E0C2
:10AD200089E0220F331F441F551F8A95D1F7529691
:10AD30008D919D910D90BC91A02D820F931FA41F0A
:10AD4000B51FF801828B938BA48BB58B02C0C0E03A
:10AD5000D0E0CE01DF91CF911F910F91FF90EF9046
:10AD6000DF90CF90BF90AF909F9008953F924F9209
:10AD70005F926F927F928F929F92AF92BF92CF928B
:10AD8000DF92EF92FF920F931F93CF93DF934C01CB
:10AD9000EB01442E352E522E8C819D81F40195833A
:10ADA0008483CB0140E050E060E070E00E94824F7D
:10ADB00077244FC0CE010E94945397FDABC08A8583
:10ADC0009B85AC85BD8581509E4FAF4FBF4F8A8715
:10ADD0009B87AC87BD87A090940CB090950CC090D9
:10ADE000960CD090970C24E9E22E2AE0F22E00E097
:10ADF00010E0602EF7018081882311F0853E79F400
:10AE0000772041F4F401A686B786C08AD18A63828E
:10AE100077247394F7018081882391F428C0B801C6
:10AE200095E0660F771F9A95E1F76C56754F842D64
:10AE3000932D4BE050E00E946C0A009709F47DC00E
:10AE40000F5F1F4F80E290E0E80EF91E0031110500
:10AE500081F62A853B854C855D858A899B89AC89ED
:10AE6000BD89281739074A075B0708F4A3CF56FEA8
:10AE700051C051FE4FC0772051F0F4016380C401EE
:10AE800061E00E942B50EC01009761F443C08A817D
:10AE9000823009F43FC0CE010E9434560097D1F1B0
:10AEA000EC01662480E2FE0111928A95E9F7DE0149
:10AEB000242D332DC901FC018BE001900D928150AE
:10AEC000E1F7E0918D0AF0918E0A309739F0BE01DA
:10AED000625F7F4FCE014096099508C081E298E2FB
:10AEE000998B888B80E098E09F878E8788899989E5
:10AEF0009B8B8A8B998F888F8E859F859F8B8E8B5E
:10AF00000E94EC58882331F0C401662D452D0E9423
:10AF1000665101C080E0DF91CF911F910F91FF90AA
:10AF2000EF90DF90CF90BF90AF909F908F907F90E9
:10AF30006F905F904F903F90089557FEE5CFEACF16
:10AF40002F923F924F925F926F927F928F929F9239
:10AF5000AF92BF92CF92DF92EF92FF920F931F9327
:10AF6000DF93CF93CDB7DEB7C454D0400FB6F8947B
:10AF7000DEBF0FBECDBF3C016B01DE01A05CBF4F49
:10AF800011965C934E9323962FAF2397611571050D
:10AF900009F483C01E8618A6FC018281882309F06B
:10AFA0007CC01C861EA2FA0180818F32F1F08601DE
:10AFB0005CE0E52EF12CEC0EFD1E40E4A42EB12C3D
:10AFC000AC0EBD1E4E010894811C911C2596FFAE4F
:10AFD000EEAE259736E2232E312C2C0E3D1E270196
:10AFE00024C01196B183A08301C0FD01A081B1816D
:10AFF0008C918F32B1F3D60112968C9112978250B8
:10B000008230A8F28E010A5D1F4F14966D917C91DB
:10B010001597C8010E943A4F882351F63EC0342D3F
:10B02000252D8701832F922F7C01F501808191814D
:10B03000B401A5010E94854E882329F42EC03196C3
:10B04000D501ED93FC93D501ED91FC9180818F3278
:10B05000B1F38823C9F0C701B801A40121E00E941F
:10B06000B6568823D1F00C151D0519F0C8010E94B1
:10B07000EA512596EEADFFAD2597EE16FF0679F65F
:10B08000C101322D292FCDCFC301B801A4012396D0
:10B090002FAD23970E94B65601C080E0CC5BDF4FF6
:10B0A0000FB6F894DEBF0FBECDBFCF91DF911F91D9
:10B0B0000F91FF90EF90DF90CF90BF90AF909F9057
:10B0C0008F907F906F905F904F903F902F9008955A
:10B0D0000F931F93DF93CF93CDB7DEB76A970FB669
:10B0E000F894DEBF0FBECDBF9C01AB0119821B825D
:10B0F0008E010F5F1F4FC801B90122E00E94A057C7
:10B10000882319F0C8010E94F4516A960FB6F8948A
:10B11000DEBF0FBECDBFCF91DF911F910F9108957C
:10B12000FB01242F60918B0A70918C0AAF010E9461
:10B13000A0570895FC01128210820E949058089531
:10B14000DF93CF93CDB7DEB76A970FB6F894DEBF23
:10B150000FBECDBF9C01AB0119821B82CE010196AF
:10B16000B90121E00E94A0576A960FB6F894DEBF9D
:10B170000FBECDBFCF91DF9108958FEF9FEFAFEF5F
:10B18000BFEF8093940C9093950CA093960CB09382
:10B19000970C1092980C08950F931F938C01CB017C
:10B1A000BA016250704080409040F801248130E044
:10B1B00040E050E00E94636A9B01AC01F801828587
:10B1C0009385A485B585280F391F4A1F5B1FB901D8
:10B1D000CA011F910F9108958091980C80FF3DC086
:10B1E0004091940C5091950C6091960C7091970C35
:10B1F0008091990C90919A0C24E93AE00E94E45EC7
:10B20000882369F18091980C81FF22C080918F0A78
:10B210008230F0F04091900A5091910A6091920A28
:10B220007091930A8091940C9091950CA091960C3A
:10B23000B091970C480F591F6A1F7B1F8091990C82
:10B2400090919A0C24E93AE00E94E45E882339F058
:10B250008091980C8E7F8093980C81E0089580E017
:10B2600008950E94EC580895DF92EF92FF920F9399
:10B270001F937B018C01D42E8091940C9091950C9E
:10B28000A091960CB091970C8E159F05A007B10761
:10B29000E1F00E94EC58882311F1D2FC0CC080919F
:10B2A000990C90919A0CB801A70124E93AE00E9408
:10B2B0005B5F8823A1F01092980CE092940CF092BE
:10B2C000950C0093960C1093970C83E0D8228091F4
:10B2D000980C8D298093980C24E93AE002C020E074
:10B2E00030E0C9011F910F91FF90EF90DF9008951A
:10B2F0006F927F928F929F92AF92BF92CF92DF9286
:10B30000EF92FF920F931F93CF93DF93EC01142FD3
:10B3100070939A0C6093990C1A8A82E090E0A0E0F6
:10B32000B0E088839983AA83BB831092980C8FEF37
:10B330009FEFAFEFBFEF8093940C9093950CA09389
:10B34000960CB093970C442321F466247724430190
:10B3500036C0453008F0EFC060E070E080E090E07B
:10B3600040E00E943459DC01009709F4E4C0412F09
:10B3700050E041505040FA0174E0EE0FFF1F7A9503
:10B38000E1F7E80FF91FE254FE4F808190E08F77DC
:10B390009070892B09F0CFC064E0440F551F6A9567
:10B3A000E1F7A40FB51FAA53BE4F6D907D908D900D
:10B3B0009C90611471048104910409F4BCC0C4011F
:10B3C000B30140E00E9434595C01009709F4B3C016
:10B3D000FC01838594858050924009F0ACC0F50152
:10B3E0002089222309F4A7C04685578541155105B8
:10B3F00009F4A1C020938F0A85858C83198691E07A
:10B4000060E070E00AC0990F6F5F7F4F6830710590
:10B4100009F491C089858F5F89878C81891799F795
:10B42000F501668977896115710519F080E090E072
:10B4300005C0F50164A175A186A197A16093900A4A
:10B440007093910A8093920A9093930A6A01EE2472
:10B45000FF24C60CD71CE81CF91CCE86DF86E88AC0
:10B46000F98AF501018912891C8B0B8B30E040E0D1
:10B4700050E00E94636A6C0D7D1D8E1D9F1D6D8BBB
:10B480007E8B8F8B988F35E0000F111F3A95E1F777
:10B4900001501E4F012F11270695980140E050E002
:10B4A000260F371F481F591F2A873B874C875D8708
:10B4B000F50183899489009721F07C0100E010E078
:10B4C00005C0F501E0A0F1A002A113A1C401B301E0
:10B4D000621B730B840B950B6E0D7F1D801F911FDC
:10B4E000098404C096958795779567950A94D2F755
:10B4F0006D837E838F839887653FFFE07F07F0E051
:10B500008F07F0E09F0718F48CE08A8B14C0655F0A
:10B510007F4F8040904010F480E10AC0F50184A57F
:10B5200095A5A6A5B7A58D8B9E8BAF8BB88F80E216
:10B530008A8B81E001C080E0DF91CF911F910F9154
:10B54000FF90EF90DF90CF90BF90AF909F908F9043
:10B550007F906F90089542600E94345908958F92B1
:10B560009F92AF92BF92CF92DF92EF92FF920F9392
:10B570001F93CF93DF93EC016A017B0148015901CE
:10B58000423051056105710508F44BC08D819E81E3
:10B59000AF81B8850196A11DB11D84179507A60737
:10B5A000B70708F43EC08A89803129F4252F362F49
:10B5B000472F55270BC08032A1F59A01AB0117E048
:10B5C00056954795379527951A95D1F78E859F857E
:10B5D000A889B989280F391F4A1F5B1FCA01B90101
:10B5E00041E00E94AB5A9C010097D9F08A898031D2
:10B5F00049F4F601F070EE0FFF1FE20FF31F918286
:10B6000080820DC0F601EF77F070EE0FFF1FEE0F96
:10B61000FF1FE20FF31F80829182A282B38281E03A
:10B6200001C080E0DF91CF911F910F91FF90EF90CB
:10B63000DF90CF90BF90AF909F908F900895CF9262
:10B64000DF92EF92FF920F931F93CF93DF93EC0162
:10B650007A018B016901423051056105710508F4D9
:10B6600053C08D819E81AF81B8850196A11DB11D0A
:10B6700084179507A607B70708F446C08A89803162
:10B6800029F45527412F302F2F2D0BC08032E1F5A3
:10B690009A01AB0167E056954795379527956A95CE
:10B6A000D1F78E859F85A889B989280F391F4A1F30
:10B6B0005B1FCA01B90140E00E94AB5A9C01009790
:10B6C00019F18A89803159F4F701F070EE0FFF1FEC
:10B6D000E20FF31F80819181A0E0B0E00EC0F7017E
:10B6E000EF77F070EE0FFF1FEE0FFF1FE20FF31F5B
:10B6F00080819181A281B381BF70F60180839183A3
:10B70000A283B38381E001C080E0DF91CF911F91DC
:10B710000F91FF90EF90DF90CF9008958F929F92BE
:10B72000AF92BF92CF92DF92EF92FF920F931F934F
:10B73000DF93CF9300D000D0CDB7DEB75C016A01B4
:10B740007B014E010894811C911CC501B701A60123
:10B7500094010E941F5B8823B1F1C501B701A601C6
:10B7600000E010E020E030E00E94AF5A882359F159
:10B77000F50180819181A281B381C816D906EA06BC
:10B78000FB0620F4C082D182E282F382C980DA8093
:10B79000EB80FC80F5018289803151F4F8EFCF16FF
:10B7A000FFEFDF06F0E0EF06F0E0FF0670F209C001
:10B7B00088EFC8168FEFD8068FEFE8068FE0F806FF
:10B7C00020F281E001C080E00F900F900F900F9069
:10B7D000CF91DF911F910F91FF90EF90DF90CF906D
:10B7E000BF90AF909F908F9008952F923F924F926D
:10B7F0005F926F927F928F929F92AF92BF92CF9201
:10B80000DF92EF92FF920F931F93DF93CF93CDB709
:10B81000DEB766970FB6F894DEBF0FBECDBF1C0132
:10B8200049875A876B877C873E872D87DC01159671
:10B830002D913D914D915C9118972F5F3F4F4F4F48
:10B840005F4F2D833E834F835887ED85FE850081B2
:10B85000118122813381011511052105310549F03E
:10B86000480159010894811C911CA11CB11C10E0D5
:10B8700006C0DC018D909D90AD90BC9011E07501EB
:10B880006401442455243201F10185819681A78108
:10B89000B085481659066A067B0608F09DC02D81C2
:10B8A0003E814F8158852C153D054E055F0550F4AE
:10B8B000F2E08F2E912CA12CB12CE2E0CE2ED12CD7
:10B8C000E12CF12CC101B701A6019E012F5F3F4F72
:10B8D0000E941F5B882309F47FC089819A81AB8114
:10B8E000BC810097A105B10571F08C149D04AE04D4
:10B8F000BF0409F010E0460157010894811C911C17
:10B90000A11CB11C16C0D701C6010196A11DB11D15
:10B910008B8B9C8BAD8BBE8B88199909AA09BB09AF
:10B9200029853A854B855C8582179307A407B5075F
:10B9300059F00894411C511C611C711C0894C11CD5
:10B94000D11CE11CF11CA0CF112349F08B899C89EB
:10B95000AD89BE89F10180839183A283B383C10144
:10B96000B701A6010FEF1FEF2FEF3FE00E94AF5A84
:10B97000882399F431C02601370108944108510801
:10B9800061087108C101B301A201970186010E94FB
:10B99000AF5A882309F1730162018C149D04AE042F
:10B9A000BF0448F3AD85BE854D915D916D917C914D
:10B9B000411551056105710539F0C10195018401F9
:10B9C0000E94AF5A882341F0ED85FE8580829182E6
:10B9D000A282B38281E001C080E066960FB6F8943F
:10B9E000DEBF0FBECDBFCF91DF911F910F91FF90B2
:10B9F000EF90DF90CF90BF90AF909F908F907F900F
:10BA00006F905F904F903F902F900895FF920F930B
:10BA10001F93CF93DF938B010E943564EB01FF24CA
:10BA2000FA9409C00E9435646C1B7D0B6017710786
:10BA300010F080E008C0FEBC0DB407FEFDCF8EB54F
:10BA40008F3F81F781E0DF91CF911F910F91FF90A0
:10BA50000895FC01808161E00E9437658FEF8EBD03
:10BA60000DB407FEFDCF0895CF93DF93EC01DA010B
:10BA70006EBD0DB407FEFDCF8C918EBD1196EC917D
:10BA8000119782E090E00DB407FEFDCFEEBD22E0FD
:10BA90008030920731F0FD01E80FF91FE081019637
:10BAA000F2CF0DB407FEFDCF8FEF8EBD0DB407FEB4
:10BAB000FDCF8FEF8EBD0DB407FEFDCF8FEF8EBD96
:10BAC0000DB407FEFDCF8EB58B838F71853011F4D9
:10BAD00081E006C083E18983CE010E94295D80E078
:10BAE000DF91CF910895BF92CF92DF92EF92FF92B4
:10BAF0000F931F93CF93DF93EC016B017A010E94A8
:10BB000035648B01BB24BA9409C00E943564601B64
:10BB1000710B6D52714010F081E10BC0BEBC0DB4D1
:10BB200007FEFDCF8EB58B838F3F79F38E3F39F0C3
:10BB30008FE08983CE010E94295D80E030C0D7016B
:10BB40001197EF28D9F08FEF8EBD20E030E09FEF06
:10BB50000BC00DB407FEFDCF8EB59EBDF601E20F02
:10BB6000F31F80832F5F3F4F2A173B0790F30DB4DD
:10BB700007FEFDCF8EB5AC0DBD1D8C931B828FEFE4
:10BB80008EBD0DB407FEFDCF8EB58FEF8EBD0DB40B
:10BB900007FEFDCF8EB5CE010E94295D81E0DF91C9
:10BBA000CF911F910F91FF90EF90DF90CF90BF90BA
:10BBB00008950F931F938C018BE99CE0F80162813B
:10BBC0000E940B4EF801808160E00E9437651F9152
:10BBD0000F910895CF93DF93EC010E94D95DCE01C0
:10BBE00068E572E00E94065D882389F08DEF8EBDC6
:10BBF0000DB407FEFDCFCE0168E572E00E94065D40
:10BC0000882329F0CE010E94295D81E006C082E1EF
:10BC10008983CE010E94295D80E0DF91CF91089554
:10BC20000F931F93CF93DF93EC018B010E94D95D9B
:10BC3000CE0168E572E00E94065D882361F0CE01C6
:10BC40006CEFA8010E94345D882329F0CE010E9488
:10BC5000295D81E006C085E18983CE010E94295DCE
:10BC600080E0DF91CF911F910F910895EF92FF92A5
:10BC70000F931F938C017B010E94D95DC801B7010E
:10BC800040E052E00E94735D1F910F91FF90EF9092
:10BC90000895FF920F931F93DF93CF9300D000D0AE
:10BCA000CDB7DEB78C01F62E29833A834B835C83B4
:10BCB0000E94D95DC80168E572E00E94065D8F2D83
:10BCC00080648EBD0DB407FEFDCFFE0131969E014E
:10BCD0002350304083818EBD0DB407FEFDCF3197D8
:10BCE000E217F307B9F7FF2011F087E801C085E9F3
:10BCF0008EBD0DB407FEFDCF8CE0F81631F48FEF4A
:10BD00008EBD0DB407FEFDCF8EB590E02FEF2EBD9A
:10BD10000DB407FEFDCF8EB587FF02C09150B9F775
:10BD2000F80183830F900F900F900F90CF91DF91C8
:10BD30001F910F91FF900895AF92BF92CF92DF9223
:10BD4000EF92FF920F931F93CF93DF93EC015A0171
:10BD50006B017801890167E320E030E040E050E0CA
:10BD60000E94495ECE0167E1A80197010E94495EE9
:10BD7000882311F089E013C08C81833039F089E089
:10BD8000AA0CBB1CCC1CDD1C8A95D1F7CE0169E145
:10BD9000A60195010E94495E882339F087E08983D6
:10BDA000CE010E94295D80E004C0CE010E94295D81
:10BDB00081E0DF91CF911F910F91FF90EF90DF9085
:10BDC000CF90BF90AF900895CF92DF92EF92FF9205
:10BDD0000F931F93CF93DF93EC017A018B016901DD
:10BDE0008C81833039F099E0EE0CFF1C001F111F8D
:10BDF0009A95D1F7CE0168E1A80197010E94495EAA
:10BE0000882319F086E089830CC0CE016EEFA6016D
:10BE10000E94345D882329F0CE010E94295D81E0D3
:10BE200004C0CE010E94295D80E0DF91CF911F9177
:10BE30000F91FF90EF90DF90CF900895CF93DF9315
:10BE4000EC016CE020E030E040E050E00E94495E10
:10BE5000882339F083E08983CE010E94295D80E048
:10BE600004C0CE010E94295D81E0DF91CF91089549
:10BE7000CF93DF93EC019A01AB018C81833039F0D1
:10BE800069E0220F331F441F551F6A95D1F7CE0179
:10BE900062E10E94495E882339F085E08983CE0102
:10BEA0000E94295D80E004C0CE010E94295D81E0EE
:10BEB000DF91CF910895CF92DF92EF92FF920F938F
:10BEC0001F93CF93DF93EC017A018B0169018C8181
:10BED000833039F0B9E0EE0CFF1C001F111FBA953A
:10BEE000D1F7CE0161E1A80197010E94495E882344
:10BEF00039F084E08983CE010E94295D80E006C08C
:10BF0000CE01B60140E052E00E94735DDF91CF9117
:10BF10001F910F91FF90EF90DF90CF900895BF9207
:10BF2000CF92DF92EF92FF920F931F93CF93DF9305
:10BF3000EC01B42E1C82198268830E9435646B0167
:10BF4000888161E00E94F864888161E00E94376521
:10BF50008BE99CE00E94254E80E48A838BE99CE07B
:10BF600060E40E940B4E80E09FEF9EBD0DB407FE83
:10BF7000FDCF8F5F8A30C9F709C00E9435646C1904
:10BF80007D09615D774010F081E063C0CE0160E023
:10BF900020E030E040E050E00E94495E813069F7E7
:10BFA0001FEFCE0168E02AEA31E040E050E00E9455
:10BFB000495E853011F481E00DC080E01EBD0DB4F6
:10BFC00007FEFDCF9EB58F5F8430C1F79B839A3A01
:10BFD00031F482E08C838C81823051F40DC00E9458
:10BFE00035646C197D09615D7740D8F282E031C01B
:10BFF000EE24FF2487010FC0E12CF12C012D80E4F9
:10C00000182F09C00E9435646C197D09615D774065
:10C0100010F08AE01EC0CE0167E320E030E040E08F
:10C0200050E00E94495ECE0169E2A80197010E949A
:10C03000495E882339F78C81823031F5CE016AE37D
:10C0400020E030E040E050E00E94495E882339F073
:10C0500088E08983CE010E94295D80E01AC08FEFBD
:10C060008EBD0DB407FEFDCF8EB5807C803C11F4F3
:10C0700083E08C8380E09FEF9EBD0DB407FEFDCF73
:10C080002EB58F5F8330C1F7CE010E94295DBA8241
:10C0900081E0DF91CF911F910F91FF90EF90DF90A2
:10C0A000CF90BF900895DB010D900020E9F7119724
:10C0B000A61BB70B0496AD010E943E540895DF9372
:10C0C000CF930F92CDB7DEB769830496BE016F5F41
:10C0D0007F4F41E050E00E943E5420E030E0019765
:10C0E00011F421E030E0C9010F90CF91DF91089564
:10C0F0000F931F938C0104960E949A58F8011382A3
:10C1000012828DEA93E0918380831F910F910895AD
:10C110008091C10085FDFCCF8091C00085FFF8CFE4
:10C120006093C60081E090E0089510929F0C1092F9
:10C130009E0C85EB93E090939D0C80939C0C08954E
:10C1400081E08093E50C6093C20C1092E30C109296
:10C15000E40C08952091C10C30E08091C00C281BA4
:10C160003109C90108954091C00C8091C10C481754
:10C1700018F02FEF3FEF0AC0E42FF0E0E056F34F46
:10C180008081282F30E04F5F4093C00CC901089593
:10C19000E091C00C8091C10CE81718F0EFEFFFEFB1
:10C1A00006C0F0E0E056F34F8081E82FF0E0CF01C9
:10C1B000089508951092E90C1092E80C88EE93E02F
:10C1C000A0E0B0E08093EA0C9093EB0CA093EC0C11
:10C1D000B093ED0C8DEB93E09093E70C8093E60C1D
:10C1E0000895CF92DF92EF92FF920F931F93CF9318
:10C1F000DF937C016B018A018091E50C8823A1F01B
:10C20000C0E0D0E00DC0D701ED91FC91D601AC0F9C
:10C21000BD1F0190F081E02DC7016C910995219619
:10C22000C017D10780F304C0CB01642F0E942362A2
:10C23000C801DF91CF911F910F91FF90EF90DF9098
:10C24000CF900895DF93CF930F92CDB7DEB7FC0167
:10C2500069838091E50C8823C9F08091E40C8032D9
:10C2600038F081E090E09383828320E030E015C0D5
:10C270008091E30CE82FF0E0ED53F34F9981908328
:10C280008F5F8093E30C8093E40C05C0CE01019690
:10C2900061E00E94236221E030E0C9010F90CF915C
:10C2A000DF9108950F93062F8091C20C63EC7CE020
:10C2B0004091E40C21E00E94CE611092E30C1092B8
:10C2C000E40C1092E50C0F91089561E00E94526118
:10C2D0000895413208F040E2862F60EA7CE00E9437
:10C2E00085611092C00C8093C10C089521E00E94DA
:10C2F000696108951092C00C1092C10C1092E30C69
:10C300001092E40C0E94CF630895382F413210F050
:10C3100040E042C08091F20C8823E1F791E09093D5
:10C32000F20C2093F40C8FEF80935F0D10921A0D96
:10C33000415040931B0D4F5F9093F30C8091F30C91
:10C34000330F832B8093F30C8091F50C813041F4F3
:10C350001092F50C8091F30C8093BB0085EC01C02A
:10C3600085EE8093BC008091F20C8130E1F38091E6
:10C370001A0D841710F440911A0D20E030E00AC025
:10C38000FB01E20FF31FD901A650B34F8C918083BC
:10C390002F5F3F4F2417A0F3842F08950F931F930F
:10C3A000582F122F413210F081E04AC08091F20CD8
:10C3B0008823E1F782E08093F20C0093F40C8FEF76
:10C3C00080935F0D10921A0D40931B0DAAEFBCE0F5
:10C3D000FB0102C081918D938E2F861B8417D0F3B1
:10C3E0001092F30C8091F30C550F852B8093F30C76
:10C3F0008091F50C813041F41092F50C8091F30C92
:10C400008093BB0085EC01C085EE8093BC001123B6
:10C4100021F08091F20C8230E1F380915F0D8F3F2B
:10C4200011F480E00DC080915F0D803211F482E044
:10C4300007C080915F0D803311F084E001C083E07C
:10C440001F910F910895482F613210F081E00895F7
:10C450008091F20C843011F082E0089560933D0DDC
:10C46000ACE1BDE0842F9C01F90102C081918D9364
:10C470008E2F841B8617D0F380E008951F920F92B1
:10C480000FB60F9211242F933F934F935F936F93A7
:10C490007F938F939F93AF93BF93EF93FF9380917D
:10C4A000B90090E0887F90708036910509F4F2C061
:10C4B00081369105CCF58832910509F47BC089322B
:10C4C0009105B4F48031910509F46FC08131910573
:10C4D0003CF4009709F447C1089709F04FC165C0C3
:10C4E0008831910509F466C0809709F047C182C080
:10C4F0008034910509F4A4C08134910544F480335B
:10C50000910509F482C0C89709F038C189C0803507
:10C51000910509F489C08835910509F496C08834DD
:10C52000910509F02BC1AEC08839910509F413C1FA
:10C5300089399105ECF48837910509F4ABC0893746
:10C5400091054CF48836910509F4A4C08037910513
:10C5500009F014C19FC08838910509F4FCC08039E6
:10C56000910509F49DC08038910509F007C198C074
:10C57000803B910509F4C6C0813B91054CF4803A9B
:10C58000910509F49FC0883A910509F0F7C0BAC037
:10C59000803C910509F4E3C0883C910509F4DFC0B3
:10C5A000883B910509F0EAC0C2C08091F30C8093EA
:10C5B000BB00CFC090911A0D80911B0D981768F4A5
:10C5C00090911A0DE92FF0E0E650F34F80818093AF
:10C5D000BB009F5F90931A0DBCC08091F40C882320
:10C5E00009F44BC085ED8093BC008091BC0084FDB4
:10C5F000FCCFC2C080E280935F0D85ED8093BC00CC
:10C600008091BC0084FDFCCFB7C080E380935F0DB8
:10C6100085ED8093BC008091BC0084FDFCCFACC054
:10C6200088E380935F0D9BC080911A0D9091BB00B1
:10C63000E82FF0E0E650F34F90838F5F80931A0D60
:10C6400090911A0D80911B0D82C080911A0D9091CE
:10C65000BB00E82FF0E0E650F34F90838F5F8093AC
:10C660001A0D8091F40C882341F085ED8093BC0075
:10C670008091BC0084FDFCCF7FC081E08093F50CED
:10C6800084EA6EC085ED8093BC008091BC0084FD7F
:10C69000FCCF72C083E08093F20C10925E0D59C003
:10C6A00080915E0D803208F056C080915E0D9091B1
:10C6B000BB00E82FF0E0E25CF24F90838F5F809345
:10C6C0005E0D47C080915E0D803230F4E0915E0DCA
:10C6D000F0E0E25CF24F108285ED8093BC00809127
:10C6E000BC0084FDFCCF1092F20C60915E0DE091D5
:10C6F000F80CF091F90C8EE39DE070E00995109232
:10C700005E0D2DC084E08093F20C10923C0D1092CF
:10C710003D0DE091F60CF091F70C099580913D0DDF
:10C72000882329F481E080933D0D10921C0D909197
:10C730003C0DE92FF0E0E45EF24F80818093BB0076
:10C740009F5F90933C0D90913C0D80913D0D98170B
:10C7500010F485EC01C085E88093BC000FC085EC27
:10C760008093BC0009C010925F0D85ED8093BC00E2
:10C770008091BC0084FDFCCF1092F20CFF91EF91F0
:10C78000BF91AF919F918F917F916F915F914F91E9
:10C790003F912F910F900FBE0F901F901895109200
:10C7A000F20C81E08093F40C1092F50C81E161E0D1
:10C7B0000E94376580E161E00E943765E9EBF0E0B7
:10C7C00080818E7F808380818D7F808384E38093CE
:10C7D000B80085E48093BC0008951F920F920FB6B5
:10C7E0000F9211242F933F938F939F93AF93BF93F7
:10C7F0008091640D9091650DA091660DB091670DCB
:10C800003091680D0196A11DB11D232F235D2D3799
:10C8100020F02D570196A11DB11D2093680D809326
:10C82000640D9093650DA093660DB093670D809194
:10C83000600D9091610DA091620DB091630D019614
:10C84000A11DB11D8093600D9093610DA093620DA9
:10C85000B093630DBF91AF919F918F913F912F91B5
:10C860000F900FBE0F901F9018958FB7F8942091DE
:10C87000640D3091650D4091660D5091670D8FBF2D
:10C88000B901CA010895EF92FF920F931F937B01A4
:10C890008C019FB7F8942091600D3091610D40910B
:10C8A000620D5091630D86B5A89B06C08F3F21F0A5
:10C8B0002F5F3F4F4F4F5F4F9FBF542F432F322F5C
:10C8C0002227280F311D411D511DDA01C90162E0E7
:10C8D000880F991FAA1FBB1F6A95D1F7820F931F5C
:10C8E000A41FB51FBC0135C09FB7F8942091600DFF
:10C8F0003091610D4091620D5091630D86B5A89BFA
:10C9000006C08F3F21F02F5F3F4F4F4F5F4F9FBFBC
:10C91000542F432F322F2227280F311D411D511D27
:10C92000DA01C901E2E0880F991FAA1FBB1FEA952F
:10C93000D1F7820F931FA41FB51F861B970B885E2C
:10C94000934090F20894E108F10801091109685137
:10C950007C4FE114F1040105110531F61F910F918F
:10C96000FF90EF900895019739F0880F991F880F75
:10C97000991F02970197F1F70895789484B5826022
:10C9800084BD84B5816084BD85B5826085BD85B573
:10C99000816085BDEEE6F0E0808181608083E1E822
:10C9A000F0E010828081826080838081816080835A
:10C9B000E0E8F0E0808181608083E1EBF0E080815D
:10C9C00084608083E0EBF0E0808181608083EAE72F
:10C9D000F0E08081846080838081826080838081B8
:10C9E000816080838081806880831092C100089577
:10C9F000CF93DF93482F50E0CA018251904FFC0142
:10CA000034914253504FFA018491882369F190E0A8
:10CA1000880F991FFC01E055F04FA591B491FC01DE
:10CA2000E654F04FC591D491662351F42FB7F89492
:10CA30008C91932F909589238C93888189230BC0A7
:10CA4000623061F42FB7F8948C91932F90958923DD
:10CA50008C938881832B88832FBF06C09FB7F8945F
:10CA60008C91832B8C939FBFDF91CF910895482F9A
:10CA700050E0CA01825F9F4EFC012491CA0182519D
:10CA8000904FFC0194914253504FFA01349133235B
:10CA900009F440C0222351F1233071F0243028F4EE
:10CAA0002130A1F0223011F514C02630B1F027302A
:10CAB000C1F02430D9F404C0809180008F7703C086
:10CAC000809180008F7D8093800010C084B58F7727
:10CAD00002C084B58F7D84BD09C08091B0008F777E
:10CAE00003C08091B0008F7D8093B000E32FF0E011
:10CAF000EE0FFF1FE654F04FA591B4912FB7F894B5
:10CB0000662321F48C919095892302C08C91892B06
:10CB10008C932FBF0895682F70E0CB01825F9F4EEA
:10CB2000FC012491CB018251904FFC01449162534E
:10CB3000704FFB019491992319F420E030E03CC040
:10CB4000222351F1233071F0243028F42130A1F058
:10CB5000223011F514C02630B1F02730C1F0243056
:10CB6000D9F404C0809180008F7703C08091800049
:10CB70008F7D8093800010C084B58F7702C084B50C
:10CB80008F7D84BD09C08091B0008F7703C08091F4
:10CB9000B0008F7D8093B000892F90E0880F991F9F
:10CBA0008C53904FFC01A591B4918C9120E030E022
:10CBB000842311F021E030E0C9010895982F8E30D0
:10CBC00008F09E509770809150038295880F880FCF
:10CBD000807C892B80937C0080917A008064809394
:10CBE0007A0080917A0086FDFCCF209178004091F8
:10CBF0007900942F80E030E0282B392BC90108956B
:10CC00001F93CF93DF93182FEB0161E00E94F8642C
:10CC1000209709F44AC0CF3FD10509F449C0E12F5C
:10CC2000F0E0E25FFF4E84918330C1F0843028F45D
:10CC3000813051F08230B1F50CC0863019F1873067
:10CC400049F1843079F514C084B5806884BDC7BDCE
:10CC500033C084B5806284BDC8BD2EC08091800081
:10CC6000806880938000D0938900C093880024C09E
:10CC700080918000806280938000D0938B00C0936D
:10CC80008A001AC08091B00080688093B000C09381
:10CC9000B30012C08091B00080628093B000C09356
:10CCA000B4000AC0C038D1051CF4812F60E002C076
:10CCB000812F61E00E943765DF91CF911F91089528
:10CCC000CF92DF92EF92FF920F931F93CF93DF9358
:10CCD0007C016B018A01C0E0D0E00FC0D6016D91EC
:10CCE0006D01D701ED91FC910190F081E02DC7011C
:10CCF0000995C80FD91F015010400115110571F792
:10CD0000CE01DF91CF911F910F91FF90EF90DF90B7
:10CD1000CF900895DC01ED91FC910190F081E02D20
:10CD200009950895CF93DF93DB010D900020E9F77B
:10CD30001197A61BB70BEC01E881F9810280F38102
:10CD4000E02DAD010995DF91CF9108954F925F924B
:10CD50007F928F929F92AF92BF92CF92DF92EF928B
:10CD6000FF920F931F93DF93CF93CDB7DEB7A197B9
:10CD70000FB6F894DEBF0FBECDBF2C01742ECB01D1
:10CD8000223008F42AE019A231E2C32ED12CCC0EB5
:10CD9000DD1E822E9924AA24BB24672D752FA501A0
:10CDA00094010E94B56A79018A01C801B701A50101
:10CDB00094010E94636A472D461B0894C108D1085C
:10CDC0004A3014F4405D01C0495CF6014083E1142F
:10CDD000F1040105110521F07E2C5F2DC801DDCF86
:10CDE000C201B6010E949266A1960FB6F894DEBF0A
:10CDF0000FBECDBFCF91DF911F910F91FF90EF90AC
:10CE0000DF90CF90BF90AF909F908F907F905F907A
:10CE10004F900895CF92DF92EF92FF920F931F935E
:10CE2000CF93DF93EC016A017B012115310541F4B9
:10CE3000E881F9810190F081E02D642F09951FC0F0
:10CE40002A303105D1F477FF17C0E881F9810190CC
:10CE5000F081E02D6DE209958C0144275527BA0138
:10CE60004C195D096E097F09CE012AE00E94A66671
:10CE70009801280F391F04C02AE00E94A6669C0171
:10CE8000C901DF91CF911F910F91FF90EF90DF903B
:10CE9000CF900895EF92FF920F931F937B019A0119
:10CEA0000027F7FC0095102FB801A7010E940A6720
:10CEB0001F910F91FF90EF9008950F931F93CF93C1
:10CEC000DF93FC018B0141155105F9F061157105E6
:10CED000E1F0848195812817390718F0FB01108251
:10CEE00014C041505040EC01C21BD30B4C175D07DE
:10CEF00008F4EA0160817181620F731FC801AE01FD
:10CF00000E94B40AC00FD11F1882DF91CF911F91E8
:10CF10000F9108950F931F93CF93DF93EC018B0133
:10CF20006F5F7F4F888199810E944909009711F4B2
:10CF300080E005C0998388831B830A8381E0DF91A9
:10CF4000CF911F910F910895CF93DF93EC018881CA
:10CF50009981892B29F08A819B818617970760F434
:10CF6000CE010E948A67882341F08C819D81892BA4
:10CF700019F4E881F981108281E0DF91CF91089561
:10CF8000EF92FF920F931F93CF93DF93EC017B01FE
:10CF90006C817D81E114F104C1F04115510599F0D6
:10CFA0008A01060F171FB8010E94A467882369F041
:10CFB000888199812C813D81820F931FB7010E9446
:10CFC0009F0A1D830C8381E001C080E0DF91CF9137
:10CFD0001F910F91FF90EF900895EF92FF920F93A2
:10CFE0001F93DF93CF93CDB7DEB72B970FB6F8948F
:10CFF000DEBF0FBECDBF7C01CB01BA018E010F5F3A
:10D000001F4FA8012AE030E00E94850BF801019033
:10D010000020E9F73197E01BF10BC701B801AF0120
:10D020000E94C0672B960FB6F894DEBF0FBECDBF2F
:10D03000CF91DF911F910F91FF90EF900895EF92A4
:10D04000FF920F931F93DF93CF9300D000D000D0B7
:10D05000CDB7DEB77C01CB018E010F5F1F4FB8014A
:10D060004AE050E00E94AA0BF80101900020E9F785
:10D070003197E01BF10BC701B801AF010E94C067F7
:10D0800026960FB6F894DEBF0FBECDBFCF91DF91CD
:10D090001F910F91FF90EF900895EF92FF920F93E1
:10D0A0001F93DF93CF9300D000D0CDB7DEB77C01C4
:10D0B000862F90E08E010F5F1F4FB8014AE050E0CD
:10D0C0000E94470BF80101900020E9F73197E01B1F
:10D0D000F10BC701B801AF010E94C0670F900F901C
:10D0E0000F900F90CF91DF911F910F91FF90EF90D4
:10D0F00008956115710511F480E00895DB010D902C
:10D100000020E9F71197A61BB70BAD010E94C0677D
:10D110000895CF93DF93EC0188819981009711F0F6
:10D120000E94F108198218821D821C821B821A82B9
:10D13000DF91CF910895EF92FF920F931F93CF93BA
:10D14000DF93EC017B018A01BA010E94A467882366
:10D1500021F4CE010E94896807C01D830C83888159
:10D160009981B7010E949F0ACE01DF91CF911F9153
:10D170000F91FF90EF900895CF93DF93EC01198208
:10D1800018821B821A821D821C821E826115710503
:10D1900051F0DB010D900020E9F71197A61BB70BAA
:10D1A000AD010E949B68DF91CF910895FC018081C1
:10D1B00091810E94F108089508951F920F920FB671
:10D1C0000F9211242F933F934F938F939F93EF933D
:10D1D000FF934091C6002091A90D3091AA0D2F5FB9
:10D1E0003F4F2F7330708091AB0D9091AC0D28178D
:10D1F000390759F0E091A90DF091AA0DE759F24FC6
:10D2000040833093AA0D2093A90DFF91EF919F9138
:10D210008F914F913F912F910F900FBE0F901F90C4
:10D220001895E091FD0DF091FE0DE05CFF4F8191AE
:10D23000919120813181821B930B8F739070892B88
:10D2400011F00E94DC6808951F920F920FB60F92A2
:10D2500011242F933F938F939F93EF93FF932091EC
:10D26000ED0D3091EE0D8091EF0D9091F00D28179E
:10D27000390731F48091C1008F7D8093C10014C0C3
:10D28000E091EF0DF091F00DE355F24F2081809188
:10D29000EF0D9091F00D01968F7390709093F00DBB
:10D2A0008093EF0D2093C600FF91EF919F918F9196
:10D2B0003F912F910F900FBE0F901F901895DC019A
:10D2C0001C96ED91FC911D97E05CFF4F21913191EF
:10D2D00080819181281B390B2F733070C90108950B
:10D2E000DC011C96ED91FC911D97E05CFF4F2081C5
:10D2F0003181E054F040DF01AE5BBF4F8D919C91D6
:10D3000011972817390719F42FEF3FEF07C08D91B8
:10D310009C91E80FF91F8081282F30E0C901089502
:10D32000DC011C96ED91FC911D97E05CFF4F208184
:10D330003181E054F040DF01AE5BBF4F8D919C9195
:10D3400011972817390719F42FEF3FEF10C08D916F
:10D350009C911197E80FF91F20818D919C91119755
:10D3600001968F73907011969C938E9330E0C90153
:10D370000895FC0186859785DC01A05CBF4FFC0108
:10D38000EE5BFF4F2D913C91119780819181281781
:10D390003907C1F70895CF93DF93EC01EE85FF8540
:10D3A000E05CFF4F20813181E054F0402F5F3F4F20
:10D3B0002F733070DF01AE5BBF4F8D919C91119741
:10D3C00028173907D1F3E05CFF4F80819181E05449
:10D3D000F040E80FF91F6083EE85FF85E05CFF4FAA
:10D3E00031832083EE89FF89208181E090E00D8CDC
:10D3F00002C0880F991F0A94E2F7282B208381E04E
:10D4000090E0DF91CF9108951092F40D1092F30DFA
:10D4100088EE93E0A0E0B0E08093F50D9093F60DD8
:10D42000A093F70DB093F80D8DEC93E09093F20D6F
:10D430008093F10D89E69DE09093FE0D8093FD0DA4
:10D440008DEA9DE09093000E8093FF0D85EC90E0B7
:10D450009093020E8093010E84EC90E09093040E62
:10D460008093030E80EC90E09093060E8093050E5F
:10D4700081EC90E09093080E8093070E86EC90E08C
:10D4800090930A0E8093090E84E080930B0E83E044
:10D4900080930C0E87E080930D0E85E080930E0E36
:10D4A00081E080930F0E0895CF93DF930E94BD64B7
:10D4B0000E94EF2CC1E1D9E60E94CB2D2097E1F329
:10D4C0000E941169F9CF629FD001739FF001829F82
:10D4D000E00DF11D649FE00DF11D929FF00D839F03
:10D4E000F00D749FF00D659FF00D9927729FB00DA0
:10D4F000E11DF91F639FB00DE11DF91FBD01CF01B3
:10D5000011240895991B79E004C0991F961708F01B
:10D51000961B881F7A95C9F780950895AA1BBB1B97
:10D5200051E107C0AA1FBB1FA617B70710F0A61B23
:10D53000B70B881F991F5A95A9F780959095BC0144
:10D54000CD01089597FB092E07260AD077FD04D058
:10D55000E5DF06D000201AF4709561957F4F08959D
:10D56000F6F7909581959F4F0895A1E21A2EAA1B78
:10D57000BB1BFD010DC0AA1FBB1FEE1FFF1FA21783
:10D58000B307E407F50720F0A21BB30BE40BF50B80
:10D59000661F771F881F991F1A9469F76095709509
:10D5A000809590959B01AC01BD01CF01089597FB3B
:10D5B000092E05260ED057FD04D0D7DF0AD0001C57
:10D5C00038F450954095309521953F4F4F4F5F4F20
:10D5D0000895F6F790958095709561957F4F8F4FE0
:10D5E0009F4F0895EE0FFF1F0590F491E02D0994D1
:10D5F0002F923F924F925F926F927F928F929F9263
:10D60000AF92BF92CF92DF92EF92FF920F931F9350
:10D61000CF93DF93CDB7DEB7CA1BDB0B0FB6F89401
:10D62000DEBF0FBECDBF09942A88398848885F8441
:10D630006E847D848C849B84AA84B984C884DF80B2
:10D64000EE80FD800C811B81AA81B981CE0FD11D96
:10D650000FB6F894DEBF0FBECDBFED010895F8946C
:02D66000FFCFFA
:10D66200687474703A2F2F72617973686F6262798D
:10D672002E6E65742F736372697074732F6A61768C
:10D68200612F737663322E302E3700737461727499
:10D6920000656E64002E7478740074007077006AFE
:10D6A2007370007069640064006D007900763D5B00
:10D6B200005B002C005D000D0A00646179006C6F54
:10D6C2006300747474006E70770063707700727315
:10D6D2006E0072627400656E006D6D00726400749B
:10D6E2003D5B006F70656E646F6F7200426F7374A2
:10D6F2006F6E2C4D4100687474703A2F2F726179ED
:10D7020073686F6262792E6E65742F7363726970CB
:10D7120074732F6A6176612F737663322E302E37DF
:10D72200002000140E00000069692D31007BD10138
:10D73200F828D401AA23D701431EDA016E24DD01A1
:10D742000525E0011A22E3016F14E6016027E901D1
:10D752006213EF019319F201A21CF501AA18F80154
:10D76200152AFB01200EFE01AB1A01029F1F0402C3
:10D7720020110702680D0A029D0F0D02F926100200
:10D78200C70E1302401C0100010A50004F70656E63
:10D79200537072696E6B6C65722D30300037030105
:10D7A2000306FF638253633501100E0000CF0007AA
:10D7B2000D720C00206C150D760C030101200D7901
:10D7C2000C0301012A0D7D0C01C0FF340D820C01F6
:10D7D200A8FF400D860C0101FF4C0D8A0C0116FFBB
:10D7E200580D8E0C01C0FF640D920C01A8FF710D43
:10D7F200960C0101FF7E0D9A0C0101FF8B0D9E0C10
:10D802000150FF980DA20C0200FFA30DA60C02010D
:10D8120001A40DAA0C030005B40DAD0C030101C552
:10D822000DB10C0300F0D60DB50C030008E50DB9DF
:10D832000C03003CF50DBD0C033C78060EC20C0334
:10D842000001170EC70C030101280ECB0C0364FA6A
:10D85200370ECF0C030AF0450ED20C010001540E14
:10D86200D60C0300FF650EDB0C036EFF700EE10C9D
:10D872000164FF7E0EE50C0105FF8D0EE90C01CC63
:10D88200FF9A0EED0C0109FFAA0EF20C0136FFBA47
:10D892000EF70C0177FFCA0EFC0C010001DA0E0133
:10D8A2000D01E50EE90EED0EF10EF50EF90EFD0E6F
:10D8B2000100000000E50B60666F000000002E6FA3
:10D8C2004FFFFFFFFFFFFFFFFFFFFFFFFF00000013
:10D8D20000523E606600004000140054001F1C1FEE
:10D8E2001E1F1E1F1F1E1F1E1F00000703050810FC
:10D8F20000000006091F00151500001F111F11135B
:10D902001E0014081501050515000000005F606087
:10D91200660000000088606066000000002261F17D
:10D9220060AA60B360C860D96000000000CB696083
:0AD93200665F6990697069B96900C9
:00000001FF
